S01900006D69785F73746174696F6E5F626F6172642E73726563F5
S3150802000000000A206D48060825F403082DF40308A3
S3150802001035F403083DF4030845F40308BD48060809
S31508020020000000000000000000000000BD480608AD
S315080200304DF4030800000000C9020208B1040208D0
S31508020040BD480608BD480608BD480608BD48060854
S31508020050BD480608BD480608BD480608BD48060844
S31508020060BD480608BD480608BD4806085BF40308ED
S31508020070BD48060869F40308BD480608BD480608CF
S31508020080BD480608BD480608BD480608BD48060814
S31508020090BD480608BD48060877F40308BD480608A1
S315080200A0BD480608BD480608BD480608BD480608F4
S315080200B0BD480608BD480608BD480608BD480608E4
S315080200C0BD480608BD480608BD480608BD480608D4
S315080200D000000000BD480608BD48060889F4030862
S315080200E0BD480608BD480608BD480608BD480608B4
S315080200F0BD480608BD480608BD480608BD480608A4
S31508020100BD4806089DF40308BD480608BD4806080A
S31508020110BD480608BD480608BD480608BD48060883
S31508020120BD480608BD480608D5F40308BD480608B2
S31508020130BD480608BD480608BD480608BD48060863
S31508020140BD480608BD480608BD480608BD48060853
S31508020150BD480608BD480608BD480608BD48060843
S31508020160BD480608BD480608BD480608BD48060833
S31508020170BD480608BD480608BD480608BD48060823
S31508020180BD480608BD480608BD480608BD48060813
S31508020190BD480608BD480608BD480608BD48060803
S315080201A0BD480608BD480608BD480608BD480608F3
S315080201B0BD480608BD480608BD480608BD480608E3
S315080201C0BD480608BD480608BD480608BD480608D3
S315080201D0BD480608BD480608BD480608BD480608C3
S315080201E0BD480608BD480608BD480608BD480608B3
S315080201F0BD480608BD480608BD480608BD480608A3
S31508020200BD480608BD480608BD48060800000000A5
S3150802021000000000BD48060800000000BD480608A8
S31508020220BD480608BD480608BD480608BD48060872
S31508020230BD480608BD480608BD480608BD48060862
S31508020240BD480608BD480608BD4806080000000065
S3150802025010B5054C237833B9044B13B10448AFF3F0
S3150802026000800123237010BD9814002000000000AE
S31508020270EC95070808B5034B1BB103490348AFF3CE
S31508020280008008BD000000009C140020EC950708B9
S31508020290EFF3108180F31088081C70474FF00000B6
S315080202A02D4A1060EFF3148020F0040080F31488BE
S315080202B062B64FF080504FF0E021C1F8040DBFF34B
S315080202C04F8FBFF36F8FFEE72448254A4FF000038E
S315080202D0016891B10360EFF3098C2CE9F00F1EF067
S315080202E0100F01D12CED108A1E4C4CF804EDC1F802
S315080202F008C025680DB18D61236072B61168D1B147
S31508020300016062B64F68174C8D6907F101074F60A5
S315080203102560D1F80CC08CF30B88D1F808C05CF8BC
S3150802032004EB1EF0100F01D1BCEC108ABCE8F00FEA
S315080203308CF30988704772B61168016009B962B60A
S31508020340F9E74FF000674FF0E028C8F8047D62B677
S31508020350D8E700BF7047000088150020F014002077
S31508020360F4140020F41A0020026922F00702A2F10E
S3150802037044026FF0430313604FF000035360936027
S31508020380D360136153619361D361136253629362BB
S31508020390D362136353634FF0FF339363D1634FF012
S315080203A080731364826070472249086800F101006D
S315080203B00860214B1A683AB1A2F101021A601AB909
S315080203C01E4B4FF0010018601D490868026822B1E9
S315080203D01C4B4FF001021A6008E000F104001A4BA8
S315080203E01A68904201D1194B18680860134B1A68AB
S315080203F012B914490868C8B101B51249086808B1A2
S315080204000EF070FB0D4B1A6872B10EF0DDFA104849
S31508020410016849B90F4801680F4A13680F484FF037
S315080204208052994200D00260BDE80140BFF34F8F67
S315080204307047000094150020F41A00209815002031
S315080204402416002028160020201600201C1600203C
S3150802045088150020F0140020F414002004ED00E0B2
S3150802046072B64FF0E0201749C0F8081D1648016811
S3150802047041F00101016015481249096801604FF00F
S31508020480E020134941614FF0070101614FF0000175
S31508020490C0F8181D4FF07F41C0F81C1D0D49C0F861
S315080204A0201D7047FFF7FEBF01B5BDE80140704742
S315080204B001B5FFF779FFBDE801407047FFF7FEBFB8
S315080204C0FFF7FEBF00000208001000E0EC1400204F
S315080204D08FD003000000FF40034613F8012B002AC1
S315080204E0FBD1181A0138704781F0004102E000BFBB
S315080204F083F0004330B54FEA41044FEA430594EAD4
S31508020500050F08BF90EA020F1FBF54EA000C55EA0E
S31508020510020C7FEA645C7FEA655C00F0E2804FEADF
S315080205205454D4EB5555B8BF6D420CDD2C4480EAC1
S31508020530020281EA030382EA000083EA010180EAF1
S31508020540020281EA0303362D88BF30BD11F0004F3F
S315080205504FEA01314FF4801C4CEA113102D0404275
S3150802056061EB410113F0004F4FEA03334CEA1333B0
S3150802057002D0524263EB430394EA050F00F0A780C8
S31508020580A4F10104D5F1200E0DDB02FA0EFC22FAC3
S3150802059005F2801841F1000103FA0EF2801843FAB7
S315080205A005F359410EE0A5F120050EF1200E012AA8
S315080205B003FA0EFC28BF4CF0020C43FA05F3C018E6
S315080205C051EBE37101F0004507D54FF0000EDCF15F
S315080205D0000C7EEB00006EEB0101B1F5801F1BD308
S315080205E0B1F5001F0CD349085FEA30004FEA3C0C0C
S315080205F004F101044FEA445212F5800F80F09A8002
S31508020600BCF1004F08BF5FEA500C50F1000041EB05
S31508020610045141EA050130BD5FEA4C0C404141EB09
S315080206200101013C28BFB1F5801FE9D291F0000F04
S3150802063004BF01460020B1FA81F308BF2033A3F1B3
S315080206400B03B3F120020CDA0C3208DD02F1140CAA
S31508020650C2F10C0201FA0CF021FA02F10CE002F1E5
S315080206601402D8BFC2F1200C01FA02F120FA0CFCDE
S31508020670DCBF41EA0C019040E41AA2BF01EB045127
S31508020680294330BD6FEA04041F3C1CDA0C340EDC25
S3150802069004F11404C4F1200220FA04F001FA02F368
S315080206A040EA030021FA04F345EA030130BDC4F126
S315080206B00C04C4F1200220FA02F001FA04F340EA1B
S315080206C00300294630BD21FA04F0294630BD94F0CC
S315080206D0000F83F4801306BF81F480110134013DB3
S315080206E04EE77FEA645C18BF7FEA655C29D094EA24
S315080206F0050F08BF90EA020F05D054EA000C04BFA2
S315080207001946104630BD91EA030F1EBF002100208C
S3150802071030BD5FEA545C05D14000494128BF41F02B
S31508020720004130BD14F580043CBF01F5801130BD8F
S3150802073001F0004545F0FE4141F470014FF000001A
S3150802074030BD7FEA645C1ABF194610467FEA655CCB
S315080207501CBF0B46024650EA013406BF52EA03356D
S3150802076091EA030F41F4002130BD00BF90F0000F5B
S3150802077004BF0021704730B54FF4806404F1320497
S315080207804FF000054FF0000150E700BF90F0000F50
S3150802079004BF0021704730B54FF4806404F1320477
S315080207A010F0004548BF40424FF000013EE700BF47
S315080207B042004FEAE2014FEA31014FEA02701FBFD7
S315080207C012F07F4393F07F4F81F06051704732F009
S315080207D07F4208BF704793F07F4F04BF41F4002160
S315080207E0704730B54FF4607401F0004521F00041BE
S315080207F01CE700BF50EA010208BF704730B54FF048
S3150802080000050AE050EA010208BF704730B511F048
S31508020810004502D5404261EB41014FF4806404F180
S3150802082032045FEA915C3FF4D8AE4FF003025FEA06
S31508020830DC0C18BF03325FEADC0C18BF033202EB8A
S31508020840DC02C2F1200300FA03FC20FA02F001FAE4
S3150802085003FE40EA0E0021FA02F11444BDE600BF87
S3150802086070B54FF0FF0C4CF4E06C1CEA11541DBF36
S315080208701CEA135594EA0C0F95EA0C0F00F0DEF801
S315080208802C4481EA030621EA4C5123EA4C5350EAE6
S31508020890013518BF52EA033541F4801143F4801337
S315080208A038D0A0FB02CE4FF00005E1FB02E506F0C8
S315080208B00042E0FB03E54FF00006E1FB03569CF01D
S315080208C0000F18BF4EF0010EA4F1FF04B6F5007F23
S315080208D064F5407404D25FEA4E0E6D4146EB060695
S315080208E042EAC62141EA55514FEAC52040EA5E501E
S315080208F04FEACE2EB4F1FD0C88BFBCF5E06F1ED8C8
S31508020900BEF1004F08BF5FEA500E50F1000041EBFE
S31508020910045170BD06F0004646EA010140EA0200AB
S3150802092081EA0301B4EB5C04C2BFD4EB0C0541EACD
S31508020930045170BD41F480114FF0000E013C00F3E2
S31508020940AB8014F1360FDEBF002001F0004170BD06
S31508020950C4F10004203C35DA0C341BDC04F114041F
S31508020960C4F1200500FA05F320FA04F001FA05F2AB
S3150802097040EA020001F0004221F0004110EBD37078
S3150802098021FA04F642EB06015EEA430E08BF20EAA4
S31508020990D37070BDC4F10C04C4F1200500FA04F347
S315080209A020FA05F001FA04F240EA020001F00041D9
S315080209B010EBD37041F100015EEA430E08BF20EA4C
S315080209C0D37070BDC4F1200500FA05F24EEA020E94
S315080209D020FA04F301FA05F243EA020321FA04F0C3
S315080209E001F0004121FA04F220EA020000EBD3707A
S315080209F05EEA430E08BF20EAD37070BD94F0000F7A
S31508020A000FD101F00046400041EB010111F4801FAD
S31508020A1008BF013CF7D041EA060195F0000F18BF5E
S31508020A20704703F00046520043EB030313F4801F9A
S31508020A3008BF013DF7D043EA0603704794EA0C0F54
S31508020A400CEA135518BF95EA0C0F0CD050EA41066A
S31508020A5018BF52EA4306D1D181EA030101F00041E7
S31508020A604FF0000070BD50EA410606BF104619460F
S31508020A7052EA430619D094EA0C0F02D150EA01361B
S31508020A8013D195EA0C0F05D152EA03361CBF10465C
S31508020A9019460AD181EA030101F0004141F0FE41FB
S31508020AA041F470014FF0000070BD41F0FE4141F47F
S31508020AB0780170BD70B54FF0FF0C4CF4E06C1CEA7F
S31508020AC011541DBF1CEA135594EA0C0F95EA0C0F34
S31508020AD000F0A7F8A4EB050481EA030E52EA0335EF
S31508020AE04FEA013100F088804FEA03334FF0805510
S31508020AF045EA131343EA12634FEA022245EA11153D
S31508020B0045EA10654FEA00260EF000419D4208BFED
S31508020B10964244F1FD0404F5407402D25B084FEA9A
S31508020B203202B61A65EB03055B084FEA32024FF446
S31508020B3080104FF4002CB6EB020E75EB030E22BFA3
S31508020B40B61A754640EA0C005B084FEA3202B6EB63
S31508020B50020E75EB030E22BFB61A754640EA5C0012
S31508020B605B084FEA3202B6EB020E75EB030E22BFA2
S31508020B70B61A754640EA9C005B084FEA3202B6EBA3
S31508020B80020E75EB030E22BFB61A754640EADC0062
S31508020B9055EA060E18D04FEA051545EA16754FEAC4
S31508020BA006164FEAC30343EA52734FEAC2025FEAE2
S31508020BB01C1CC0D111F4801F0BD141EA00014FF071
S31508020BC000004FF0004CB6E711F4801F04BF014342
S31508020BD00020B4F1FD0C88BFBCF5E06F3FF6AFAE5E
S31508020BE0B5EB030C04BFB6EB020C5FEA500C50F1EE
S31508020BF0000041EB045170BD0EF0004E4EEA113171
S31508020C0014EB5C04C2BFD4EB0C0541EA045170BD77
S31508020C1041F480114FF0000E013C90E645EA060EBB
S31508020C208DE60CEA135594EA0C0F08BF95EA0C0FE9
S31508020C303FF43BAF94EA0C0F0AD150EA01347FF431
S31508020C4034AF95EA0C0F7FF425AF104619462CE708
S31508020C5095EA0C0F06D152EA03353FF4FDAE10466B
S31508020C60194622E750EA410618BF52EA43067FF4BC
S31508020C70C5AE50EA41047FF40DAF52EA43057FF44C
S31508020C80EBAE12E74FF0FF3C06E000BF4FF0010C57
S31508020C9002E000BF4FF0010C4DF804CD4FEA410CBB
S31508020CA07FEA6C5C4FEA430C18BF7FEA6C5C1BD088
S31508020CB001B050EA410C0CBF52EA430C91EA030F09
S31508020CC002BF90EA020F0020704710F1000F91EA66
S31508020CD0030F58BF994208BF90422CBFD8176FEA34
S31508020CE0E37040F0010070474FEA410C7FEA6C5C02
S31508020CF002D150EA013C07D14FEA430C7FEA6C5C09
S31508020D00D6D152EA033CD3D05DF8040B704700BF34
S31508020D108446104662468C461946634600E000BF82
S31508020D2001B5FFF7B7FF002848BF10F1000F01BD54
S31508020D304DF808EDFFF7F4FF0CBF012000205DF81F
S31508020D4008FB00BF4DF808EDFFF7EAFF34BF0120A4
S31508020D5000205DF808FB00BF4DF808EDFFF7E0FF3D
S31508020D6094BF012000205DF808FB00BF4DF808ED8E
S31508020D70FFF7CEFF94BF012000205DF808FB00BFF5
S31508020D804DF808EDFFF7C4FF34BF012000205DF8D7
S31508020D9008FB00BF4FEA410C7FEA6C5C02D150EABD
S31508020DA0013C0AD14FEA430C7FEA6C5C02D152EA53
S31508020DB0033C02D14FF0000070474FF00100704724
S31508020DC04FEA410212F5001215D211D56FF4787363
S31508020DD0B3EB625212D94FEAC12343F0004343EA06
S31508020DE0505311F0004F23FA02F018BF40427047E1
S31508020DF04FF00000704750EA013005D111F000406B
S31508020E0008BF6FF0004070474FF00000704700BF00
S31508020E104A0011D212F5001211D20DD56FF4787369
S31508020E20B3EB62520ED44FEAC12343F0004343EABE
S31508020E30505323FA02F070474FF00000704750EA09
S31508020E40013002D14FF0FF3070474FF00000704773
S31508020E504FEA4102B2F1E04324BFB3F5001CDCF1CC
S31508020E60FE5C0DD901F0004C4FEAC0024CEA507004
S31508020E70B2F1004F40EB830008BF20F00100704733
S31508020E8011F0804F21D113F13872BCBF01F0004036
S31508020E90704741F480114FEA5252C2F11802C2F168
S31508020EA0200C10FA0CF320FA02F018BF40F00100E9
S31508020EB04FEAC1234FEAD32303FA0CFC40EA0C009B
S31508020EC023FA02F34FEA4303CCE77FEA625307D1D8
S31508020ED050EA01331EBF4FF0FE4040F4400070470F
S31508020EE001F0004040F0FE4040F40000704700BFA9
S31508020EF053B94AB9002908BF00281CBF4FF0FF3171
S31508020F004FF0FF3000F0B4B9ADF1080C6DE904CE2C
S31508020F1000F03CF8DDF804E0DDE9022304B070478E
S31508020F2038B50022002304460D46FFF70BFF28B901
S31508020F3020462946BDE8384000F00AB8204605F1A1
S31508020F40004100F005F8404261EB410138BD00BF9F
S31508020F50D0B500220B4B06460F46FFF781FCFFF77A
S31508020F6057FF0446FFF702FC0022074BFFF778FCFF
S31508020F7002460B4630463946FFF7BAFAFFF748FFEC
S31508020F802146D0BD0000F03D0000F0412DE9F04FAA
S31508020F90099D0C46002B4DD18A420F468446964639
S31508020FA0B2FA82F360D94BB102FA03FEC3F1200208
S31508020FB09F4000FA03FC20FA02F217434FEA1E4644
S31508020FC01FFA8EF44FEA1C42B7FBF6F106FB1177BD
S31508020FD001FB04F042EA0742904208D91EEB0202DC
S31508020FE001F1FF3702D2904200F22D813946121AD8
S31508020FF01FFA8CFCB2FBF6F006FB102200FB04F487
S315080210004CEA024C644508D91EEB0C0C00F1FF327F
S3150802101002D2644500F21A81104640EA0140ACEB5E
S31508021020040C002125B12CFA03F30022C5E900328B
S31508021030BDE8F08F8B4205D90DB1C5E90001002143
S315080210400846F5E7B3FA83F100294DD1A342C0F069
S31508021050F280904280F0EF80064623460846002D2D
S31508021060E6D0C5E90063E3E7002B40F0A2808A1ABE
S315080210704FEA1E471FFA8EF60121B2FBF7F407FB69
S3150802108014204FEA1C4242EA004206FB04F0904250
S315080210900FD91EEB020204F1FF382CBF4FF00109EB
S315080210A04FF00009904203D9B9F1000F00F0C88049
S315080210B04446121A1FFA8CFCB2FBF7F007FB102201
S315080210C000FB06F64CEA024C664508D91EEB0C0CE8
S315080210D000F1FF3202D2664500F2BB801046ACEB45
S315080210E0060C40EA04409DE7C1F120068B4004FA4B
S315080210F001FE22FA06F720FA06FCF4408A401F434C
S315080211004EEA0C0300FA01FE4FEA17484FEA134962
S315080211101FFA87FCB4FBF8F008FB104449EA0444BA
S3150802112000FB0CF9A1450ED93C1900F1FF3A2CBF78
S315080211304FF0010B4FF0000BA14503D9BBF1000F8D
S3150802114000F093805046A4EB09041FFA83F9B4FB16
S31508021150F8F308FB134403FB0CFC49EA0444A445D0
S3150802116006D93C1903F1FF3801D2A4457AD8434679
S3150802117043EA0040A4EB0C04A0FB02984445CC4683
S31508021180434602D306D1CE4504D20138B9EB020C46
S3150802119068EB07035DB1BEEB0C0264EB030404FAC9
S315080211A006F622FA01F3CC401E43C5E90064002183
S315080211B03EE702FA03FEC3F1200104FA03F200FA3B
S315080211C003FCCC404FEA1E4720FA01F11FFA8EF6BD
S315080211D0B4FBF7F00A4307FB1044110C41EA044139
S315080211E000FB06F48C420ED91EEB010100F1FF3812
S315080211F02CBF4FF001094FF000098C4202D9B9F110
S31508021200000F2CD04046091B92B2B1FBF7F407FB3C
S31508021210141142EA014204FB06F1914207D91EEB78
S31508021220020204F1FF3801D2914215D84446521AF5
S3150802123044EA004121E7861A64EB030301200EE71C
S31508021240023C724435E702397244D0E6F444023865
S31508021250E3E6F444023842E7023C7244E7E702381E
S315080212607144D0E7023B3C4482E702383C446AE7D1
S31508021270704700BF80B500AF032000F012F902F0F4
S3150802128011FD02460B4B1B6A03F00F030A49CB5C9E
S3150802129022FA03F3094A13600F201EF04DF803469B
S315080212A0002B01D0012302E01DF0AEFD00231846F3
S315080212B080BD00BF000C0244DC8D0808C412002061
S315080212C080B400AF064B1B781A46064B1B681344BC
S315080212D0044A136000BFBD465DF8047B704700BF31
S315080212E004000020B414002080B400AF034B1B682E
S315080212F01846BD465DF8047B704700BFB41400204B
S3150802130080B485B000AF78607B6803F00703FB60A2
S315080213100C4BDB68BB60BA684FF6FF031340BB6031
S31508021320FB681A02BB68134343F0BF6343F40033F6
S31508021330BB60044ABB68D36000BF1437BD465DF87C
S31508021340047B704700ED00E080B400AF044BDB6815
S315080213501B0A03F007031846BD465DF8047B70476F
S3150802136000ED00E080B483B000AF0346FB80B7F916
S315080213700630002B0BDBFB8803F01F020749B7F97F
S3150802138006305B09012000FA02F241F8232000BF69
S315080213900C37BD465DF8047B704700BF00E100E0EC
S315080213A080B483B000AF0346FB80B7F90630002B42
S315080213B012DBFB8803F01F020A49B7F906305B09FC
S315080213C0012000FA02F2203341F82320BFF34F8F9F
S315080213D000BFBFF36F8F00BF00BF0C37BD465DF875
S315080213E0047B704700E100E080B483B000AF034697
S315080213F03960FB80B7F90630002B0ADB3B68DAB2A4
S315080214000C49B7F906301201D2B20B4483F800230D
S315080214100AE03B68DAB20849FB8803F00F03043B8B
S315080214201201D2B20B441A7600BF0C37BD465DF8DC
S31508021430047B704700E100E000ED00E080B489B06B
S3150802144000AFF860B9607A60FB6803F00703FB61D6
S31508021450FB69C3F10703042B28BF0423BB61FB699D
S315080214600433062B02D9FB69033B00E000237B61A8
S315080214704FF0FF32BB6902FA03F3DA43BB681A403C
S315080214807B699A404FF0FF317B6901FA03F3D9432E
S315080214907B680B40134318462437BD465DF8047B28
S315080214A0704780B582B000AF78607868FFF728FF8A
S315080214B000BF0837BD4680BD80B586B000AF03467B
S315080214C0B9607A60FB81FFF73FFF78617A68B9688D
S315080214D07869FFF7B3FF0246B7F90E301146184688
S315080214E0FFF782FF00BF1837BD4680BD80B582B0C0
S315080214F000AF0346FB80B7F906301846FFF732FFFE
S3150802150000BF0837BD4680BD80B582B000AF03462E
S31508021510FB80B7F906301846FFF742FF00BF0837C7
S31508021520BD4680BD80B584B000AF7860FFF7DCFEAB
S31508021530F8607B68002B01D101236BE07B6893F886
S315080215405430DBB2022B08D07B6820229A657B686E
S31508021550002283F84C2001235CE07B681B685A69E9
S315080215607B681B6842F004025A617B68052283F88D
S31508021570542020E0FFF7B8FE0246FB68D31A052B73
S3150802158019D97B689B6D43F010027B689A657B6864
S31508021590032283F854207B681B6D03F08003002B1B
S315080215A003D07B685B6F01221A737B68002283F87B
S315080215B04C2001232EE07B681B681B6903F4005349
S315080215C0002BD7D07B681B685A697B681B6842F078
S315080215D002025A617B68042283F854207B681B68DE
S315080215E04FF4FE42DA607B68012283F854207B6856
S315080215F01B6D03F08003002B07D07B685B6F01220B
S315080216001A737B681B6800229A647B68002283F837
S315080216104C20002318461037BD4680BD80B483B0DF
S3150802162000AF78607B68002B01D1012319E07B6843
S3150802163093F85430DBB2022B04D07B6820229A65D9
S3150802164001230EE07B68042283F854207B681B681A
S315080216505B697A68126843F4005343F004035361E2
S31508021660002318460C37BD465DF8047B7047000018
S3150802167080B584B000AF78607B68002B01D1012366
S3150802168047E17B6893F85C30DBB2002B06D17B68B6
S31508021690002283F85D2078681DF0BEFB7B681B6814
S315080216A09A697B681B6822F010029A61FFF71CFE92
S315080216B0F86012E0FFF718FE0246FB68D31A0A2BF7
S315080216C00BD97B681B6E43F001027B681A667B683E
S315080216D0032283F85C2001231BE17B681B689B6954
S315080216E003F00803082BE5D07B681B689A697B68B8
S315080216F01B6842F001029A61FFF7F6FDF86012E0F4
S31508021700FFF7F2FD0246FB68D31A0A2B0BD97B6850
S315080217101B6E43F001027B681A667B68032283F814
S315080217205C200123F5E07B681B689B6903F00103D3
S31508021730002BE5D07B681B689A697B681B6842F0B8
S3150802174002029A617B681B68744A934203D1744AFF
S315080217507B685B6813607B681B7C012B08D17B68FE
S315080217601B689A697B681B6822F040029A6107E047
S315080217707B681B689A697B681B6842F040029A611B
S315080217807B685B7C012B08D17B681B689A697B683E
S315080217901B6842F480429A6107E07B681B689A6973
S315080217A07B681B6822F480429A617B689B7C012BCA
S315080217B008D17B681B689A697B681B6822F4805289
S315080217C09A6107E07B681B689A697B681B6842F422
S315080217D080529A617B681B689B6923F440717B6817
S315080217E09A687B681B680A439A617B681B689A69D0
S315080217F07B681B6822F0A4029A617B681B681A69D7
S315080218007B681B6822F010021A617B68DB68012B71
S3150802181008D17B681B689A697B681B6842F00402D8
S315080218209A612CE07B68DB68002B28D07B68DB6832
S31508021830022B1CD07B681B689A697B681B6842F07E
S3150802184080029A617B681B681A697B681B6842F08A
S3150802185010021A617B68DB68032B10D17B681B6850
S315080218609A697B681B6842F020029A6107E07B68E6
S315080218701B689A697B681B6842F020029A617B683A
S315080218809B69013B5A067B68DB69013B1B021A43CB
S315080218907B681B6A013B42EA03017B685B69013B81
S315080218A01A047B681B680A43DA617B689B68B3F58E
S315080218B0407F15D17B689B6A5A1E7B68DB6A013BAF
S315080218C01B021A437B681B6B013B1B0142EA03019D
S315080218D07B685B6A013B1A047B681B680A43DA6009
S315080218E07B681B68D3F8C0107B68DA6B7B681B6859
S315080218F00A43C3F8C020786800F036FD7B680022E8
S315080219009A657B6800221A667B68012283F85C2046
S31508021910002318461037BD4680BD00BF00A400400C
S3150802192000A5004080B487B000AF786039607B6854
S3150802193093F85C30FB75FB7D012B02D0FB7D022BF5
S315080219403DD13B681B68002B19D13B689B689A07F7
S315080219503B68DB68DB061A433B681B691B041A43B0
S315080219603B685B6913433B617B681A6C3B685B683F
S315080219709B001344BB60BB683A691A601DE03B686A
S31508021980DB685A073B681B6913433B613B689B68E4
S315080219909A073B685B691343FB607B685A6C3B6832
S315080219A05B68DB001344BB60BB683A691A60BB68B4
S315080219B00433BB60BB68FA681A60002306E07B68DA
S315080219C01B6E43F002027B681A66012318461C370F
S315080219D0BD465DF8047B704780B485B000AFF860F9
S315080219E0B9607A603B60FB6893F85C30DBB2012B26
S315080219F016D1FB681B68D3F8803023F03F01BB6819
S31508021A001A017B689B001A433B685B001A43BB6951
S31508021A101A43FB681B680A43C3F88020002306E0C2
S31508021A20FB681B6E43F00402FB681A66012318461C
S31508021A301437BD465DF8047B704780B483B000AFA7
S31508021A4078607B6893F85C30DBB2012B10D17B6837
S31508021A50022283F85C207B681B689A697B681B688C
S31508021A6022F001029A617B6800221A66002306E0C8
S31508021A707B681B6E43F004027B681A6601231846CC
S31508021A800C37BD465DF8047B704780B586B000AF5B
S31508021A90F860B9607A60FB6893F85C30DBB2022BB7
S31508021AA02CD1FB681B68D3F8C43003F40013002B4F
S31508021AB007D0FB681B6E43F40072FB681A660123A3
S31508021AC023E0FB681B68D3F8C4301B0C03F003033E
S31508021AD07B617B697A68B968F86800F0A7FCFB68DD
S31508021AE01B6801217A6901FA02F2C3F8CC200122A5
S31508021AF07B699A40FB689A65002306E0FB681B6EC1
S31508021B0043F00802FB681A66012318461837BD46D1
S31508021B1080BD80B483B000AF78607B689B6D184641
S31508021B200C37BD465DF8047B704780B483B000AFBE
S31508021B30786039607B6893F85C30DBB2022B06D199
S31508021B407B681B683A68C3F8D020002306E07B68E6
S31508021B501B6E43F008027B681A66012318460C3787
S31508021B60BD465DF8047B704780B48BB000AFF86061
S31508021B70B9607A603B600023FB61FB6893F85C30CE
S31508021B80FB76FB7E022B40F0E880BB68402B37D100
S31508021B90FB681B68D3F8903003F00F03002B07D1BC
S31508021BA0FB681B6E43F48072FB681A660123DBE04E
S31508021BB0FB681B68D3F890301B0E03F00103012B58
S31508021BC00AD1FB681B68D3F880305B0A03F001036D
S31508021BD0012B01D10123FB61FB681B68D3F8903006
S31508021BE01B0A03F00303FA691344FB61FB68996C49
S31508021BF0FA691346DB001344DB000B447B6236E0CA
S31508021C00FB681B68D3F8983003F00F03002B07D143
S31508021C10FB681B6E43F48072FB681A660123A3E015
S31508021C20FB681B68D3F898301B0E03F00103012BDF
S31508021C300AD1FB681B68D3F880301B0A03F001033C
S31508021C40012B01D10123FB61FB681B68D3F898308D
S31508021C501B0A03F00303FA691344FB61FB68D96C98
S31508021C60FA691346DB001344DB000B447B627B6A8A
S31508021C701B6803F080427B685A607B685B68002BAE
S31508021C8007D17B6A1B689B0CC3F30A027B681A603E
S31508021C9005E07B6A1B6823F060427B681A607B6AF0
S31508021CA01B6803F000527B689A607B6A1B6803F024
S31508021CB000427B681A617B6A04337B627B6A1B6813
S31508021CC09AB27B68DA617B6A1B681B0C03F00F0207
S31508021CD07B68DA607B6A1B6803F480127B685A6148
S31508021CE07B6A1B6803F400127B689A617B6A1B682D
S31508021CF01B0E03F07F027B681A627B6A1B68DA0F87
S31508021D007B685A627B6A04337B627B6A7B61002347
S31508021D103B620AE07A693B6A1A4439683B6A0B44B1
S31508021D2012781A703B6A01333B627B68DB68114A98
S31508021D30D35C1A463B6A9342ECD3BB68402B05D167
S31508021D40FB681B68FA69C3F8942004E0FB681B6801
S31508021D50FA69C3F89C20002306E0FB681B6E43F071
S31508021D600802FB681A66012318462C37BD465DF839
S31508021D70047B7047A48D080880B485B000AF7860EC
S31508021D8039607B681B685B6CFB60FB6803F00702C3
S31508021D903B681A60FB681B0A03F007023B685A6035
S31508021DA0FB6803F018023B689A60FB685B0903F05C
S31508021DB001023B68DA60FB689B0903F001023B6893
S31508021DC01A61FB68DB0903F001023B685A61FB688A
S31508021DD0DB0A03F001023B689A61FB681B0B03F0FE
S31508021DE001023B68DA61FB685B0B03F001023B68A0
S31508021DF01A62FB689B0B03F001023B685A62FB6896
S31508021E001B0C03F07F023B689A62002318461437BC
S31508021E10BD465DF8047B704780B483B000AF786036
S31508021E2039607B681B68D3F8C8203B681340002BCF
S31508021E3001D1002300E0012318460C37BD465DF8A0
S31508021E40047B704780B485B000AF786039603B6820
S31508021E50402B07D17B681B68D3F8903003F00F0339
S31508021E60FB6006E07B681B68D3F8983003F00F0323
S31508021E70FB60FB6818461437BD465DF8047B70475D
S31508021E8080B487B000AFF860B9607A60FB6893F8EF
S31508021E905C30FB75FB7D012B03D0FB7D022B40F0EA
S31508021EA0C880FB681B689B6D3B61BB6803F0070330
S31508021EB0002B04D03B6903F00103002B3BD0BB681F
S31508021EC003F03803002B04D03B6903F00203002B0E
S31508021ED031D0BB6803F4E073002B04D03B6903F0EE
S31508021EE00403002B27D0BB6803F4F053002B04D05D
S31508021EF03B6903F00803002B1DD0BB6803F460435B
S31508021F00002B04D03B6903F01003002B13D0BB68E7
S31508021F1003F44033002B04D03B6903F02003002B63
S31508021F2009D0BB6803F47C03002B0CD03B6903F091
S31508021F304003002B07D1FB681B68DA6DFB681B6838
S31508021F4042F00102DA65BB6803F00703002B04D0EE
S31508021F503B6903F00103002B3BD1BB6803F038034E
S31508021F60002B04D03B6903F00203002B31D1BB6876
S31508021F7003F4E073002B04D03B6903F00403002B3F
S31508021F8027D1BB6803F4F053002B04D03B6903F056
S31508021F900803002B1DD1BB6803F46043002B04D051
S31508021FA03B6903F01003002B13D1BB6803F44033DB
S31508021FB0002B04D03B6903F02003002B09D1BB6830
S31508021FC003F47C03002B0CD03B6903F04003002B7F
S31508021FD007D0FB681B68DA6DFB681B6842F00202D1
S31508021FE0DA65BB6803F08003002B09D0FB681B681F
S31508021FF0D3F8DC10FB681B687A680A43C3F8DC204E
S31508022000BB6803F48073002B09D0FB681B68D3F8FE
S31508022010E010FB681B687A680A43C3F8E020FB688D
S315080220201B68596DFB681B68BA680A435A65002320
S3150802203006E0FB681B6E43F00202FB681A66012380
S3150802204018461C37BD465DF8047B704780B58CB0D0
S3150802205000AF78607B681B681B6D03F4E053FB6274
S315080220607B681B685B6DFA6A1340FB627B681B68B8
S315080220701B6D03F00703BB627B681B685B6DBA6A5C
S315080220801340BB627B681B681B6D03F038037B62D7
S315080220907B681B685B6D7A6A13407B627B681B6888
S315080220A01B6D03F471033B627B681B685B6D3A6ABE
S315080220B013403B627B681B681B6D03F46023FB615C
S315080220C07B681B685B6DFA691340FB617B681B685A
S315080220D05B6DBB617B681B681B6D7B617B6903F06B
S315080220E04003002B0BD0BB6903F04003002B06D03C
S315080220F07B681B6840221A65786800F016F97B69C6
S3150802210003F48073002B19D0BB6903F48073002B88
S3150802211014D07B681B68D3F8D8303B617B681B6890
S31508022120D3F8E0303A6913403B617B681B684FF489
S3150802213080721A653969786800F0D8F8FB6A002B4C
S3150802214007D07B681B68FA6A1A65F96A786800F02C
S31508022150A2F8BB6A002B07D07B681B68BA6A1A65A5
S31508022160B96A78681AF020F87B6A002B07D07B6870
S315080221701B687A6A1A65796A786800F097F87B6943
S3150802218003F40073002B0CD0BB6903F40073002B15
S3150802219007D07B681B684FF400721A65786800F0EE
S315080221A090F87B6903F08003002B18D0BB6903F013
S315080221B08003002B13D07B681B68D3F8D430FB60EE
S315080221C07B681B68D3F8DC30FA681340FB607B68CF
S315080221D01B6880221A65F968786800F07CF87B69C2
S315080221E003F40053002B0CD0BB6903F40053002BF5
S315080221F007D07B681B684FF400521A65786800F0AE
S3150802220080F87B6903F40043002B0CD0BB6903F406
S315080222100043002B07D07B681B684FF400421A65FF
S31508022220786800F078F87B6903F48043002B0FD0B6
S31508022230BB6903F48043002B0AD07B681B684FF402
S3150802224080421A657B681B6E43F080027B681A66B9
S31508022250FB69002B07D07B681B68FA691A65F9695E
S31508022260786800F076F83B6A002B09D07B681B6811
S315080222703A6A1A657B681A6E3B6A1A437B681A665B
S315080222807B681B6E002B02D0786800F058F800BFF6
S315080222903037BD4680BD80B483B000AF7860396000
S315080222A000BF0C37BD465DF8047B704780B483B027
S315080222B000AF7860396000BF0C37BD465DF8047B15
S315080222C0704780B483B000AF786000BF0C37BD4654
S315080222D05DF8047B704780B483B000AF78603960DC
S315080222E000BF0C37BD465DF8047B704780B483B0E7
S315080222F000AF7860396000BF0C37BD465DF8047BD5
S31508022300704780B483B000AF786000BF0C37BD4613
S315080223105DF8047B704780B483B000AF786000BF75
S315080223200C37BD465DF8047B704780B483B000AFB6
S31508022330786000BF0C37BD465DF8047B704780B4F1
S3150802234083B000AF786000BF0C37BD465DF8047BEA
S31508022350704780B483B000AF7860396000BF0C372D
S31508022360BD465DF8047B704780B485B000AF7860DF
S315080223702C4BBB607B681B682B4A934203D1BB6814
S3150802238003F55473BB607B68BA681A647B681B687A
S31508022390D3F8803023F4F8117B685B6B1A047B68E8
S315080223A01B680A43C3F88020BB6803F170027B6886
S315080223B05A647B681B68D3F8803023F070617B68A7
S315080223C09B6B1A067B681B680A43C3F88020BB68A6
S315080223D003F1B0027B689A64BB6803F5C4727B6832
S315080223E0DA64BB6803F518727B681A65BB6803F57D
S315080223F01E727B685A65BB68FB6005E0FB680022B3
S315080224001A60FB680433FB60BB6803F55473FA6809
S315080224109A42F3D300BF00BF1437BD465DF8047B6A
S31508022420704700BF00AC004000A8004080B489B0E5
S3150802243000AFF860B9607A603B60BB685B68002BE6
S315080224400AD1BB681A69BB689B681A43BB681B68D2
S315080224509B041343FB610AE0BB681A69BB689B6865
S315080224601A43BB681B68134343F08043FB61BB688E
S315080224701B6A1A06BB68DB691A43BB689B691A435F
S31508022480BB685B691A43BB68DB681B0413433B6181
S31508022490FB68596D3A681346DB001344DB000B44AC
S315080224A0BB61BB69FA691A60BB690433BB61BB6964
S315080224B03A691A60BB690433BB6100237B6120E079
S315080224C07B6903337A6813441B781A067B690233DD
S315080224D079680B441B781B041A437B6901337968B4
S315080224E00B441B781B02134379687A690A441278EB
S315080224F01A43BB691A60BB690433BB617B6904333F
S315080225007B61BB68DB68064AD35C1A467B699342E1
S31508022510D6D300BF00BF2437BD465DF8047B70479B
S31508022520A48D080880B588B000AFF860B9607A60F3
S31508022530324B1B78012B01D102235AE02F4B012281
S315080225401A702E4B00225A604FF47A7000F0A4F8E3
S315080225500346FB77FB7F002B47D1284AFB6893602B
S31508022560274BBB61FB6823F00043022B04D1796831
S31508022570B86800F0DFF81BE0FB68224A934203D0F2
S31508022580FB68214A934204D17968B86800F00EF9CB
S315080225900EE0FB6823F000431C4A934204D1796893
S315080225A0B86800F04FF903E07968B86800F04AF9AC
S315080225B04FF47A7000F070F80346FB77BB691A6825
S315080225C0FB6823F0304323F00403DB431A40BB695C
S315080225D01A60FB680C4A934207D10D4B7B617B69F3
S315080225E01B6823F004027B691A60044B00221A70E6
S315080225F0FB7F18462037BD4680BD00BF0800002075
S3150802260028200240020000100600001002000040C6
S315080226104020024080B483B000AF0023FB710D4B0B
S315080226209B6A03F00103002B0DD00A4B0A4A5A6033
S31508022630084B0A4A5A60074B9B6A03F00103002BB0
S3150802264001D00123FB71FB7918460C37BD465DF8AC
S31508022650047B70470020024023016745AB89EFCD12
S3150802266080B483B000AF0023FB710A4B9B6A094A08
S3150802267043F001039362074B9B6A03F00103002BA5
S3150802268001D10123FB71FB7918460C37BD465DF86B
S31508022690047B70470020024080B586B000AF7860A0
S315080226A0FEF722FE7861204B3B6110E07B68B3F1AE
S315080226B0FF3F0CD0FEF718FE02467B69D31A7A68EA
S315080226C09A4202D37B68002B01D1032327E03B6998
S315080226D01B6803F00B03002BE8D1144BFB603B6924
S315080226E01B6803F47E03BB60BB68002B0CD0104B3F
S315080226F05A68BB6813430E4A5360BB6803F47E02EA
S31508022700FB681A6001230AE03B691B6803F48033FD
S31508022710002B03D0FB684FF480321A600023184658
S315080227201837BD4680BD00BF202002403020024037
S315080227300800002080B48BB000AF786039600423AB
S3150802274087F827307B683B623B68FB61164BBB61A7
S31508022750BB691B6843F00202BB691A60EFF3108378
S315080227603B613B697B6172B600BFFB691A683B6ACB
S315080227701A603B6A04333B62FB690433FB6197F8D0
S315080227802730013B87F8273097F82730002BECD102
S315080227907B69FB60FB6883F3108800BF00BF2C3798
S315080227A0BD465DF8047B70472820024080B48BB092
S315080227B000AF78603960042387F827307B683B626C
S315080227C03B68FB611C4BBB611C4B7B61BB691B688D
S315080227D043F00202BB691A607B691A68184B9B6848
S315080227E003F004031A437B691A60EFF31083FB6054
S315080227F0FB683B6172B600BFFB691A683B6A1A60DE
S315080228003B6A04333B62FB690433FB6197F8273062
S31508022810013B87F8273097F82730002BECD13B6924
S31508022820BB60BB6883F3108800BF00BF2C37BD4668
S315080228305DF8047B704700BF282002404020024012
S315080228400800002080B485B000AF78603960094B73
S31508022850FB60FB681B6843F00202FB681A603A6871
S315080228607B68128892B21A8000BF1437BD465DF89B
S31508022870047B70472820024080B586B000AF786096
S3150802288039603A4B1B78012B01D102236AE0374B98
S3150802289001221A70354B00225A604FF47A70FFF7FC
S315080228A0FBFE0346FB75FB7D002B57D17B681B6835
S315080228B02E4A93602E4BFB607B681B6823F000430D
S315080228C048F2080293420BD17B685B68184600F00F
S315080228D053F84FF47A70FFF7DFFE0346FB7533E0D1
S315080228E07B681B68234A934208D100F0B5F84FF477
S315080228F07A70FFF7D1FE0346FB7525E03B684FF079
S31508022900FF321A607B689B683B6115E07B685B68EF
S315080229101946386900F068F84FF47A70FFF7BCFE7A
S315080229200346FB75FB7D002B03D03B683A691A60A8
S315080229300AE03B6901333B617B68DA687B689B681E
S3150802294013443A699A42E1D3FB681A687B681B68A2
S3150802295023F00043DB431A40FB681A60034B00224C
S315080229601A70FB7D18461837BD4680BD0800002040
S31508022970282002400800008080B485B000AF786045
S31508022980184BFB607B6803F00303032B08D1FB6833
S315080229901B6843F4004343F02003FA6813601BE004
S315080229A07B6803F00103002B09D0FB681B6823F040
S315080229B0004323F0280343F02802FB681A607B6869
S315080229C003F00203002B07D0FB681B6843F00043A1
S315080229D043F02803FA68136000BF1437BD465DF852
S315080229E0047B70472820024080B485B000AF786027
S315080229F03960184BFB603B6803F00103002B11D0CA
S31508022A00FB681B6823F0004323F4FE53FA6813603D
S31508022A10FB681A687B689B01134343F02402FB6830
S31508022A201A6010E0FB681B6823F4FE52FB681A6002
S31508022A30FB681A687B689B01134343F0004343F023
S31508022A402403FA68136000BF1437BD465DF8047B99
S31508022A50704700BF2820024080B483B000AF074BFE
S31508022A607B607B681B6843F008027B681A6000BFBC
S31508022A700C37BD465DF8047B704700BF4020024014
S31508022A8080B487B000AF7860396000233B6136E1D5
S31508022A903B681A6801213B6901FA03F31340FB609C
S31508022AA0FB68002B00F028813B685B68022B03D089
S31508022AB03B685B68122B25D13B69DA087B680832CA
S31508022AC053F822307B613B6903F007039B000F2210
S31508022AD002FA03F3DB437A6913407B613B681B699D
S31508022AE003F00F023B6903F007039B0002FA03F3A4
S31508022AF07A6913437B613B69DA087B68083279692C
S31508022B0043F822107B681B687B613B695B000322E2
S31508022B1002FA03F3DB437A6913407B613B685B681D
S31508022B2003F003023B695B0002FA03F37A69134373
S31508022B307B617B687A691A603B685B68012B0BD0FC
S31508022B403B685B68022B07D03B685B68112B03D096
S31508022B503B685B68122B30D17B689B687B613B695B
S31508022B605B00032202FA03F3DB437A6913407B61B3
S31508022B703B68DA683B695B0002FA03F37A69134336
S31508022B807B617B687A699A607B685B687B610122F4
S31508022B903B6902FA03F3DB437A6913407B613B68BC
S31508022BA05B681B0903F001023B6902FA03F37A69BF
S31508022BB013437B617B687A695A603B685B68032BBF
S31508022BC017D07B68DB687B613B695B00032202FAEC
S31508022BD003F3DB437A6913407B613B689A683B6976
S31508022BE05B0002FA03F37A6913437B617B687A69AD
S31508022BF0DA603B685B6803F08053002B7CD0474A57
S31508022C003B699B08183352F823307B613B6903F012
S31508022C100303DB000F2202FA03F3DB437A6913404C
S31508022C207B617B689A0A3E4B13403A6902F00302BB
S31508022C30D20093407A6913437B6138493B699B0802
S31508022C4018337A6941F82320344B1B687B61FB6889
S31508022C50DB437A6913407B613B685B6803F4801344
S31508022C60002B03D07A69FB6813437B612B4A7B6985
S31508022C7013602A4B5B687B61FB68DB437A69134006
S31508022C807B613B685B6803F40013002B03D07A6907
S31508022C90FB6813437B61214A7B6953601F4BD3F858
S31508022CA084307B61FB68DB437A6913407B613B684E
S31508022CB05B6803F40033002B03D07A69FB6813437D
S31508022CC07B61164A7B69C2F88430144BD3F880308C
S31508022CD07B61FB68DB437A6913407B613B685B680F
S31508022CE003F48033002B03D07A69FB6813437B61B4
S31508022CF00A4A7B69C2F880303B6901333B613B680B
S31508022D001A683B6922FA03F3002B7FF4C1AE00BFAF
S31508022D1000BF1C37BD465DF8047B7047002002449D
S31508022D207F7F2F0080B487B000AF786039600023B8
S31508022D307B61A0E001227B6902FA03F33A68134039
S31508022D403B613B69002B00F09380524A7B699B08E2
S31508022D50183352F82330FB607B6903F00303DB0068
S31508022D600F2202FA03F3FA681340FB607B689A0A99
S31508022D70494B13407A6902F00302D2009340FA687B
S31508022D809A4236D1434BD3F880203B69DB4341490B
S31508022D901340C1F880303F4BD3F884203B69DB43AC
S31508022DA03C491340C1F884303A4B1A683B69DB4305
S31508022DB0384913400B60374B5A683B69DB43354940
S31508022DC013404B607B6903F00303DB000F2202FA10
S31508022DD003F3FB602F4A7B699B08183352F82310CA
S31508022DE0FB68DA432B487B699B080A40183340F88C
S31508022DF023207B681A687B695B00032101FA03F3C7
S31508022E001A437B681A607B69DA087B68083253F8CA
S31508022E1022107B6903F007039B000F2202FA03F3D1
S31508022E20DB437A69D20819407B68083243F82210D4
S31508022E307B689A687B695B00032101FA03F3DB432B
S31508022E401A407B689A607B685A6801217B6901FA95
S31508022E5003F3DB431A407B685A607B68DA687B694E
S31508022E605B00032101FA03F3DB431A407B68DA604D
S31508022E707B6901337B613A687B6922FA03F3002B8B
S31508022E807FF458AF00BF00BF1C37BD465DF8047B10
S31508022E90704700BF002002447F7F2F0080B485B0B0
S31508022EA000AF78600B467B807B681A697B88134083
S31508022EB0002B02D00123FB7301E00023FB73FB7B8B
S31508022EC018461437BD465DF8047B704780B483B054
S31508022ED000AF78600B467B8013467B707B78002BAD
S31508022EE003D07A887B689A6102E07A887B689A625C
S31508022EF000BF0C37BD465DF8047B704780B485B0C9
S31508022F0000AF78600B467B807B685B69FB607A88DA
S31508022F10FB6813401A04FB68D9437B880B401A43A3
S31508022F207B689A6100BF1437BD465DF8047B70471B
S31508022F3080B582B000AF0346FB800F4BDA68FB8888
S31508022F401340002B06D00C4AFB88D360FB88184630
S31508022F5000F014F8084B1A69FB881340002B06D0B8
S31508022F60054AFB881361FB8818461CF0BDFA00BFA8
S31508022F700837BD4680BD00BF0020024480B483B036
S31508022F8000AF0346FB8000BF0C37BD465DF8047BE5
S31508022F90704780B584B000AF78607B68002B01D19A
S31508022FA0012370E0786800F072F87B681B684CF6BB
S31508022FB0CC421A607B681B6845F255521A607B68D8
S31508022FC01B687A6852685A607B681B687A689268D6
S31508022FD09A60FEF789F9F8600FE0FEF785F902466E
S31508022FE0FB68D31A212B08D97B681B68DB6803F0B8
S31508022FF00203002B01D0032345E07B681B68DB68CC
S3150802300003F00203002BE8D17B681B69002B05D16C
S315080230107B681B684FF480425A6106E07B681A692E
S315080230207B681B6842F440425A61FEF75DF9F86014
S315080230300FE0FEF759F90246FB68D31A212B08D985
S315080230407B681B68DB6803F00F03002B01D00323A0
S3150802305019E07B681B68DB6803F00F03002BE8D1D5
S315080230607B681B681A697B68DB689A4205D07B68AD
S315080230701B687A68D2681A6104E07B681B684AF69C
S31508023080AA221A60002318461037BD4680BD80B4AE
S3150802309083B000AF786000BF0C37BD465DF8047B8D
S315080230A0704780B483B000AF78607B681B684AF6C5
S315080230B0AA221A60002318460C37BD465DF8047B1F
S315080230C07047000080B588B000AF78607B68002B37
S315080230D002D1012300F028BC944BDB6903F01803E4
S315080230E0FB61924B9B6A03F00303BB617B681B6817
S315080230F003F01003002B5BD0FB69082B05D0FB6994
S31508023100182B14D1BB69022B11D17B68DB69002B02
S3150802311002D1012300F008BC844B9B6923F47C127C
S315080231207B681B6A1B04814913438B6140E07B68F9
S31508023130DB69002B23D07D4B1B687C4A43F48073E2
S315080231401360FEF7D1F8786108E0FEF7CDF802467B
S315080231507B69D31A022B01D90323E5E3734B1B6858
S3150802316003F40073002BF0D0704B9B6923F47C1296
S315080231707B681B6A1B046D4913438B6118E06B4B12
S315080231801B686A4A23F480731360FEF7ADF8786108
S3150802319008E0FEF7A9F802467B69D31A022B01D981
S315080231A00323C1E3614B1B6803F40073002BF0D1C0
S315080231B07B681B6803F00103002B00F0A080FB6903
S315080231C0102B05D0FB69182B09D1BB69032B06D135
S315080231D07B685B68002B40F092800123A4E37B683E
S315080231E05B68B3F5803F06D1504B1B684F4A43F4E0
S315080231F08033136058E07B685B68002B12D14B4B17
S315080232001B684A4A23F480331360484B1B68474AB3
S3150802321023F480131360454B1B68444A23F4802326
S31508023220136041E07B685B68B3F5A02F12D13F4B70
S315080232301B683E4A43F4802313603C4B1B683B4A97
S3150802324023F480131360394B1B68384A43F48033DE
S31508023250136029E07B685B68B3F5A81F12D1334B6C
S315080232601B68324A43F480231360304B1B682F4A8B
S3150802327043F4801313602D4B1B682C4A43F48033A6
S31508023280136011E0294B1B68284A23F48033136024
S31508023290264B1B68254A23F480231360234B1B689D
S315080232A0224A23F4801313607B685B68002B13D0D1
S315080232B0FEF71AF8786108E0FEF716F802467B6907
S315080232C0D31A642B01D903232EE3184B1B6803F484
S315080232D00033002BF0D012E0FEF706F8786108E01A
S315080232E0FEF702F802467B69D31A642B01D9032337
S315080232F01AE30E4B1B6803F40033002BF0D17B68EC
S315080233001B6803F00203002B00F09A80FB69002B6E
S3150802331005D0FB69182B49D1BB69012B46D17B68BD
S31508023320DB68002B04D10123FEE200BF000C024435
S31508023330FB69002B1CD19A4B1B6803F018027B68A9
S315080233401B699A4214D0964B1B6823F018027B68B5
S315080233501B69934913430B6000F0D0FD914B1B6820
S3150802336018461BF0E9FF0346002B01D00123DBE2D6
S31508023370FDF7BAFF786108E0FDF7B6FF02467B69FA
S31508023380D31A022B01D90323CEE2854B1B6803F01D
S315080233900203002BF0D0824B1B6923F4FE027B68E2
S315080233A05B691B047E4913430B6149E07B68DB6852
S315080233B0002B2CD07A4B1B6823F018027B681B69FA
S315080233C0774913430B60764B1B68754A43F0010332
S315080233D01360FDF789FF786108E0FDF785FF02466D
S315080233E07B69D31A022B01D903239DE26C4B1B6816
S315080233F003F00203002BF0D0694B1B6923F4FE028B
S315080234007B685B691B04664913430B6118E0644BCE
S315080234101B68634A23F001031360FDF765FF7861B1
S3150802342008E0FDF761FF02467B69D31A022B01D930
S31508023430032379E25A4B1B6803F00203002BF0D1EF
S315080234407B681B6803F00803002B3CD07B689B69EA
S31508023450002B1CD0524BD3F8F030514A43F080630C
S31508023460C2F8F030FDF740FF786108E0FDF73CFF4F
S3150802347002467B69D31A022B01D9032354E2484B2D
S31508023480D3F8F03003F00063002BEFD01BE0444B77
S31508023490D3F8F030424A23F08063C2F8F030FDF7E1
S315080234A023FF786108E0FDF71FFF02467B69D31AFE
S315080234B0022B01D9032337E2394BD3F8F03003F054
S315080234C00063002BEFD17B681B6803F00403002B13
S315080234D000F0D280344B5B6A03F00103002B18D14B
S315080234E0314B5B6A304A43F001035362FDF7FCFE37
S315080234F0786108E0FDF7F8FE02467B69D31A022BCB
S3150802350001D9032310E2284B5B6A03F00103002B5F
S31508023510F0D07B689B68012B08D1214BD3F8F03099
S315080235201F4A43F00103C2F8F03074E07B689B68D7
S31508023530002B18D11A4BD3F8F030194A23F001039D
S31508023540C2F8F030164BD3F8F030154A23F0800350
S31508023550C2F8F030124BD3F8F030114A23F00403C4
S31508023560C2F8F03057E07B689B68052B1ED10C4BDE
S31508023570D3F8F0300A4A43F00403C2F8F030084B95
S31508023580D3F8F030064A23F08003C2F8F030044B31
S31508023590D3F8F030024A43F00103C2F8F0303AE0B9
S315080235A0000C024400000020000802447B689B6865
S315080235B0852B18D1A24BD3F8F030A14A43F0040365
S315080235C0C2F8F0309E4BD3F8F0309D4A43F08003A0
S315080235D0C2F8F0309A4BD3F8F030994A43F0010317
S315080235E0C2F8F03017E0964BD3F8F030944A23F03D
S315080235F00103C2F8F030924BD3F8F030904A23F028
S315080236000403C2F8F0308E4BD3F8F0308C4A23F01C
S315080236108003C2F8F0307B689B68002B16D0FDF752
S3150802362063FE78610AE0FDF75FFE02467B69D31AFC
S3150802363041F28832934201D9032375E1804BD3F8CC
S31508023640F03003F00203002BEDD015E0FDF74CFE37
S3150802365078610AE0FDF748FE02467B69D31A41F211
S315080236608832934201D903235EE1754BD3F8F030D1
S3150802367003F00203002BEDD17B681B6803F02003DD
S31508023680002B36D07B685B6A002B19D06C4B1B6803
S315080236906B4A43F480531360FDF726FE786108E00F
S315080236A0FDF722FE02467B69D31A022B01D90323B0
S315080236B03AE1634B1B6803F40053002BF0D018E081
S315080236C05F4B1B685E4A23F480531360FDF70CFEBA
S315080236D0786108E0FDF708FE02467B69D31A022BD9
S315080236E001D9032320E1564B1B6803F40053002B30
S315080236F0F0D17B689B6A002B00F01581FB69182BB9
S3150802370000F0AF807B689B6A022B40F086804C4BA8
S315080237101B684B4A23F080731360FDF7E5FD786159
S3150802372008E0FDF7E1FD02467B69D31A022B01D9AF
S315080237300323F9E0424B1B6803F00073002BF0D118
S315080237403F4B9B6A23F47C5323F003037A68D16ABE
S315080237507A68126B12020A43394913438B627B68F1
S315080237605B6B013BC3F308027B689B6B013B5B0205
S315080237709BB21A437B68DB6B013B1B0403F4FE0313
S315080237801A437B681B6C013B1B0603F0FE432C495C
S3150802379013434B632A4B9B6A294A23F0100393620D
S315080237A07B68DB6C264ADB009363254B9B6A244ABB
S315080237B043F010039362224B9B6A23F00C027B6848
S315080237C05B6C1F4913438B621D4B9B6A23F02002D5
S315080237D07B689B6C1A4913438B62194B9B6A184A7E
S315080237E043F480339362164B1B68154A43F0807381
S315080237F01360FDF779FD786108E0FDF775FD02466D
S315080238007B69D31A022B01D903238DE00C4B1B6863
S3150802381003F00073002BF0D085E0094B1B68084AB9
S3150802382023F080731360FDF75FFD78610AE0FDF708
S315080238305BFD02467B69D31A022B03D9032373E085
S31508023840000C02443A4B1B6803F00073002BEED1BE
S31508023850374B9B6A364A23F4E02323F00303936229
S3150802386061E0334B9B6A3B61314B5B6BFB607B6868
S315080238709B6A012B31D03B6903F003027B68DB6A42
S315080238809A422AD13B691B0A03F03F027B681B6BEB
S315080238909A4222D1FB68C3F308027B685B6B013B41
S315080238A09A421AD1FB685B0A03F07F027B689B6B1C
S315080238B0013B9A4211D1FB681B0C03F07F027B681D
S315080238C0DB6B013B9A4208D1FB681B0E03F07F02B1
S315080238D07B681B6C013B9A4201D0012324E0144BFE
S315080238E09B6BDB08C3F30C027B68DB6C9A421AD02B
S315080238F00F4B9B6A0E4A23F010039362FDF7F4FC02
S31508023900786100BFFDF7F0FC02467B699342F9D065
S315080239107B68DB6C064ADB009363054B9B6A044AA9
S3150802392043F010039362002318462037BD4680BD34
S31508023930000C024480B584B000AF786039607B68B9
S31508023940002B01D101239EE1834B1B6803F00F0371
S315080239503A689A4210D9804B1B6823F00F027E49B7
S315080239603B6813430B607C4B1B6803F00F033A68F2
S315080239709A4201D0012386E17B681B6803F0100393
S31508023980002B12D07B685A69744B1B6A1B0A03F018
S3150802399070039A4209D9714B1B6A23F4E0427B6889
S315080239A05B691B026D4913430B627B681B6803F054
S315080239B00803002B12D07B681A69684B1B6A1B091D
S315080239C003F070039A4209D9644B1B6A23F4E06236
S315080239D07B681B691B01614913430B627B681B6881
S315080239E003F00403002B10D07B68DA685B4B1B6A72
S315080239F003F070039A4208D9584B1B6A23F07002E7
S31508023A007B68DB68554913430B627B681B6803F0C6
S31508023A100203002B10D07B689A68504B1B6A03F08E
S31508023A200F039A4208D94D4B1B6A23F00F027B6893
S31508023A309B684A4913430B627B681B6803F00103C0
S31508023A40002B00F093807B685B68032B07D1434BFE
S31508023A501B6803F00073002B21D1012313E17B6855
S31508023A605B68022B07D13D4B1B6803F40033002B1E
S31508023A7015D1012307E17B685B68012B07D1374B18
S31508023A801B6803F40073002B09D10123FBE0334BB7
S31508023A901B6803F00203002B01D10123F3E02F4B2D
S31508023AA0DB6923F003027B685B682C491343CB610D
S31508023AB0FDF71AFCF8607B685B68032B12D10AE0F3
S31508023AC0FDF712FC0246FB68D31A41F2883293428A
S31508023AD001D90323D7E0214BDB6903F01803182B1E
S31508023AE0EED143E07B685B68022B12D10AE0FDF750
S31508023AF0FBFB0246FB68D31A41F28832934201D98C
S31508023B000323C0E0154BDB6903F01803102BEED133
S31508023B102CE07B685B68012B22D10AE0FDF7E4FB07
S31508023B200246FB68D31A41F28832934201D903232B
S31508023B30A9E00A4BDB6903F01803082BEED115E05E
S31508023B40FDF7D2FB0246FB68D31A41F2883293424A
S31508023B5006D9032397E000BF00200240000C024466
S31508023B604B4BDB6903F01803002BE9D17B681B6812
S31508023B7003F00203002B10D07B689A68444B1B6A39
S31508023B8003F00F039A4208D2414B1B6A23F00F0235
S31508023B907B689B683E4913430B623E4B1B6803F0E6
S31508023BA00F033A689A4210D23A4B1B6823F00F0267
S31508023BB038493B6813430B60364B1B6803F00F0307
S31508023BC03A689A4201D001235DE07B681B6803F0DC
S31508023BD00403002B10D07B68DA682D4B1B6A03F0AE
S31508023BE070039A4208D22A4B1B6A23F070027B683A
S31508023BF0DB68274913430B627B681B6803F00803DB
S31508023C00002B12D07B681A69214B1B6A1B0903F029
S31508023C1070039A4209D21E4B1B6A23F4E0627B6840
S31508023C201B691B011A4913430B627B681B6803F065
S31508023C301003002B12D07B685A69154B1B6A1B0AA4
S31508023C4003F070039A4209D2114B1B6A23F4E0422D
S31508023C507B685B691B020E4913430B6200F022F86C
S31508023C6002460B4B1B6A03F00F030B49CB5C22FA85
S31508023C7003F30A4A13600A4B1B6818461BF05CFBDF
S31508023C800346FB72FB7A18461037BD4680BD00BF55
S31508023C90000C024400200240DC8D0808C4120020F1
S31508023CA00000002080B489B000AF8C4BDB6903F0BA
S31508023CB01803082B02D18A4BFB6107E1874BDB69A4
S31508023CC003F01803002B12D1844B1B6803F0200360
S31508023CD0002B09D0814B1B68DB0803F00303814ADA
S31508023CE022FA03F3FB61F1E07E4BFB61EEE07B4BCC
S31508023CF0DB6903F01803102B02D17B4BFB61E5E06D
S31508023D00764BDB6903F01803182B40F0DD80734B02
S31508023D109B6A03F003037B61704B9B6A1B0A03F0E1
S31508023D203F033B616D4B9B6A1B0903F00103FB6072
S31508023D306A4B9B6BDB08C3F30C03FA6802FB03F3BB
S31508023D4007EE903AF8EE677AC7ED027A3B69002BDE
S31508023D5000F0B7807B69012B03D07B69032B56D011
S31508023D6077E05E4B1B6803F02003002B2DD05B4BDC
S31508023D701B68DB0803F003035A4A22FA03F37B6043
S31508023D807B6807EE903AF8EE676A3B6907EE903A67
S31508023D90F8EE677A86EEA77A504B5B6BC3F3080395
S31508023DA007EE903AF8EE676A97ED026ADFED4F5A28
S31508023DB0C6EE257A76EEA77AF7EE006A77EEA67A47
S31508023DC067EE277AC7ED067A65E03B6907EE903A11
S31508023DD0F8EE677ADFED466A86EEA77A3F4B5B6BAB
S31508023DE0C3F3080307EE903AF8EE676A97ED026A9C
S31508023DF0DFED3E5AC6EE257A76EEA77AF7EE006A28
S31508023E0077EEA67A67EE277AC7ED067A43E03B692C
S31508023E1007EE903AF8EE677ADFED366A86EEA77A0B
S31508023E202E4B5B6BC3F3080307EE903AF8EE676A0C
S31508023E3097ED026ADFED2D5AC6EE257A76EEA77A57
S31508023E40F7EE006A77EEA67A67EE277AC7ED067A64
S31508023E5021E03B6907EE903AF8EE677ADFED266ACB
S31508023E6086EEA77A1D4B5B6BC3F3080307EE903AFF
S31508023E70F8EE676A97ED026ADFED1C5AC6EE257AF6
S31508023E8076EEA77AF7EE006A77EEA67A67EE277AD3
S31508023E90C7ED067A00BF114B5B6B5B0A03F07F0323
S31508023EA001333B603B6807EE903AB8EE677AD7ED86
S31508023EB0066AC6EE877AFCEEE77A17EE903AFB6157
S31508023EC004E00023FB6101E0064BFB61FB6918462F
S31508023ED02437BD465DF8047B704700BF000C0244D8
S31508023EE000093D000090D003001BB7000000004601
S31508023EF00024744C001B374B0024744A80B500AF6B
S31508023F00FFF7D0FE0246084B1B6A03F00F03074968
S31508023F10CB5C03F01F0322FA03F3054A1360044B32
S31508023F201B68184680BD00BF000C0244DC8D0808D9
S31508023F30C412002080B500AFFFF7E0FF0246064B29
S31508023F401B6A1B0903F007030449CB5C03F01F0332
S31508023F5022FA03F3184680BD000C0244EC8D0808C9
S31508023F6080B500AFFFF7CAFF0246064B1B6A1B0A5B
S31508023F7003F007030449CB5C03F01F0322FA03F399
S31508023F80184680BD000C0244EC8D080880B500AFC7
S31508023F90FFF7B4FF0246064B1B6A1B0B03F0070327
S31508023FA00449CB5C03F01F0322FA03F3184680BDCB
S31508023FB0000C0244EC8D080880B485B000AF786026
S31508023FC039607B681F221A60154BDB6903F003020E
S31508023FD07B685A60124B1B6AFB60FB6803F00F0290
S31508023FE07B689A60FB6803F070027B68DA60FB689C
S31508023FF01B0903F070027B681A61FB681B0A03F04F
S3150802400070027B685A61074B1B6803F00F023B6814
S315080240101A6000BF1437BD465DF8047B704700BFBF
S31508024020000C0244002002402DE9B04FD8B000AF80
S31508024030C7F84C01002387F85B31002387F85A3109
S31508024040D7F84C31D3E9002302F08074002554EAEC
S3150802405005030BD0CD4BD3F8E83023F04041D7F80F
S315080240604C319B6DC94A0B43C2F8E830D7F84C313C
S31508024070D3E9002302F001084FF0000958EA0903C0
S3150802408042D0D7F84C31DB6D052B23D801A252F862
S3150802409023F000BFDD400208AD400208C140020815
S315080240A0DD400208DD400208DD400208D7F84C313F
S315080240B00833184604F0DAFE034687F85B310EE049
S315080240C0D7F84C313033184604F068FF034687F8B0
S315080240D05B3104E0012387F85B3100E000BF97F803
S315080240E05B31002B0CD1A94BD3F8D83023F007014A
S315080240F0D7F84C31DB6DA54A0B43C2F8D83003E03A
S3150802410097F85B3187F85A31D7F84C31D3E900234F
S3150802411002F0020A4FF0000B5AEA0B0300F08880FD
S31508024120D7F84C311B6E282B68D801A252F823F017
S3150802413005420208FD410208FD410208FD41020846
S31508024140FD410208FD410208FD410208FD4102083F
S31508024150D5410208FD410208FD410208FD41020857
S31508024160FD410208FD410208FD410208FD4102081F
S31508024170E9410208FD410208FD410208FD41020823
S31508024180FD410208FD410208FD410208FD410208FF
S3150802419005420208FD410208FD410208FD410208E6
S315080241A0FD410208FD410208FD410208FD410208DF
S315080241B005420208FD410208FD410208FD410208C6
S315080241C0FD410208FD410208FD410208FD410208BF
S315080241D005420208D7F84C310833184604F046FE61
S315080241E0034687F85B310EE0D7F84C313033184670
S315080241F004F0D4FE034687F85B3104E0012387F80E
S315080242005B3100E000BF97F85B31002B0CD15F4BA6
S31508024210D3F8D83023F03801D7F84C311B6E5B4AF5
S315080242200B43C2F8D83003E097F85B3187F85A3166
S31508024230D7F84C31D3E9002302F00403C7F840311A
S315080242400023C7F84431D7E950120B4613434ED020
S31508024250D7F84C315B6EB3F5A07F2CD0B3F5A07FAF
S3150802426025D8B3F5807F28D0B3F5807F1FD8C02B19
S3150802427025D0C02B1BD8802B0FD0802B17D8002B0C
S315080242801FD0402B13D1D7F84C310833184604F007
S31508024290EDFD034687F85B3114E0D7F84C3130332D
S315080242A0184604F07BFE034687F85B310AE00123D1
S315080242B087F85B3106E000BF04E000BF02E000BFFA
S315080242C000E000BF97F85B31002B0CD12F4BD3F8D7
S315080242D0D83023F4E071D7F84C315B6E2B4A0B4386
S315080242E0C2F8D83003E097F85B3187F85A31D7F825
S315080242F04C31D3E9002302F00803C7F8383100230A
S31508024300C7F83C31D7E94E120B46134356D0D7F8B5
S315080243104C319B6EB3F5206F31D0B3F5206F2AD896
S31508024320B3F5006F2DD0B3F5006F24D8B3F5C06F7F
S3150802433029D0B3F5C06F1ED8B3F5806F11D0B3F587
S31508024340806F18D8002B23D0B3F5007F13D1D7F886
S315080243504C310833184604F089FD034687F85B3169
S3150802436017E0D7F84C313033184604F017FE0346E7
S3150802437087F85B310DE0012387F85B3109E000BF5E
S3150802438007E000BF05E000BF03E000BF000C0244DF
S3150802439000BF97F85B31002B0CD1BB4BD3F8D83052
S315080243A023F46061D7F84C319B6EB74A0B43C2F8C7
S315080243B0D83003E097F85B3187F85A31D7F84C3191
S315080243C0D3E9002302F01003C7F830310023C7F8F7
S315080243D03431D7E94C120B46134353D0D7F84C3134
S315080243E0DB6EB3F5A04F31D0B3F5A04F2AD8B3F59B
S315080243F0804F2DD0B3F5804F24D8B3F5405F29D02E
S31508024400B3F5405F1ED8B3F5005F11D0B3F5005F70
S3150802441018D8002B20D0B3F5805F13D1D7F84C31CA
S315080244200833184604F022FD034687F85B3114E088
S31508024430D7F84C313033184604F0B0FD034687F8F6
S315080244405B310AE0012387F85B3106E000BF04E02E
S3150802445000BF02E000BF00E000BF97F85B31002B07
S315080244600CD1894BD3F8D83023F4E041D7F84C3134
S31508024470DB6E854A0B43C2F8D83003E097F85B3106
S3150802448087F85A31D7F84C31D3E9002302F02003D2
S31508024490C7F828310023C7F82C31D7E94A120B4648
S315080244A0134353D0D7F84C311B6FB3F5203F31D0A5
S315080244B0B3F5203F2AD8B3F5003F2DD0B3F5003F18
S315080244C024D8B3F5C03F29D0B3F5C03F1ED8B3F5FB
S315080244D0803F11D0B3F5803F18D8002B20D0B3F512
S315080244E0004F13D1D7F84C310833184604F0BEFCF6
S315080244F0034687F85B3114E0D7F84C313033184657
S3150802450004F04CFD034687F85B310AE0012387F87D
S315080245105B3106E000BF04E000BF02E000BF00E036
S3150802452000BF97F85B31002B0CD1574BD3F8D83024
S3150802453023F46031D7F84C311B6F534A0B43C2F848
S31508024540D83003E097F85B3187F85A31D7F84C31FF
S31508024550D3E9002302F04003C7F820310023C7F845
S315080245602431D7E948120B46134353D0D7F84C31B6
S315080245705B6FB3F5A01F31D0B3F5A01F2AD8B3F5E8
S31508024580801F2DD0B3F5801F24D8B3F5402F29D02C
S31508024590B3F5402F1ED8B3F5002F11D0B3F5002F6F
S315080245A018D8002B20D0B3F5802F13D1D7F84C3169
S315080245B00833184604F05AFC034687F85B3114E0C0
S315080245C0D7F84C313033184604F0E8FC034687F82E
S315080245D05B310AE0012387F85B3106E000BF04E09D
S315080245E000BF02E000BF00E000BF97F85B31002B76
S315080245F00CD1254BD3F8D83023F4E011D7F84C3137
S315080246005B6F214A0B43C2F8D83003E097F85B3157
S3150802461087F85A31D7F84C31D3E9002302F08003E0
S31508024620C7F818310023C7F81C31D7E946120B46DA
S31508024630134355D0D7F84C319B6FB3F5200F33D0BF
S31508024640B3F5200F2CD8B3F5000F2FD0B3F5000F12
S3150802465026D8B3F5C00F2BD0B3F5C00F20D8B3F5C3
S31508024660800F13D0B3F5800F1AD8002B22D0B3F5DA
S31508024670001F15D1D7F84C310833184604F0F6FB5B
S31508024680034687F85B3116E0000C0244D7F84C3132
S315080246903033184604F082FC034687F85B310AE099
S315080246A0012387F85B3106E000BF04E000BF02E0A1
S315080246B000BF00E000BF97F85B31002B0CD1BB4B63
S315080246C0D3F8D83023F46001D7F84C319B6FB74A38
S315080246D00B43C2F8D83003E097F85B3187F85A31B2
S315080246E0D7F84C31D3E9002302F48073C7F81031A6
S315080246F00023C7F81431D7E944120B46134353D0A3
S31508024700D7F84C31DB6FB3F1A06F31D0B3F1A06F9C
S315080247102AD8B3F1806F2DD0B3F1806F24D8B3F1C4
S31508024720407F29D0B3F1407F1ED8B3F1007F11D064
S31508024730B3F1007F18D8002B20D0B3F1807F13D1B4
S31508024740D7F84C310833184604F090FB034687F82D
S315080247505B3114E0D7F84C313033184604F01EFCAE
S31508024760034687F85B310AE0012387F85B3106E0E6
S3150802477000BF04E000BF02E000BF00E000BF97F8F8
S315080247805B31002B0CD1894BD3F8D83023F0E0618A
S31508024790D7F84C31DB6F854A0B43C2F8D83003E0B1
S315080247A097F85B3187F85A31D7F84C31D3E90023A9
S315080247B002F40073C7F808310023C7F80C31D7E9A9
S315080247C042120B46134355D0D7F84C31D3F88030F2
S315080247D0B3F1205F31D0B3F1205F2AD8B3F1005F7D
S315080247E02DD0B3F1005F24D8B3F1C05F29D0B3F15D
S315080247F0C05F1ED8B3F1805F11D0B3F1805F18D8BD
S31508024800002B20D0B3F1006F13D1D7F84C310833FF
S31508024810184604F02BFB034687F85B3114E0D7F8F9
S315080248204C313033184604F0B9FB034687F85B313E
S315080248300AE0012387F85B3106E000BF04E000BF07
S3150802484002E000BF00E000BF97F85B31002B0DD1F4
S31508024850564BD3F8D83023F06051D7F84C31D3F8F9
S315080248608030524A0B43C2F8D83003E097F85B31DE
S3150802487087F85A31D7F84C31D3E9002302F480631A
S31508024880C7F800310023C7F80431D7E940120B46AE
S31508024890134344D0D7F84C31D3F88430052B23D8A8
S315080248A001A252F823F000BFF1480208C1480208E3
S315080248B0D5480208F1480208F1480208F1480208F8
S315080248C0D7F84C310833184604F0D0FA034687F86D
S315080248D05B310EE0D7F84C313033184604F05EFBF4
S315080248E0034687F85B3104E0012387F85B3100E071
S315080248F000BF97F85B31002B0DD12C4BD3F8DC3077
S3150802490023F00701D7F84C31D3F88430274A0B43F2
S31508024910C2F8DC3003E097F85B3187F85A31D7F8EA
S315080249204C31D3E9002302F40063C7F8F8300023B8
S31508024930C7F8FC30D7E93E120B4613434FD0D7F8D7
S315080249404C31D3F88830502B29D0502B23D8402B02
S3150802495027D0402B1FD8302B25D0302B1BD8202B05
S315080249600FD0202B17D8002B22D0102B13D1D7F813
S315080249704C310833184604F079FA034687F85B3156
S3150802498017E0D7F84C313033184604F007FB0346D4
S3150802499087F85B310DE0012387F85B3109E000BF38
S315080249A007E000BF05E000BF03E000BF000C0244B9
S315080249B000BF97F85B31002B0DD1AF4BD3F8DC3033
S315080249C023F07001D7F84C31D3F88830AA4A0B4342
S315080249D0C2F8DC3003E097F85B3187F85A31D7F82A
S315080249E04C31D3E9002302F48053C7F8F030002390
S315080249F0C7F8F430D7E93C120B46134355D0D7F81B
S31508024A004C31D3F88C30B3F1A06F31D0B3F1A06F2B
S31508024A102AD8B3F1806F2DD0B3F1806F24D8B3F1C1
S31508024A20407F29D0B3F1407F1ED8B3F1007F11D061
S31508024A30B3F1007F18D8002B20D0B3F1807F13D1B1
S31508024A40D7F84C310833184604F010FA034687F8AB
S31508024A505B3114E0D7F84C313033184604F09EFA2D
S31508024A60034687F85B310AE0012387F85B3106E0E3
S31508024A7000BF04E000BF02E000BF00E000BF97F8F5
S31508024A805B31002B0DD17C4BD3F8E03023F0E0618B
S31508024A90D7F84C31D3F88C30774A0B43C2F8E0305A
S31508024AA003E097F85B3187F85A31D7F84C31D3E9E6
S31508024AB0002302F40053C7F8E8300023C7F8EC30A5
S31508024AC0D7E93A120B4613433DD0D7F84C31D3F8FF
S31508024AD09030B3F5403F1BD0B3F5403F14D8B3F539
S31508024AE0003F17D0B3F5003F0ED8002B14D0B3F50C
S31508024AF0803F09D1D7F84C313033184604F04EFAC4
S31508024B00034687F85B3108E0012387F85B3104E046
S31508024B1000BF02E000BF00E000BF97F85B31002B40
S31508024B200DD1554BD3F8E43023F44031D7F84C3144
S31508024B30D3F89030504A0B43C2F8E43003E097F8B2
S31508024B405B3187F85A31D7F84C31D3E9002302F49E
S31508024B508043C7F8E0300023C7F8E430D7E93812B3
S31508024B600B4613433DD0D7F84C31D3F89430B3F5FE
S31508024B70402F1BD0B3F5402F14D8B3F5002F17D00A
S31508024B80B3F5002F0ED8002B14D0B3F5802F09D118
S31508024B90D7F84C313033184604F000FA034687F842
S31508024BA05B3108E0012387F85B3104E000BF02E0CD
S31508024BB000BF00E000BF97F85B31002B0DD12E4BEA
S31508024BC0D3F8E43023F44021D7F84C31D3F89430A3
S31508024BD0294A0B43C2F8E43003E097F85B3187F8B9
S31508024BE05A31D7F84C31D3E9002302F40043C7F807
S31508024BF0D8300023C7F8DC30D7E936120B46134300
S31508024C0040D0D7F84C31D3F89830B3F5401F1BD0B3
S31508024C10B3F5401F14D8B3F5001F17D0B3F5001F1C
S31508024C200ED8002B14D0B3F5801F09D1D7F84C3112
S31508024C303033184604F0B2F9034687F85B3108E0C8
S31508024C40012387F85B3104E000BF02E000BF00E001
S31508024C5000BF97F85B31002B10D1074BD3F8E4302D
S31508024C6023F44011D7F84C31D3F89830024A0B4353
S31508024C70C2F8E43006E000BF000C024497F85B3144
S31508024C8087F85A31D7F84C31D3E900230021C7F8FF
S31508024C90D01003F48063C7F8D430D7E934120B4630
S31508024CA013433DD0D7F84C31D3F89C30B3F5400FB7
S31508024CB01BD0B3F5400F14D8B3F5000F17D0B3F5D0
S31508024CC0000F0ED8002B14D0B3F5800F09D1D7F8F0
S31508024CD04C313033184604F061F9034687F85B31E4
S31508024CE008E0012387F85B3104E000BF02E000BF59
S31508024CF000E000BF97F85B31002B0DD1BE4BD3F80D
S31508024D00E43023F44001D7F84C31D3F89C30BA4A40
S31508024D100B43C2F8E43003E097F85B3187F85A315F
S31508024D20D7F84C31D3E9002302F48033C7F8C830E8
S31508024D300023C7F8CC30D7E932120B46134335D0D5
S31508024D40D7F84C31D3F8A030B3F1007F15D0B3F1C0
S31508024D50007F0ED8002B12D0B3F1807F09D1D7F885
S31508024D604C313033184604F019F9034687F85B319B
S31508024D7006E0012387F85B3102E000BF00E000BFCE
S31508024D8097F85B31002B0DD19B4BD3F8E43023F017
S31508024D904071D7F84C31D3F8A030974A0B43C2F882
S31508024DA0E43003E097F85B3187F85A31D7F84C318B
S31508024DB0D3E900230021C7F8C01003F40063C7F83B
S31508024DC0C430D7E930120B4613430ED08A4BDB693F
S31508024DD0894A23F40043D361874BD969D7F84C3102
S31508024DE0D3F80431844A0B43D361D7F84C31D3E95B
S31508024DF0002302F40033C7F8B8300023C7F8BC30E2
S31508024E00D7E92E120B46134355D0D7F84C31D3F8AF
S31508024E10A430B3F5A06F31D0B3F5A06F2AD8B3F595
S31508024E20806F2DD0B3F5806F24D8B3F5407F29D093
S31508024E30B3F5407F1ED8B3F5007F11D0B3F5007FD6
S31508024E4018D8002B20D0B3F5807F13D1D7F84C3170
S31508024E500833184604F00AF8034687F85B3114E06B
S31508024E60D7F84C313033184604F098F8034687F8D9
S31508024E705B310AE0012387F85B3106E000BF04E0F4
S31508024E8000BF02E000BF00E000BF97F85B31002BCD
S31508024E900DD1594BD3F8DC3023F4E061D7F84C3105
S31508024EA0D3F8A430544A0B43C2F8DC3003E097F82F
S31508024EB05B3187F85A31D7F84C31D3E9002302F42B
S31508024EC08023C7F8B0300023C7F8B430D7E92C12CC
S31508024ED00B46134355D0D7F84C31D3F8A830B3F55F
S31508024EE0A04F31D0B3F5A04F2AD8B3F5804F2DD0B5
S31508024EF0B3F5804F24D8B3F5405F29D0B3F5405FA8
S31508024F001ED8B3F5005F11D0B3F5005F18D8002B91
S31508024F1020D0B3F5805F13D1D7F84C310833184641
S31508024F2003F0A4FF034687F85B3114E0D7F84C3147
S31508024F303033184604F032F8034687F85B310AE044
S31508024F40012387F85B3106E000BF04E000BF02E0F8
S31508024F5000BF00E000BF97F85B31002B0DD1264B4E
S31508024F60D3F8DC3023F4E041D7F84C31D3F8A83033
S31508024F70214A0B43C2F8DC3003E097F85B3187F825
S31508024F805A31D7F84C31D3E900230021C7F8A810C3
S31508024F9003F02003C7F8AC30D7E92A120B461343AD
S31508024FA057D0D7F84C31D3F8AC30B3F5A02F33D05D
S31508024FB0B3F5A02F2CD8B3F5802F2FD0B3F5802FB9
S31508024FC026D8B3F5403F2BD0B3F5403F20D8B3F5EA
S31508024FD0003F13D0B3F5003F1AD8002B22D0B3F501
S31508024FE0803F15D1D7F84C310833184603F03EFFF7
S31508024FF0034687F85B3116E0000C0244D7F84C31B9
S315080250003033184603F0CAFF034687F85B310AE0D5
S31508025010012387F85B3106E000BF04E000BF02E027
S3150802502000BF00E000BF97F85B31002B0DD1BB4BE8
S31508025030D3F8DC3023F4E021D7F84C31D3F8AC307E
S31508025040B64A0B43C2F8DC3003E097F85B3187F8BF
S315080250505A31D7F84C31D3E900230021C7F8A010FA
S3150802506003F04003C7F8A430D7E928120B461343C6
S3150802507055D0D7F84C31D3F8B030B3F5A00F31D0AC
S31508025080B3F5A00F2AD8B3F5800F2DD0B3F5800F4C
S3150802509024D8B3F5401F29D0B3F5401F1ED8B3F55F
S315080250A0001F11D0B3F5001F18D8002B20D0B3F576
S315080250B0801F13D1D7F84C310833184603F0D6FEB1
S315080250C0034687F85B3114E0D7F84C31303318467B
S315080250D003F064FF034687F85B310AE0012387F889
S315080250E05B3106E000BF04E000BF02E000BF00E05B
S315080250F000BF97F85B31002B0DD1884BD3F8DC3013
S3150802510023F4E001D7F84C31D3F8B030834A0B4385
S31508025110C2F8DC3003E097F85B3187F85A31D7F8E2
S315080251204C31D3E900230021C7F8981003F0800315
S31508025130C7F89C30D7E926120B46134355D0D7F841
S315080251404C31D3F8B430B3F1A06F31D0B3F1A06FBC
S315080251502AD8B3F1806F2DD0B3F1806F24D8B3F17A
S31508025160407F29D0B3F1407F1ED8B3F1007F11D01A
S31508025170B3F1007F18D8002B20D0B3F1807F13D16A
S31508025180D7F84C310833184603F070FE034687F801
S315080251905B3114E0D7F84C313033184603F0FEFE83
S315080251A0034687F85B310AE0012387F85B3106E09C
S315080251B000BF04E000BF02E000BF00E000BF97F8AE
S315080251C05B31002B0DD1554BD3F8DC3023F0E0616F
S315080251D0D7F84C31D3F8B430504A0B43C2F8DC3016
S315080251E003E097F85B3187F85A31D7F84C31D3E99F
S315080251F000230021C7F8901003F48073C7F894308F
S31508025200D7E924120B46134355D0D7F84C31D3F8B5
S31508025210B830B3F1A04F31D0B3F1A04F2AD8B3F1C9
S31508025220804F2DD0B3F1804F24D8B3F1405F29D0F7
S31508025230B3F1405F1ED8B3F1005F11D0B3F1005F3E
S3150802524018D8002B20D0B3F1805F13D1D7F84C3190
S315080252500833184603F00AFE034687F85B3114E062
S31508025260D7F84C313033184603F098FE034687F8D0
S315080252705B310AE0012387F85B3106E000BF04E0F0
S3150802528000BF02E000BF00E000BF97F85B31002BC9
S315080252900DD1224BD3F8DC3023F0E041D7F84C315C
S315080252A0D3F8B8301D4A0B43C2F8DC3003E097F84E
S315080252B05B3187F85A31D7F84C31D3E9002302F427
S315080252C00023C7F888300023C7F88C30D7E92212A2
S315080252D00B46134355D0D7F84C31D3F8C030B3F543
S315080252E0802F35D0B3F5802F2ED8B3F5403F31D075
S315080252F0B3F5403F28D8B3F5003F1BD0B3F5003FBE
S3150802530022D8002B03D0B3F5803F09D01CE0034B0B
S315080253109B6A024A43F4003393621CE0000C02447F
S31508025320D7F84C310833184603F0A0FD034687F830
S315080253305B3110E0D7F84C313033184603F02EFEB5
S31508025340034687F85B3106E0012387F85B3102E002
S3150802535000BF00E000BF97F85B31002B0DD1C34BAD
S31508025360D3F8E83023F4E021D7F84C31D3F8C0302B
S31508025370BE4A0B43C2F8E83003E097F85B3187F878
S315080253805A31D7F84C31D3E9002302F48013C7F80F
S3150802539080300023C7F88430D7E920120B4613431E
S315080253A051D0D7F84C31D3F8C430B3F5001F33D0F7
S315080253B0B3F5001F2CD8B3F5C01F2DD0B3F5C01F07
S315080253C026D8B3F5801F19D0B3F5801F20D8002B35
S315080253D003D0B3F5002F07D01AE0A44B9B6AA34A61
S315080253E043F40033936218E0D7F84C310833184671
S315080253F003F03CFD034687F85B310EE0D7F84C31E3
S315080254003033184603F0CAFD034687F85B3104E0D9
S31508025410012387F85B3100E000BF97F85B31002B68
S315080254200DD1924BD3F8E83023F46011D7F84C31FA
S31508025430D3F8C4308D4A0B43C2F8E83003E097F834
S315080254405B3187F85A31D7F84C31D3E9002302F495
S315080254500013BB670023FB67D7E91E120B461343EB
S3150802546032D0D7F84C31D3F8D430052B0FD8032BCA
S3150802547011D2012B11D9022B09D1D7F84C31083395
S31508025480184603F0F3FC034687F85B3106E001236E
S3150802549087F85B3102E000BF00E000BF97F85B3196
S315080254A0002B0DD1714BD3F8E83023F00701D7F85A
S315080254B04C31D3F8D4306D4A0B43C2F8E83003E0D6
S315080254C097F85B3187F85A31D7F84C31D3E900237C
S315080254D00021396703F400737B67D7E91C120B4670
S315080254E0134324D0D7F84C31D3F8D830002B05D043
S315080254F0082B05D0012387F85B3102E000BF00E0E4
S3150802550000BF97F85B31002B0DD1584BD3F8E83022
S3150802551023F00801D7F84C31D3F8D830534A0B4355
S31508025520C2F8E83003E097F85B3187F85A31D7F8C2
S315080255304C31D3E9002302F00073BB660023FB66F5
S31508025540D7E91A120B46134300F0B980484B5B6A37
S31508025550474A43F001035362FBF7C6FEC7F85401F4
S315080255600BE0FBF7C1FE0246D7F85431D31A022BD9
S3150802557003D9032387F85B3105E03D4B5B6A03F0E9
S315080255800103002BEDD097F85B31002B40F0938096
S31508025590364BD3F8F03003F44073C7F85C31D7F8CA
S315080255A05C31002B23D0D7F84C31D3F8F820D7F842
S315080255B05C3193421BD02D4BD3F8F03023F4407361
S315080255C0C7F85C31294BD3F8F030284A43F48033C4
S315080255D0C2F8F030254BD3F8F030244A23F480334E
S315080255E0C2F8F030214AD7F85C31C2F8F030D7F861
S315080255F05C3103F00103002B19D0FBF775FEC7F8DF
S3150802560054010DE0FBF770FE0246D7F85431D21A60
S3150802561041F288339A4203D9032387F85B3106E0BD
S31508025620124BD3F8F03003F00203002BEAD097F8B6
S315080256305B31002B3AD1D7F84C31D3F8F83003F462
S315080256404073B3F5407F15D1084BDB6923F47C51CF
S31508025650D7F84C31D3F8F8301B0923F07F4323F0EF
S315080256603003024A0B43D3610AE000BF000C02442E
S31508025670000802449F4BDB699E4A23F47C53D3619C
S315080256809C4BD3F8F0309B4A23F44073C2F8F030AF
S31508025690984BD3F8F010D7F84C31D3F8F830C3F357
S315080256A00B03944A0B43C2F8F03008E097F85B31D3
S315080256B087F85A3103E097F85B3187F85A31D7F8F9
S315080256C04C31D3E9002302F080633B6600237B66F4
S315080256D0D7E918120B46134335D0D7F84C31D3F80D
S315080256E0C830302B14D0302B0ED8202B12D0202BBA
S315080256F00AD8002B10D0102B06D17E4B9B6A7D4A06
S3150802570043F40033936208E0012387F85B3104E02F
S3150802571000BF02E000BF00E000BF97F85B31002B34
S315080257200DD1744BD3F8E83023F03001D7F84C3159
S31508025730D3F8C8306F4A0B43C2F8E83003E097F84B
S315080257405B3187F85A31D7F84C31D3E9002302F492
S315080257508003BB650023FB65D7E916120B46134384
S3150802576033D0D7F84C31D3F8CC30002B02D0402BAB
S3150802577007D010E05F4B9B6A5E4A43F4003393629C
S315080257800DE0D7F84C310833184603F06FFB034691
S3150802579087F85B3103E0012387F85B3100BF97F88E
S315080257A05B31002B0DD1534BD3F8E43023F0400183
S315080257B0D7F84C31D3F8CC304E4A0B43C2F8E43012
S315080257C003E097F85B3187F85A31D7F84C31D3E9B9
S315080257D0002302F400033B6500237B65D7E9141214
S315080257E00B46134333D0D7F84C31D3F8D030002BBD
S315080257F002D0802B07D010E03E4B9B6A3D4A43F409
S31508025800003393620DE0D7F84C310833184603F09B
S315080258102DFB034687F85B3103E0012387F85B31EA
S3150802582000BF97F85B31002B0DD1324BD3F8E43029
S3150802583023F08001D7F84C31D3F8D0302D4A0B43E8
S31508025840C2F8E43003E097F85B3187F85A31D7F8A3
S315080258504C31D3E9002302F00063BB640023FB64E6
S31508025860D7E912120B4613434AD0D7F84C31D3F86C
S31508025870E030042B27D801A252F823F091580208E7
S315080258809F580208B3580208CF580208CF58020890
S31508025890184B9B6A174A43F40033936218E0D7F809
S315080258A04C310833184603F0E1FA034687F85B31B0
S315080258B00EE0D7F84C313033184603F06FFB034637
S315080258C087F85B3104E0012387F85B3100E000BF0B
S315080258D097F85B31002B0FD1064BD3F8E03023F053
S315080258E00701D7F84C31D3F8E030024A0B43C2F825
S315080258F0E03005E0000C024497F85B3187F85A312C
S31508025900D7F84C31D3E9002302F080533B640023D5
S315080259107B64D7E910120B46134300F08180D7F84F
S315080259204C31D3F8E430202B5FD801A252F823F089
S31508025930B5590208EB590208EB590208EB59020855
S31508025940EB590208EB590208EB590208EB5902080F
S31508025950C3590208EB590208EB590208EB59020827
S31508025960EB590208EB590208EB590208EB590208EF
S31508025970D7590208EB590208EB590208EB590208F3
S31508025980EB590208EB590208EB590208EB590208CF
S31508025990F3590208EB590208EB590208EB590208B7
S315080259A0EB590208EB590208EB590208EB590208AF
S315080259B0F3590208AB4B9B6AAA4A43F40033936233
S315080259C018E0D7F84C310833184603F04FFA034665
S315080259D087F85B310EE0D7F84C313033184603F0BE
S315080259E0DDFA034687F85B3104E0012387F85B3169
S315080259F000E000BF97F85B31002B0DD1994BD3F825
S31508025A00E03023F03801D7F84C31D3F8E430954A20
S31508025A100B43C2F8E03003E097F85B3187F85A3156
S31508025A20D7F84C31D3E9002302F00053BB630023B5
S31508025A30FB63D7E90E120B4613434ED0D7F84C3107
S31508025A40D3F8E830B3F5807F2ED0B3F5807F27D818
S31508025A50C02B2BD0C02B23D8802B17D0802B1FD836
S31508025A60002B02D0402B07D01AE07E4B9B6A7D4A58
S31508025A7043F4003393621AE0D7F84C3108331846D8
S31508025A8003F0F4F9034687F85B3110E0D7F84C3196
S31508025A903033184603F082FA034687F85B3106E08C
S31508025AA0012387F85B3102E000BF00E000BF97F8E8
S31508025AB05B31002B0DD16B4BD3F8E03023F4E07148
S31508025AC0D7F84C31D3F8E830664A0B43C2F8E030CF
S31508025AD003E097F85B3187F85A31D7F84C31D3E9A6
S31508025AE0002302F080433B6300237B63D7E90C1251
S31508025AF00B46134355D0D7F84C31D3F8EC30B3F5EF
S31508025B00206F31D0B3F5206F2AD8B3F5006F2DD0A8
S31508025B10B3F5006F24D8B3F5C06F29D0B3F5C06FBB
S31508025B201ED8B3F5806F11D0B3F5806F18D8002B45
S31508025B3020D0B3F5007F13D1D7F84C310833184675
S31508025B4003F094F9034687F85B3114E0D7F84C3131
S31508025B503033184603F022FA034687F85B310AE027
S31508025B60012387F85B3106E000BF04E000BF02E0CC
S31508025B7000BF00E000BF97F85B31002B0DD1394B0F
S31508025B80D3F8E03023F46061D7F84C31D3F8EC301F
S31508025B90344A0B43C2F8E03003E097F85B3187F8E2
S31508025BA05A31D7F84C31D3E9002302F00043BB62DD
S31508025BB00023FB62D7E90A120B46134358D0D7F8DB
S31508025BC04C31D3F8F030B3F5A04F31D0B3F5A04F2E
S31508025BD02AD8B3F5804F2DD0B3F5804F24D8B3F524
S31508025BE0405F29D0B3F5405F1ED8B3F5005F11D0E8
S31508025BF0B3F5005F18D8002B20D0B3F5805F13D118
S31508025C00D7F84C310833184603F030F9034687F8BB
S31508025C105B3114E0D7F84C313033184603F0BEF93D
S31508025C20034687F85B310AE0012387F85B3106E011
S31508025C3000BF04E000BF02E000BF00E000BF97F823
S31508025C405B31002B10D1074BD3F8E03023F4E04246
S31508025C50D7F84C31D3F8F03002491343C1F8E03093
S31508025C6006E000BF000C024497F85B3187F85A3108
S31508025C70D7F84C31D3E900230021396203F0010336
S31508025C807B62D7E908120B46134355D0D7F84C3135
S31508025C90D3F8F430B3F5203F31D0B3F5203F2AD8F4
S31508025CA0B3F5003F2DD0B3F5003F24D8B3F5C03F76
S31508025CB029D0B3F5C03F1ED8B3F5803F11D0B3F54E
S31508025CC0803F18D8002B20D0B3F5004F13D1D7F850
S31508025CD04C310833184603F0C9F8034687F85B3196
S31508025CE014E0D7F84C313033184603F057F9034617
S31508025CF087F85B310AE0012387F85B3106E000BFCB
S31508025D0004E000BF02E000BF00E000BF97F85B3185
S31508025D10002B0DD1884BD3F8E03023F46032D7F844
S31508025D204C31D3F8F43084491343C1F8E03003E028
S31508025D3097F85B3187F85A31D7F84C31D3E9002303
S31508025D400021B96103F00203FB61D7E906120B468B
S31508025D5013433DD0D7F84C31D3F8DC30032B1CD88B
S31508025D6001A252F823F000BFA35D0208795D02087A
S31508025D70875D0208A35D02086F4B9B6A6E4A43F46D
S31508025D80003393620EE0D7F84C310833184603F015
S31508025D906DF8034687F85B3104E0012387F85B3127
S31508025DA000E000BF97F85B31002B0DD1624BD3F8A8
S31508025DB0E43023F00302D7F84C31D3F8DC305E49DD
S31508025DC01343C1F8E43003E097F85B3187F85A3198
S31508025DD0D7F84C31D3E900230021396103F00403D3
S31508025DE07B61D7E904120B4613433AD0D7F84C31F4
S31508025DF0D3F8BC30B3F5007F0ED0B3F5007F15D8C3
S31508025E00002B17D0B3F5807F10D14B4B9B6A4A4AB9
S31508025E1043F4003393620EE0D7F84C310833184640
S31508025E2003F024F8034687F85B3104E0012387F878
S31508025E305B3100E000BF97F85B31002B0DD13E4B7A
S31508025E40D3F8E83023F44072D7F84C31D3F8BC3093
S31508025E5039491343C1F8E83003E097F85B3187F80C
S31508025E605A31D7F84C31D3E900230021B96003F03F
S31508025E701003FB60D7E902120B46134338D0D7F852
S31508025E804C31D3F80031302B1BD0302B15D8102BC0
S31508025E9002D0202B07D010E0274B9B6A264A43F4F0
S31508025EA0003393620EE0D7F84C313033184603F0CC
S31508025EB075F8034687F85B3104E0012387F85B31FE
S31508025EC000E000BF97F85B31002B0DD11A4BD3F8CF
S31508025ED0E43023F03002D7F84C31D3F800311649B2
S31508025EE01343C1F8E43003E097F85B3187F85A3177
S31508025EF0D7F84C31D3E900230021396003F00803AF
S31508025F007B60D7E900120B4613430CD00A4BD3F831
S31508025F10E83023F0C002D7F84C31D3F8FC300649F2
S31508025F201343C1F8E83097F85A31184607F5B0779F
S31508025F30BD46BDE8B08F00BF000C024480B48BB0EA
S31508025F4000AF7860AD4B5B6BC3F308033B62AB4BA8
S31508025F509B6A03F00303FB61A84B9B6A1B0A03F0C7
S31508025F603F03BB61A54B9B6A03F010037B61A34BFE
S31508025F709B6BDB08C3F30C037A6902FB03F307EE98
S31508025F80903AF8EE677AC7ED047ABB69002B00F0FF
S31508025F902681FB69032B53D0FB69032B6FD8FB6958
S31508025FA0012B03D0FB69022B2BD068E0934B1B68AD
S31508025FB0DB0803F00303924A22FA03F3FB60FB6849
S31508025FC007EE903AF8EE676ABB6907EE903AF8EE82
S31508025FD0677A86EEA77A3B6A07EE903AF8EE676A20
S31508025FE097ED046ADFED875AC6EE257A76EEA77A2A
S31508025FF0F7EE006A77EEA67A67EE277AC7ED097A90
S3150802600068E0BB6907EE903AF8EE677ADFED7E6ADA
S3150802601086EEA77A3B6A07EE903AF8EE676A97ED3C
S31508026020046ADFED785AC6EE257A76EEA77AF7EE97
S31508026030006A77EEA67A67EE277AC7ED097A49E00B
S31508026040BB6907EE903AF8EE677ADFED706A86EE7C
S31508026050A77A3B6A07EE903AF8EE676A97ED046A02
S31508026060DFED685AC6EE257A76EEA77AF7EE006A6B
S3150802607077EEA67A67EE277AC7ED097A2AE05F4BAA
S315080260801B68DB0803F003035D4A22FA03F3FB608D
S31508026090FB6807EE903AF8EE676ABB6907EE903A34
S315080260A0F8EE677A86EEA77A3B6A07EE903AF8EE3A
S315080260B0676A97ED046ADFED535AC6EE257A76EEDD
S315080260C0A77AF7EE006A77EEA67A67EE277AC7ED21
S315080260D0097A00BF494B1B6803F00073B3F1007FCE
S315080260E021D1464B9B6A03F48033002B17D0434BCE
S315080260F05B6B5B0A03F07F0307EE903AF8EE677A6A
S31508026100B7EE007A37EE877AD7ED096AC6EE877A4E
S31508026110FCEEE77A17EE902A7B681A6006E07B683F
S3150802612000221A6002E07B6800221A60334B1B6861
S3150802613003F00073B3F1007F21D1304B9B6A03F45D
S315080261400033002B17D02D4B5B6B1B0C03F07F0320
S3150802615007EE903AF8EE677AB7EE007A37EE877A64
S31508026160D7ED096AC6EE877AFCEEE77A17EE902A29
S315080261707B685A6006E07B6800225A6002E07B6808
S3150802618000225A601D4B1B6803F00073B3F1007FAF
S3150802619021D11A4B9B6A03F48023002B17D0174B85
S315080261A05B6B1B0E03F07F0307EE903AF8EE677AF5
S315080261B0B7EE007A37EE877AD7ED096AC6EE877A9E
S315080261C0FCEEE77A17EE902A7B689A6010E07B6805
S315080261D000229A600CE07B6800229A6008E07B68DD
S315080261E000221A607B6800225A607B6800229A6045
S315080261F000BF2C37BD465DF8047B7047000C02448D
S315080262000090D003000000460024744A001B374B56
S3150802621080B48BB000AF7860AD4BDB6BC3F3080379
S315080262203B62AB4BDB6A03F00303FB61A84BDB6AF9
S315080262301B0A03F03F03BB61A54BDB6A03F010039D
S315080262407B61A34B1B6CDB08C3F30C037A6902FB65
S3150802625003F307EE903AF8EE677AC7ED047ABB695C
S31508026260002B00F02681FB69032B53D0FB69032B15
S315080262706FD8FB69012B03D0FB69022B2BD068E090
S31508026280934B1B68DB0803F00303924A22FA03F3D3
S31508026290FB60FB6807EE903AF8EE676ABB6907EEA1
S315080262A0903AF8EE677A86EEA77A3B6A07EE903A54
S315080262B0F8EE676A97ED046ADFED875AC6EE257A25
S315080262C076EEA77AF7EE006A77EEA67A67EE277A6F
S315080262D0C7ED097A68E0BB6907EE903AF8EE677A85
S315080262E0DFED7E6A86EEA77A3B6A07EE903AF8EE0B
S315080262F0676A97ED046ADFED785AC6EE257A76EE76
S31508026300A77AF7EE006A77EEA67A67EE277AC7EDDE
S31508026310097A49E0BB6907EE903AF8EE677ADFED4B
S31508026320706A86EEA77A3B6A07EE903AF8EE676AD3
S3150802633097ED046ADFED685AC6EE257A76EEA77AF5
S31508026340F7EE006A77EEA67A67EE277AC7ED097A3C
S315080263502AE05F4B1B68DB0803F003035D4A22FA57
S3150802636003F3FB60FB6807EE903AF8EE676ABB69CF
S3150802637007EE903AF8EE677A86EEA77A3B6A07EE58
S31508026380903AF8EE676A97ED046ADFED535AC6EE5D
S31508026390257A76EEA77AF7EE006A77EEA67A67EEA0
S315080263A0277AC7ED097A00BF494B1B6803F00063D9
S315080263B0B3F1006F21D1464BDB6A03F48033002B1D
S315080263C017D0434BDB6B5B0A03F07F0307EE903A69
S315080263D0F8EE677AB7EE007A37EE877AD7ED096A6A
S315080263E0C6EE877AFCEEE77A17EE902A7B681A6081
S315080263F006E07B6800221A6002E07B6800221A60C7
S31508026400334B1B6803F00063B3F1006F21D1304BA5
S31508026410DB6A03F40033002B17D02D4BDB6B1B0C06
S3150802642003F07F0307EE903AF8EE677AB7EE007A42
S3150802643037EE877AD7ED096AC6EE877AFCEEE77AEF
S3150802644017EE902A7B685A6006E07B6800225A603B
S3150802645002E07B6800225A601D4B1B6803F000634A
S31508026460B3F1006F21D11A4BDB6A03F48023002BA8
S3150802647017D0174BDB6B1B0E03F07F0307EE903A20
S31508026480F8EE677AB7EE007A37EE877AD7ED096AB9
S31508026490C6EE877AFCEEE77A17EE902A7B689A6050
S315080264A010E07B6800229A600CE07B6800229A6002
S315080264B008E07B6800221A607B6800225A607B68C3
S315080264C000229A6000BF2C37BD465DF8047B7047F0
S315080264D0000C02440090D003000000460024744ACF
S315080264E0001B374B80B48BB000AF7860AD4B5B6C4A
S315080264F0C3F308033B62AB4B1B6B03F00303FB615D
S31508026500A84B1B6B1B0A03F03F03BB61A54B1B6B16
S3150802651003F010037B61A34B9B6CDB08C3F30C03EC
S315080265207A6902FB03F307EE903AF8EE677AC7ED4B
S31508026530047ABB69002B00F02681FB69032B53D032
S31508026540FB69032B6FD8FB69012B03D0FB69022B6E
S315080265502BD068E0934B1B68DB0803F00303924ACF
S3150802656022FA03F3FB60FB6807EE903AF8EE676AD5
S31508026570BB6907EE903AF8EE677A86EEA77A3B6A27
S3150802658007EE903AF8EE676A97ED046ADFED875AE6
S31508026590C6EE257A76EEA77AF7EE006A77EEA67A3F
S315080265A067EE277AC7ED097A68E0BB6907EE903A83
S315080265B0F8EE677ADFED7E6A86EEA77A3B6A07EE21
S315080265C0903AF8EE676A97ED046ADFED785AC6EEF6
S315080265D0257A76EEA77AF7EE006A77EEA67A67EE5E
S315080265E0277AC7ED097A49E0BB6907EE903AF8EED1
S315080265F0677ADFED706A86EEA77A3B6A07EE903A0B
S31508026600F8EE676A97ED046ADFED685AC6EE257AF0
S3150802661076EEA77AF7EE006A77EEA67A67EE277A1B
S31508026620C7ED097A2AE05F4B1B68DB0803F0030310
S315080266305D4A22FA03F3FB60FB6807EE903AF8EE2E
S31508026640676ABB6907EE903AF8EE677A86EEA77A2A
S315080266503B6A07EE903AF8EE676A97ED046ADFED51
S31508026660535AC6EE257A76EEA77AF7EE006A77EEE1
S31508026670A67A67EE277AC7ED097A00BF494B1B68E7
S3150802668003F00053B3F1005F21D1464B1B6B03F4B1
S315080266908033002B17D0434B5B6C5B0A03F07F03F6
S315080266A007EE903AF8EE677AB7EE007A37EE877A0F
S315080266B0D7ED096AC6EE877AFCEEE77A17EE902AD4
S315080266C07B681A6006E07B6800221A6002E07B6833
S315080266D000221A60334B1B6803F00053B3F1005FC4
S315080266E021D1304B1B6B03F40033002B17D02D4BF3
S315080266F05B6C1B0C03F07F0307EE903AF8EE677AA1
S31508026700B7EE007A37EE877AD7ED096AC6EE877A48
S31508026710FCEEE77A17EE902A7B685A6006E07B68F9
S3150802672000225A6002E07B6800225A601D4B1B68F1
S3150802673003F00053B3F1005F21D11A4B1B6B03F42C
S315080267408023002B17D0174B5B6C1B0E03F07F03BD
S3150802675007EE903AF8EE677AB7EE007A37EE877A5E
S31508026760D7ED096AC6EE877AFCEEE77A17EE902A23
S315080267707B689A6010E07B6800229A600CE07B686E
S3150802678000229A6008E07B6800221A607B68002271
S315080267905A607B6800229A6000BF2C37BD465DF8B6
S315080267A0047B7047000C02440090D00300000046A8
S315080267B00024744A001B374B90B58FB000AFC7E967
S315080267C00001D7E9000100F17E44214350D1264B4E
S315080267D0D3F8F03003F440733B63234BD3F8F0301D
S315080267E003F00203022B08D13B6BB3F5807F04D179
S315080267F04FF400437B6302F02ABB1B4BD3F8F030FD
S3150802680003F00063B3F1006F08D13B6BB3F5007F69
S3150802681004D14FF4FA437B6302F019BB124B1B688F
S3150802682003F40033B3F5003F19D13B6BB3F5407F50
S3150802683015D10D4BDB6903F47C53B3F5007F0AD3FC
S31508026840094BDB691B0A03F03F03084AB2FBF3F361
S315080268507B6302F0FCBA00237B6302F0F8BA0023DA
S315080268607B6302F0F4BA00BF000C0244001BB700B7
S31508026870D7E90001A1F5806450EA040101F07582A6
S31508026880D7E90001012871F5806182F0DD82D7E936
S315080268900001A1F5007450EA040101F06C81D7E900
S315080268A00001012871F5007182F0CE82D7E9000154
S315080268B0A1F5807450EA040101F00286D7E90001C5
S315080268C0012871F5807182F0BF82D7E90001A1F132
S315080268D0800450EA040101F04C85D7E90001012839
S315080268E071F1800182F0B082D7E90001A1F140047A
S315080268F050EA040101F09E84D7E90001012871F1EA
S31508026900400182F0A182D7E90001A1F1200450EAF0
S31508026910040101F0E883D7E90001012871F1200199
S3150802692082F09282D7E90001A1F1100450EA04012B
S3150802693002F05682D7E90001012871F1100182F0AE
S315080269408382D7E90001A1F1080450EA040102F0A2
S31508026950CC81D7E90001012871F1080182F074821D
S31508026960D7E900010C1F50EA040101F04886D7E96D
S315080269700001012871F1040182F06682D7E900015B
S315080269808C1E50EA040102F04381D7E9000101286E
S3150802699071F1020182F05882D7E900014C1E50EAD1
S315080269A0040102F0CE80D7E90001012871F1010144
S315080269B082F04A82D7E9000100F10044214302F03D
S315080269C05980D7E90001D94CA04271F1000182F041
S315080269D03B82D7E9000100F14044214301F0D987FF
S315080269E0D7E90001D24CA04271F1000182F02C8253
S315080269F0D7E9000100F16044214301F05187D7E944
S31508026A000001CC4CA04271F1000182F01D82D7E947
S31508026A10000100F17044214301F09A86D7E900018A
S31508026A20C54CA04271F1000182F00E82D7E900013D
S31508026A3000F17844214301F01286D7E90001BF4CE0
S31508026A40A04271F1000182F0FF81D7E9000100F14D
S31508026A507C44214302F07E81D7E90001B84CA0426A
S31508026A6071F1000182F0F081D7E90001A0F5000476
S31508026A70214300F09E82D7E90001B24CA04271F18F
S31508026A80000182F0E181D7E90001A0F580042143E3
S31508026A9000F06D82D7E90001AB4CA04271F100010A
S31508026AA082F0D281D7E90001A0F50014214301F052
S31508026AB00D80D7E90001A54CA04271F1000182F0D0
S31508026AC0C381D7E90001A0F58014214300F0D081E3
S31508026AD0D7E900019E4CA04271F1000182F0B4810F
S31508026AE0D7E90001A0F50024214300F04281D7E945
S31508026AF00001984CA04271F1000182F0A581D7E904
S31508026B000001A0F58024214301F04E82D7E9000155
S31508026B10914CA04271F1000182F09681D7E90001F9
S31508026B20A0F50034214301F09781D7E900018B4C87
S31508026B30A04271F1000182F08781D7E90001A0F530
S31508026B408034214301F05481D7E90001B0F1011FD5
S31508026B5071F1000182F07881D7E90001A0F50044BD
S31508026B60214301F0B780D7E9000148F20104A042A7
S31508026B7071F1000182F06881D7E90001A0F580442D
S31508026B80214301F06480D7E9000144F20104A042DE
S31508026B9071F1000182F05881D7E90001A0F500548D
S31508026BA0214301F01180D7E9000142F20104A04213
S31508026BB071F1000182F04881D7E90001A0F58054FD
S31508026BC0214300F01E87D7E9000141F20104A042E1
S31508026BD071F1000182F03881D7E90001A0F500645D
S31508026BE0214300F0A886D7E9000140F60104A04235
S31508026BF071F1000182F02881D7E90001A0F58064CD
S31508026C00214300F03286D7E9000140F20144A0424E
S31508026C1071F1000182F01881D7E90001A0F500742C
S31508026C20214300F0B085D7E9000140F20124A042D1
S31508026C3071F1000182F00881D7E90001A0F580749C
S31508026C40214300F03585D7E9000140F20114A0423C
S31508026C5071F1000182F0F880D7E90001A0F1800401
S31508026C60214300F0BA84D7E90001812871F10001B5
S31508026C7082F0EA80D7E90001212871F100016FD27A
S31508026C80D7E90001014302F0DF80D7E90001421E7D
S31508026C9041F1FF33202A73F1000182F0D5801F2AC1
S31508026CA002F2D28001A151F822F000BF0D7002084B
S31508026CB0D9700208498E020899710208498E02089B
S31508026CC0498E0208498E020869720208498E02082C
S31508026CD0498E0208498E0208498E0208498E020820
S31508026CE0498E0208498E02084B730208498E020829
S31508026CF0498E0208498E0208498E0208498E020800
S31508026D00498E0208498E0208498E0208498E0208EF
S31508026D10498E0208498E0208498E0208498E0208DF
S31508026D20498E0208498E0208217402080100008071
S31508026D3001000040010000200100001001000008C7
S31508026D40010000040100800001004000010020004B
S31508026D500100100001000800010004000100020001
S31508026D60D7E90023A2F140010B4300F0C48302F0E5
S31508026D706BB8A14BD3F8E83003F4E0233B633B6BD3
S31508026D80B3F5802F36D03B6BB3F5802F6BD83B6BB0
S31508026D90B3F5403F2BD03B6BB3F5403F63D83B6B13
S31508026DA0B3F5003F1BD03B6BB3F5003F5BD83B6B9B
S31508026DB0002B04D03B6BB3F5803F08D053E007F1B4
S31508026DC020031846FFF7BAF87B6A7B634EE007F1A1
S31508026DD014031846FFF71CFA7B697B6346E007F142
S31508026DE008031846FFF77EFBBB687B633EE0834BCE
S31508026DF07B633BE0804BD3F8E83003F04043FB6209
S31508026E007D4B1B6803F00203022B0CD1FB6A002B95
S31508026E1009D1794B1B68DB0803F00303784A22FA87
S31508026E2003F37B631EE0744B1B6803F40073B3F52C
S31508026E30007F06D1FB6AB3F1804F02D1714B7B63A7
S31508026E4010E06D4B1B6803F40033B3F5003F06D11F
S31508026E50FB6AB3F1004F02D16B4B7B6302E000235E
S31508026E607B6303E002E000237B6300BF01F0EFBF10
S31508026E70614BD3F8E83003F460133B633B6BB3F51D
S31508026E80001F36D03B6BB3F5001F6BD83B6BB3F5CF
S31508026E90C01F2BD03B6BB3F5C01F63D83B6BB3F552
S31508026EA0801F1BD03B6BB3F5801F5BD83B6B002B57
S31508026EB004D03B6BB3F5002F08D053E007F120034B
S31508026EC01846FFF73BF87B6A7B634EE007F114032B
S31508026ED01846FFF79DF97B697B6346E007F10803CD
S31508026EE01846FFF7FFFABB687B633EE0434B7B63BA
S31508026EF03BE0414BD3F8E83003F04043FB623E4B9C
S31508026F001B6803F00203022B0CD1FB6A002B09D182
S31508026F10394B1B68DB0803F00303394A22FA03F3E9
S31508026F207B631EE0344B1B6803F40073B3F5007FE2
S31508026F3006D1FB6AB3F1804F02D1324B7B6310E074
S31508026F402D4B1B6803F40033B3F5003F06D1FB6AE9
S31508026F50B3F1004F02D12C4B7B6302E000237B6323
S31508026F6003E002E000237B6300BF01F070BF224BFF
S31508026F70D3F8E43003F040033B633B6B002B08D1A4
S31508026F8007F120031846FEF7D9FF7B6A7B6301F0F7
S31508026F905EBF3B6B402B08D107F114031846FFF777
S31508026FA037F9FB697B6301F052BF00237B6301F06B
S31508026FB04EBF114BD3F8E43003F080033B633B6BBF
S31508026FC0002B08D107F120031846FEF7B7FF7B6AA4
S31508026FD07B6301F03CBF3B6B802B08D107F114039E
S31508026FE01846FFF715F9FB697B6301F030BF0023EA
S31508026FF07B6301F02CBF00BF000C02440080BB007B
S315080270000090D00300093D00001BB7009D4BD3F842
S31508027010D83003F007033B633B6B002B04D1FCF724
S315080270209FFF786301F013BF964B1B6803F000635A
S31508027030B3F1006F0AD13B6B012B07D107F1140399
S315080270401846FFF7E5F8BB697B6343E08D4B1B687F
S3150802705003F00053B3F1005F0AD13B6B022B07D151
S3150802706007F108031846FFF73DFAFB687B6331E030
S31508027070844B1B6803F00203022B0CD13B6B032BD8
S3150802708009D1804B1B68DB0803F003037E4A22FA08
S3150802709003F37B631EE07B4B1B6803F40073B3F5B3
S315080270A0007F05D13B6B042B02D1784B7B6311E041
S315080270B0744BD3F8F03003F00203022B06D13B6B74
S315080270C0052B03D14FF400437B6303E000237B6364
S315080270D001F0BDBE01F0BBBE6A4BD3F8D83003F04F
S315080270E038033B633B6B002B04D1FCF723FF786321
S315080270F001F0ADBE634B1B6803F00063B3F1006F8A
S315080271000AD13B6B082B07D107F114031846FFF780
S315080271107FF8BB697B633DE03B6B102B08D107F117
S3150802712008031846FFF7DEF9FB687B6301F08FBE9A
S31508027130544B1B6803F00203022B0CD13B6B182B32
S3150802714009D1504B1B68DB0803F003034E4A22FAA7
S3150802715003F37B631EE04B4B1B6803F40073B3F522
S31508027160007F05D13B6B202B02D1484B7B6311E094
S31508027170444BD3F8F03003F00203022B06D13B6BE3
S31508027180282B03D14FF400437B6303E000237B6380
S3150802719001F05DBE01F05BBE3A4BD3F8D83003F47A
S315080271A0E0733B633B6B002B04D1FCF7C3FE7863A9
S315080271B001F04DBE334B1B6803F00063B3F1006F59
S315080271C00AD13B6B402B07D107F114031846FFF788
S315080271D01FF8BB697B6345E02A4B1B6803F0005323
S315080271E0B3F1005F0AD13B6B802B07D107F1080385
S315080271F01846FFF777F9FB687B6333E0214B1B6878
S3150802720003F00203022B0CD13B6BC02B09D11D4B99
S315080272101B68DB0803F003031B4A22FA03F37B63AA
S3150802722020E0184B1B6803F40073B3F5007F06D100
S315080272303B6BB3F5807F02D1144B7B6312E0114B93
S31508027240D3F8F03003F00203022B07D13B6BB3F5F8
S31508027250A07F03D14FF400437B6303E000237B63E3
S3150802726001F0F5BD01F0F3BD064BD3F8D83003F4AF
S3150802727060633B633B6B002B0AD1FCF75BFE7863CA
S3150802728001F0E5BD000C02440090D00300093D0060
S31508027290A04B1B6803F00063B3F1006F0BD13B6B85
S315080272A0B3F5007F07D107F114031846FEF7B0FFBE
S315080272B0BB697B6347E0974B1B6803F00053B3F146
S315080272C0005F0BD13B6BB3F5806F07D107F108035B
S315080272D01846FFF707F9FB687B6334E08D4B1B689A
S315080272E003F00203022B0DD13B6BB3F5C06F09D134
S315080272F0884B1B68DB0803F00303874A22FA03F369
S315080273007B6320E0834B1B6803F40073B3F5007FAD
S3150802731006D13B6BB3F5006F02D1804B7B6312E05B
S315080273207C4BD3F8F03003F00203022B07D13B6BF8
S31508027330B3F5206F03D14FF400437B6303E00023C8
S315080273407B6301F084BD01F082BD724BD3F8D8305D
S3150802735003F4E0433B633B6B002B04D1FCF7EAFDE5
S31508027360786301F074BD6B4B1B6803F00063B3F1DD
S31508027370006F0BD13B6BB3F5805F07D107F114039E
S315080273801846FEF745FFBB697B6347E0614B1B68FE
S3150802739003F00053B3F1005F0BD13B6BB3F5005F0B
S315080273A007D107F108031846FFF79CF8FB687B63C9
S315080273B034E0584B1B6803F00203022B0DD13B6BDA
S315080273C0B3F5405F09D1534B1B68DB0803F003038F
S315080273D0514A22FA03F37B6320E04E4B1B6803F4FF
S315080273E00073B3F5007F06D13B6BB3F5804F02D12C
S315080273F04A4B7B6312E0474BD3F8F03003F00203A3
S31508027400022B07D13B6BB3F5A04F03D14FF40043D0
S315080274107B6303E000237B6301F019BD01F017BD0E
S315080274203C4BD3F8D83003F460333B633B6B002BF9
S3150802743004D1FCF77FFD786301F009BD354B1B6863
S3150802744003F00063B3F1006F0BD13B6BB3F5004F4A
S3150802745007D107F114031846FEF7DAFEBB697B6308
S3150802746047E02C4B1B6803F00053B3F1005F0BD1C6
S315080274703B6BB3F5803F07D107F108031846FFF7C0
S3150802748031F8FB687B6334E0224B1B6803F0020386
S31508027490022B0DD13B6BB3F5C03F09D11D4B1B68BF
S315080274A0DB0803F003031C4A22FA03F37B6320E09A
S315080274B0184B1B6803F40073B3F5007F06D13B6BC8
S315080274C0B3F5003F02D1154B7B6312E0114BD3F89B
S315080274D0F03003F00203022B07D13B6BB3F5203FD2
S315080274E003D14FF400437B6303E000237B6301F07F
S315080274F0AEBC01F0ACBC074BD3F8D83003F4E013AA
S315080275003B633B6B002B0BD1FCF714FD786301F050
S315080275109EBC00BF000C02440090D00300093D0047
S31508027520A04B1B6803F00063B3F1006F0BD13B6BF2
S31508027530B3F5802F07D107F114031846FEF768FE44
S31508027540BB697B6347E0974B1B6803F00053B3F1B3
S31508027550005F0BD13B6BB3F5002F07D107F1080388
S315080275601846FEF7BFFFFB687B6334E08D4B1B684A
S3150802757003F00203022B0DD13B6BB3F5402F09D161
S31508027580884B1B68DB0803F00303874A22FA03F3D6
S315080275907B6320E0834B1B6803F40073B3F5007F1B
S315080275A006D13B6BB3F5801F02D1804B7B6312E099
S315080275B07C4BD3F8F03003F00203022B07D13B6B66
S315080275C0B3F5A01F03D14FF400437B6303E0002306
S315080275D07B6301F03CBC01F03ABC724BD3F8D8305D
S315080275E003F460033B633B6B002B04D1FCF7A2FC5C
S315080275F0786301F02CBC6B4B1B6803F00063B3F194
S31508027600006F0BD13B6BB3F5001F07D107F11403CB
S315080276101846FEF7FDFDBB697B6347E0614B1B68B5
S3150802762003F00053B3F1005F0BD13B6BB3F5800F48
S3150802763007D107F108031846FEF754FFFB687B6378
S3150802764034E0584B1B6803F00203022B0DD13B6B47
S31508027650B3F5C00F09D1534B1B68DB0803F00303CC
S31508027660514A22FA03F37B6320E04E4B1B6803F46C
S315080276700073B3F5007F06D13B6BB3F5000F02D159
S315080276804A4B7B6312E0474BD3F8F03003F0020310
S31508027690022B07D13B6BB3F5200F03D14FF40043FE
S315080276A07B6303E000237B6301F0D1BB01F0CFBB10
S315080276B03C4BD3F8D83003F0E0633B633B6B002BBB
S315080276C004D1FCF737FC786301F0C1BB354B1B6864
S315080276D003F00063B3F1006F0BD13B6BB3F1807F0C
S315080276E007D107F114031846FEF792FDBB697B63BF
S315080276F047E02C4B1B6803F00053B3F1005F0BD134
S315080277003B6BB3F1007F07D107F108031846FEF772
S31508027710E9FEFB687B6334E0224B1B6803F0020335
S31508027720022B0DD13B6BB3F1407F09D11D4B1B6870
S31508027730DB0803F003031C4A22FA03F37B6320E007
S31508027740184B1B6803F40073B3F5007F06D13B6B35
S31508027750B3F1806F02D1154B7B6312E0114BD3F85C
S31508027760F03003F00203022B07D13B6BB3F1A06F93
S3150802777003D14FF400437B6303E000237B6301F0EC
S3150802778066BB01F064BB074BD3F8D83003F06053ED
S315080277903B633B6B002B0BD1FCF7CCFB786301F008
S315080277A056BB00BF000C02440090D00300093D00FE
S315080277B0A14B1B6803F00063B3F1006F0BD13B6B5F
S315080277C0B3F1006F07D107F114031846FEF720FD3F
S315080277D0BB697B6347E0984B1B6803F00053B3F120
S315080277E0005F0BD13B6BB3F1805F07D107F108034A
S315080277F01846FEF777FEFB687B6334E08E4B1B6800
S3150802780003F00203022B0DD13B6BB3F1C05F09D122
S31508027810894B1B68DB0803F00303884A22FA03F341
S315080278207B6320E0844B1B6803F40073B3F5007F87
S3150802783006D13B6BB3F1005F02D1814B7B6312E049
S315080278407D4BD3F8F03003F00203022B07D13B6BD2
S31508027850B3F1205F03D14FF400437B6303E00023B7
S315080278607B6301F0F4BA01F0F2BA734BD3F8DC3059
S3150802787003F007033B633B6B002B04D1FCF75AFB6F
S31508027880786301F0E4BA6C4B1B6803F00063B3F14A
S31508027890006F0AD13B6B012B07D107F11403184677
S315080278A0FEF7B6FCBB697B6343E0634B1B6803F0D8
S315080278B00053B3F1005F0AD13B6B022B07D107F1E4
S315080278C008031846FEF70EFEFB687B6331E05A4B47
S315080278D01B6803F00203022B0CD13B6B032B09D165
S315080278E0554B1B68DB0803F00303544A22FA03F3D9
S315080278F07B631EE0504B1B6803F40073B3F5007FED
S3150802790005D13B6B042B02D14D4B7B6311E04A4BED
S31508027910D3F8F03003F00203022B06D13B6B052B9A
S3150802792003D14FF400437B6303E000237B6301F03A
S315080279308EBA01F08CBA404BD3F8DC3003F07003F0
S315080279403B633B6B002B04D1FCF7F4FA786301F036
S315080279507EBA394B1B6803F00063B3F1006F0AD194
S315080279603B6B102B07D107F114031846FEF750FCA0
S31508027970BB697B6343E0304B1B6803F00053B3F1EA
S31508027980005F0AD13B6B202B07D107F10803184683
S31508027990FEF7A8FDFB687B6331E0274B1B6803F003
S315080279A00203022B0CD13B6B302B09D1224B1B68ED
S315080279B0DB0803F00303214A22FA03F37B631EE082
S315080279C01D4B1B6803F40073B3F5007F05D13B6BAF
S315080279D0402B02D11A4B7B6311E0174BD3F8F030D8
S315080279E003F00203022B06D13B6B502B03D14FF453
S315080279F000437B6303E000237B6301F028BA01F0AE
S31508027A0026BA0D4BD3F8E03003F0E0633B633B6BD9
S31508027A10002B04D1FCF7BAFA786301F018BA3B6B6B
S31508027A20B3F1807F0ED107F114031846FEF7F0FB77
S31508027A30BB697B6301F00BBA000C02440090D003C9
S31508027A4000093D003B6BB3F1007F08D107F108033B
S31508027A501846FEF747FDFB687B6301F0F8B9A44BAD
S31508027A601B6803F00203022B0DD13B6BB3F1407F77
S31508027A7009D19F4B1B68DB0803F003039D4A22FAD0
S31508027A8003F37B6320E09A4B1B6803F40073B3F598
S31508027A90007F06D13B6BB3F1806F02D1964B7B63B5
S31508027AA012E0934BD3F8F03003F00203022B07D10E
S31508027AB03B6BB3F1A06F03D14FF400437B6303E042
S31508027AC000237B6301F0C3B901F0C1B9884BD3F82F
S31508027AD0E83003F007033B633B6B002B04D1FCF74A
S31508027AE00DFA786301F0B3B93B6B012B04D1FCF7AD
S31508027AF0D9F8786301F0ABB93B6B022B08D107F1D1
S31508027B0014031846FEF784FBFB697B6301F09FB9F1
S31508027B10774B1B6803F40033B3F5003F05D13B6B83
S31508027B20032B02D1754B7B6323E0714B1B6803F071
S31508027B300203022B0CD13B6B042B09D16C4B1B683D
S31508027B40DB0803F003036B4A22FA03F37B6310E0B4
S31508027B50674B1B6803F40073B3F5007F05D13B6BD3
S31508027B60052B02D1644B7B6303E000237B6301F0A0
S31508027B706EB901F06CB95E4BD3F8E83003F008032E
S31508027B803B635B4BD3F8F03003F00203022B06D1BA
S31508027B903B6B002B03D14FF400437B6312E0544B3B
S31508027BA0D3F8F03003F00063B3F1006F06D13B6BF4
S31508027BB0082B03D14FF4FA437B6303E000237B636C
S31508027BC001F045B901F043B9494BD3F8E43003F45F
S31508027BD040333B633B6B002B04D1FCF7ABF978636C
S31508027BE001F035B93B6BB3F5803F08D107F10803BD
S31508027BF01846FEF777FC3B697B6301F028B93C4BD4
S31508027C001B6803F00203022B0DD13B6BB3F5003F51
S31508027C1009D1374B1B68DB0803F00303354A22FAFE
S31508027C2003F37B6311E0324B1B6803F40073B3F56D
S31508027C30007F06D13B6BB3F5403F02D12E4B7B63E7
S31508027C4003E000237B6301F002B901F000B9284B77
S31508027C50D3F8E43003F440233B633B6B002B04D197
S31508027C60FCF768F9786301F0F2B83B6BB3F5802F3D
S31508027C7008D107F108031846FEF734FC3B697B6313
S31508027C8001F0E5B81A4B1B6803F00203022B0DD16B
S31508027C903B6BB3F5002F09D1154B1B68DB0803F0C4
S31508027CA00303144A22FA03F37B6311E0104B1B68A1
S31508027CB003F40073B3F5007F06D13B6BB3F5402F8F
S31508027CC002D10D4B7B6303E000237B6301F0BFB84F
S31508027CD001F0BDB8064BD3F8E43003F440133B6316
S31508027CE03B6B002B0CD1FCF751F9786301F0AFB866
S31508027CF0000C02440090D00300093D00001BB700A7
S31508027D003B6BB3F5801F08D107F108031846FEF747
S31508027D10E9FB3B697B6301F09AB89F4B1B6803F04A
S31508027D200203022B0DD13B6BB3F5001F09D19A4B07
S31508027D301B68DB0803F00303984A22FA03F37B6302
S31508027D4011E0954B1B6803F40073B3F5007F06D167
S31508027D503B6BB3F5401F02D1914B7B6303E00023D3
S31508027D607B6301F074B801F072B88B4BD3F8E43038
S31508027D7003F440033B633B6B002B04D1FCF706F983
S31508027D80786301F064B83B6BB3F5800F08D107F14D
S31508027D9008031846FEF7A6FB3B697B6301F057B852
S31508027DA07D4B1B6803F00203022B0DD13B6BB3F527
S31508027DB0000F09D1784B1B68DB0803F00303774AE7
S31508027DC022FA03F37B6311E0734B1B6803F4007317
S31508027DD0B3F5007F06D13B6BB3F5400F02D1704B6A
S31508027DE07B6303E000237B6301F031B801F02FB80F
S31508027DF0694BD3F8E43003F040733B633B6B002BCB
S31508027E0004D1FCF797F8786301F021B83B6BB3F11C
S31508027E10807F08D107F108031846FEF763FB3B6922
S31508027E207B6301F014B85C4B1B6803F00203022B58
S31508027E300ED13B6BB3F1007F0AD1574B1B68DB08A7
S31508027E4003F00303554A22FA03F37B6300F0FFBFEC
S31508027E5000237B6300F0FBBF4F4BD3F8DC3003F4FF
S31508027E60E0633B633B6BB3F5A06F56D03B6BB3F550
S31508027E70A06F00F28B803B6BB3F5806F3ED03B6BF5
S31508027E80B3F5806F00F282803B6BB3F5407F27D053
S31508027E903B6BB3F5407F79D83B6BB3F5007F17D0C0
S31508027EA03B6BB3F5007F71D83B6B002B04D03B6B61
S31508027EB0B3F5807F04D069E0FCF768F8786368E078
S31508027EC007F114031846FEF7A3F97B697B6360E0A2
S31508027ED007F108031846FEF705FB3B697B6358E082
S31508027EE02D4BD3F8F03003F00203022B03D14FF4E3
S31508027EF000437B634DE000237B634AE0264BD3F8BD
S31508027F00F03003F00063B3F1006F03D14FF4FA4384
S31508027F107B633EE000237B633BE01F4BD3F8E830EC
S31508027F2003F04043FB621C4B1B6803F00203022B5F
S31508027F300CD1FB6A002B09D1174B1B68DB0803F02F
S31508027F400303164A22FA03F37B631EE0124B1B68ED
S31508027F5003F40073B3F5007F06D1FB6AB3F1804FD1
S31508027F6002D10F4B7B6310E00B4B1B6803F4003303
S31508027F70B3F5003F06D1FB6AB3F1004F02D1094BB4
S31508027F807B6302E000237B6303E002E000237B635A
S31508027F9000BF00F05CBF00BF000C02440090D00393
S31508027FA000093D00001BB7009E4BD3F8DC3003F4F2
S31508027FB0E0433B633B6BB3F5A04F56D03B6BB3F53F
S31508027FC0A04F00F28B803B6BB3F5804F3ED03B6BE4
S31508027FD0B3F5804F00F282803B6BB3F5405F27D042
S31508027FE03B6BB3F5405F79D83B6BB3F5005F17D0AF
S31508027FF03B6BB3F5005F71D83B6B002B04D03B6B30
S31508028000B3F5805F04D069E0FBF794FF786368E014
S3150802801007F114031846FEF7FBF87B697B6360E0F9
S3150802802007F108031846FEF75DFA3B697B6358E0D9
S315080280307C4BD3F8F03003F00203022B03D14FF442
S3150802804000437B634DE000237B634AE0754BD3F81C
S31508028050F03003F00063B3F1006F03D14FF4FA4333
S315080280607B633EE000237B633BE06E4BD3F8E8304C
S3150802807003F04043FB626B4B1B6803F00203022BBF
S315080280800CD1FB6A002B09D1664B1B68DB0803F08F
S315080280900303654A22FA03F37B631EE0614B1B68FE
S315080280A003F40073B3F5007F06D1FB6AB3F1804F80
S315080280B002D15E4B7B6310E05A4B1B6803F4003314
S315080280C0B3F5003F06D1FB6AB3F1004F02D1584B14
S315080280D07B6302E000237B6303E002E000237B6309
S315080280E000BF00F0B4BE4F4BD3F8DC3003F4E023F4
S315080280F03B633B6BB3F5A02F56D03B6BB3F5A02F72
S3150802810000F28B803B6BB3F5802F3ED03B6BB3F509
S31508028110802F00F282803B6BB3F5403F27D03B6B42
S31508028120B3F5403F79D83B6BB3F5003F17D03B6BAD
S31508028130B3F5003F71D83B6B002B04D03B6BB3F50C
S31508028140803F04D069E0FBF721FF786368E007F116
S3150802815014031846FEF75CF87B697B6360E007F157
S3150802816008031846FEF7BEF93B697B6358E02D4BB8
S31508028170D3F8F03003F00203022B03D14FF4004385
S315080281807B634DE000237B634AE0264BD3F8F0304D
S3150802819003F00063B3F1006F03D14FF4FA437B6334
S315080281A03EE000237B633BE01E4BD3F8E83003F046
S315080281B04043FB621B4B1B6803F00203022B0CD1E4
S315080281C0FB6A002B09D1174B1B68DB0803F0030374
S315080281D0154A22FA03F37B631EE0124B1B6803F46B
S315080281E00073B3F5007F06D1FB6AB3F1804F02D163
S315080281F00E4B7B6310E00B4B1B6803F40033B3F59D
S31508028200003F06D1FB6AB3F1004F02D1084B7B63EC
S3150802821002E000237B6303E002E000237B6300BFE6
S3150802822000F015BE000C02440090D00300093D0080
S31508028230001BB7009E4BD3F8DC3003F4E0033B6324
S315080282403B6BB3F5A00F56D03B6BB3F5A00F00F20C
S315080282508B803B6BB3F5800F3ED03B6BB3F5800F3B
S3150802826000F282803B6BB3F5401F27D03B6BB3F518
S31508028270401F79D83B6BB3F5001F17D03B6BB3F59C
S31508028280001F71D83B6B002B04D03B6BB3F5801FE4
S3150802829004D069E0FBF77AFE786368E007F1140315
S315080282A01846FDF7B5FF7B697B6360E007F10803B3
S315080282B01846FEF717F93B697B6358E07C4BD3F8FF
S315080282C0F03003F00203022B03D14FF400437B6321
S315080282D04DE000237B634AE0754BD3F8F03003F098
S315080282E00063B3F1006F03D14FF4FA437B633EE0B8
S315080282F000237B633BE06E4BD3F8E83003F0404340
S31508028300FB626B4B1B6803F00203022B0CD1FB6A60
S31508028310002B09D1664B1B68DB0803F00303654A89
S3150802832022FA03F37B631EE0614B1B6803F40073B6
S31508028330B3F5007F06D1FB6AB3F1804F02D15E4BDB
S315080283407B6310E05A4B1B6803F40033B3F5003F16
S3150802835006D1FB6AB3F1004F02D1584B7B6302E0A8
S3150802836000237B6303E002E000237B6300BF00F087
S315080283706EBD4F4BD3F8DC3003F0E0633B633B6BD7
S31508028380B3F1A06F56D03B6BB3F1A06F00F28B80AE
S315080283903B6BB3F1806F3ED03B6BB3F1806F00F25B
S315080283A082803B6BB3F1407F27D03B6BB3F1407FB2
S315080283B079D83B6BB3F1007F17D03B6BB3F1007FE3
S315080283C071D83B6B002B04D03B6BB3F1807F04D092
S315080283D069E0FBF7DBFD786368E007F114031846EA
S315080283E0FDF716FF7B697B6360E007F10803184611
S315080283F0FEF778F83B697B6358E02D4BD3F8F030EB
S3150802840003F00203022B03D14FF400437B634DE0D2
S3150802841000237B634AE0264BD3F8F03003F000636F
S31508028420B3F1006F03D14FF4FA437B633EE00023B6
S315080284307B633BE01E4BD3F8E83003F04043FB6214
S315080284401B4B1B6803F00203022B0CD1FB6A002BA1
S3150802845009D1174B1B68DB0803F00303154A22FAF6
S3150802846003F37B631EE0124B1B6803F40073B3F538
S31508028470007F06D1FB6AB3F1804F02D10E4B7B63B4
S3150802848010E00B4B1B6803F40033B3F5003F06D12B
S31508028490FB6AB3F1004F02D1084B7B6302E000236B
S315080284A07B6303E002E000237B6300BF00F0CFBCDE
S315080284B0000C02440090D00300093D00001BB700DF
S315080284C09E4BD3F8DC3003F0E0433B633B6BB3F1DE
S315080284D0A04F56D03B6BB3F1A04F00F28B803B6B9B
S315080284E0B3F1804F3ED03B6BB3F1804F00F28280EE
S315080284F03B6BB3F1405F27D03B6BB3F1405F79D852
S315080285003B6BB3F1005F17D03B6BB3F1005F71D8D9
S315080285103B6B002B04D03B6BB3F1805F04D069E060
S31508028520FBF734FD786368E007F114031846FDF794
S315080285306FFE7B697B6360E007F108031846FDF767
S31508028540D1FF3B697B6358E07C4BD3F8F03003F0EC
S315080285500203022B03D14FF400437B634DE0002351
S315080285607B634AE0754BD3F8F03003F00063B3F14E
S31508028570006F03D14FF4FA437B633EE000237B632B
S315080285803BE06E4BD3F8E83003F04043FB626B4B9B
S315080285901B6803F00203022B0CD1FB6A002B09D1DC
S315080285A0664B1B68DB0803F00303654A22FA03F3EA
S315080285B07B631EE0614B1B6803F40073B3F5007F0F
S315080285C006D1FB6AB3F1804F02D15E4B7B6310E0A2
S315080285D05A4B1B6803F40033B3F5003F06D1FB6A16
S315080285E0B3F1004F02D1584B7B6302E000237B6351
S315080285F003E002E000237B6300BF00F028BC4F4B78
S31508028600D3F8E83003F440733B634C4B1B6803F41E
S315080286100033B3F5003F06D13B6B002B03D14A4B1F
S315080286207B6300F014BC3B6BB3F5807F08D107F17E
S3150802863020031846FDF782FC7B6A7B6300F007BCC1
S315080286403B6BB3F5007F07D107F114031846FDF714
S31508028650DFFDBB697B63FAE300237B63F7E3374BF2
S31508028660D3F8E03003F007033B633B6B042B61D876
S3150802867001A252F823F000BF8D8602089D860208E1
S31508028680AD860208BD860208C386020807F12003E2
S315080286901846FDF753FC7B6A7B634EE007F1140329
S315080286A01846FDF7B5FD7B697B6346E007F10803CB
S315080286B01846FDF717FFBB687B633EE0234B7B63D7
S315080286C03BE01E4BD3F8E83003F04043FB621B4BFA
S315080286D01B6803F00203022B0CD1FB6A002B09D19B
S315080286E0164B1B68DB0803F00303154A22FA03F349
S315080286F07B631EE0114B1B6803F40073B3F5007F1E
S3150802870006D1FB6AB3F1804F02D10E4B7B6310E0B0
S315080287100A4B1B6803F40033B3F5003F06D1FB6A24
S31508028720B3F1004F02D1084B7B6302E000237B635F
S3150802873003E002E000237B6300BF88E3000C0244E7
S315080287400090D00300093D00001BB7000080BB0063
S31508028750A94BD3F8E03003F038033B633B6B202B7D
S3150802876000F29A8001A252F823F000BFF1870208AC
S31508028770998802089988020899880208998802083D
S3150802878099880208998802089988020801880208C5
S31508028790998802089988020899880208998802081D
S315080287A09988020899880208998802081188020895
S315080287B099880208998802089988020899880208FD
S315080287C09988020899880208998802082188020865
S315080287D099880208998802089988020899880208DD
S315080287E0998802089988020899880208278802083F
S315080287F007F120031846FDF7A1FB7B6A7B634EE06F
S3150802880007F114031846FDF703FD7B697B6346E00F
S3150802881007F108031846FDF765FEBB687B633EE071
S31508028820764B7B633BE0744BD3F8E83003F0404366
S31508028830FB62714B1B6803F00203022B0CD1FB6A25
S31508028840002B09D16C4B1B68DB0803F003036C4A47
S3150802885022FA03F37B631EE0674B1B6803F400737B
S31508028860B3F5007F06D1FB6AB3F1804F02D1654B9F
S315080288707B6310E0604B1B6803F40033B3F5003FDB
S3150802888006D1FB6AB3F1004F02D15F4B7B6302E06C
S3150802889000237B6303E002E000237B6300BFD6E28A
S315080288A0554BD3F8E03003F4E0733B633B6BB3F507
S315080288B0807F31D03B6BB3F5807F66D83B6BC02B8C
S315080288C027D03B6BC02B60D83B6B802B19D03B6BF8
S315080288D0802B5AD83B6B002B03D03B6B402B08D01E
S315080288E053E007F120031846FDF728FB7B6A7B63F2
S315080288F04EE007F114031846FDF78AFC7B697B6391
S3150802890046E007F108031846FDF7ECFDBB687B63F2
S315080289103EE03A4B7B633BE0374BD3F8E83003F053
S315080289204043FB62344B1B6803F00203022B0CD153
S31508028930FB6A002B09D1304B1B68DB0803F00303E3
S315080289402F4A22FA03F37B631EE02B4B1B6803F4C0
S315080289500073B3F5007F06D1FB6AB3F1804F02D1EB
S31508028960284B7B6310E0244B1B6803F40033B3F5F2
S31508028970003F06D1FB6AB3F1004F02D1224B7B635B
S3150802898002E000237B6303E002E000237B6300BF6F
S315080289905DE2194BD3F8E03003F460633B633B6B4B
S315080289A0002B03D1FBF7DCFA786350E2124B1B6803
S315080289B003F00063B3F1006F0BD13B6BB3F5007F95
S315080289C007D107F114031846FDF722FCBB697B633E
S315080289D04FE0094B1B6803F00053B3F1005F15D152
S315080289E03B6BB3F5806F11D107F108031846FDF703
S315080289F079FDFB687B633CE0000C02440080BB0007
S31508028A000090D00300093D00001BB700944B1B6879
S31508028A1003F00203022B0DD13B6BB3F5C06F09D1EC
S31508028A208F4B1B68DB0803F003038E4A22FA03F313
S31508028A307B631EE08A4B1B6803F40073B3F5007F61
S31508028A4006D13B6BB3F5006F02D1874B7B6310E00F
S31508028A50834B1B6803F40033B3F5003F06D13B6B27
S31508028A60B3F5206F02D1814B7B6302E000237B635F
S31508028A70EDE1ECE17A4BD3F8E03003F4E0433B63F3
S31508028A803B6B002B03D1FBF781FA7863DFE1744B6A
S31508028A901B6803F00063B3F1006F0BD13B6BB3F5B0
S31508028AA0805F07D107F114031846FDF7B1FBBB69CE
S31508028AB07B6345E06A4B1B6803F00053B3F1005F22
S31508028AC00BD13B6BB3F5005F07D107F108031846D4
S31508028AD0FDF708FDFB687B6332E0614B1B6803F018
S31508028AE00203022B0DD13B6BB3F5405F09D15C4BF8
S31508028AF01B68DB0803F003035A4A22FA03F37B6373
S31508028B001EE0574B1B6803F40073B3F5007F06D1CA
S31508028B103B6BB3F5804F02D1534B7B6310E0504B4E
S31508028B201B6803F40033B3F5003F06D13B6BB3F57C
S31508028B30A04F02D14D4B7B6302E000237B6386E1A3
S31508028B4085E1474BD3F8E03003F460333B633B6B74
S31508028B50002B03D1FBF704FA786378E1404B1B68D4
S31508028B6003F00063B3F1006F0BD13B6BB3F5004F13
S31508028B7007D107F114031846FDF74AFBBB697B6365
S31508028B8045E0374B1B6803F00053B3F1005F0BD186
S31508028B903B6BB3F5803F07D107F108031846FDF78B
S31508028BA0A1FCFB687B6332E02D4B1B6803F00203D2
S31508028BB0022B0DD13B6BB3F5C03F09D1284B1B687D
S31508028BC0DB0803F00303274A22FA03F37B631EE05A
S31508028BD0234B1B6803F40073B3F5007F06D13B6B86
S31508028BE0B3F5003F02D1204B7B6310E01C4B1B6898
S31508028BF003F40033B3F5003F06D13B6BB3F5203FD0
S31508028C0002D11A4B7B6302E000237B631FE11EE15C
S31508028C10134BD3F8E43003F003033B633B6B032B9C
S31508028C205FD801A252F823F0398C0208418C020857
S31508028C30518C0208718C0208FBF760F9786353E0DD
S31508028C4007F120031846FDF779F97B6A7B634BE047
S31508028C5007F114031846FDF7DBFAFB697B6343E069
S31508028C60000C02440090D00300093D00001BB70027
S31508028C70794BD3F8E83003F04043FB62764B1B6826
S31508028C8003F00203022B0CD1FB6A002B09D1724BAB
S31508028C901B68DB0803F00303704A22FA03F37B63BB
S31508028CA01EE06D4B1B6803F40073B3F5007F06D113
S31508028CB0FB6AB3F1804F02D1694B7B6310E0664BC6
S31508028CC01B6803F40033B3F5003F06D1FB6AB3F120
S31508028CD0004F02D1634B7B6302E000237B6303E010
S31508028CE002E000237B6300BFB1E05B4BD3F8E830B8
S31508028CF003F0C0033B63584BD3F8F03003F002038A
S31508028D00022B06D13B6B002B03D14FF400437B6346
S31508028D101FE0514BD3F8F03003F00063B3F1006F54
S31508028D2006D13B6B402B03D14FF4FA437B6310E029
S31508028D30494B1B6803F40073B3F5007F06D13B6BFE
S31508028D40802B03D148F212037B6302E000237B6384
S31508028D507DE07CE0404BD3F8E83003F030033B6318
S31508028D603D4B1B6803F40053B3F5005F05D13B6B1B
S31508028D70002B02D13C4B7B6331E0374B1B6803F077
S31508028D800073B3F1007F0AD13B6B102B07D107F1B1
S31508028D9020031846FDF7D2F87B6A7B631FE02E4B49
S31508028DA0D3F8F03003F00203022B06D13B6B202BDB
S31508028DB003D14FF400437B6311E0274BD3F8F0301D
S31508028DC003F00063B3F1006F06D13B6B302B03D17E
S31508028DD04FF4FA437B6302E000237B6337E036E015
S31508028DE01D4BD3F8E43003F030033B633B6B102B87
S31508028DF007D107F120031846FDF7A0F87B6A7B63C3
S31508028E0025E0154B1B6803F00053B3F1005F0AD146
S31508028E103B6B202B07D107F108031846FDF762FBC7
S31508028E20FB687B630FE00C4B1B6803F40053B3F536
S31508028E30005F05D13B6B302B02D10B4B7B6302E003
S31508028E4000237B6303E002E000237B6300BF7B6BA6
S31508028E5018463C37BD4690BD000C02440090D0032C
S31508028E6000093D00001BB700006CDC0280B584B027
S31508028E7000AF7860484B1B68474A23F0806313604B
S31508028E80F8F732FAF86008E0F8F72EFA0246FB68B5
S31508028E90D31A022B01D903237AE03F4B1B6803F04E
S31508028EA00063002BF0D13C4BDB6A23F47C5323F09E
S31508028EB003037A6811687A68526812020A433649C5
S31508028EC01343CB627B689B68013BC3F308027B684A
S31508028ED0DB68013B5B029BB21A437B681B69013B59
S31508028EE01B0403F4FE031A437B685B69013B1B06FA
S31508028EF003F0FE4328491343CB63274BDB6A23F06F
S31508028F000C027B689B6924491343CB62224BDB6ABA
S31508028F1023F020027B68DB691F491343CB621E4B91
S31508028F20DA6A7B685B6A1C491343CB621A4BDB6AB3
S31508028F30194A23F01003D362174B1B6C23F47F43A1
S31508028F4023F0F8037A68126AD200134913430B64B2
S31508028F50114BDB6A104A43F01003D3620E4B1B68AF
S31508028F600D4A43F080631360F8F7BEF9F86008E02B
S31508028F70F8F7BAF90246FB68D31A022B01D903237A
S31508028F8006E0054B1B6803F00063002BF0D00023B4
S31508028F9018461037BD4680BD000C024480B584B021
S31508028FA000AF7860484B1B68474A23F0805313602A
S31508028FB0F8F79AF9F86008E0F8F796F90246FB68B6
S31508028FC0D31A022B01D903237AE03F4B1B6803F01D
S31508028FD00053002BF0D13C4B1B6B23F47C5323F03C
S31508028FE003037A6811687A68526812020A43364994
S31508028FF013430B637B689B68013BC3F308027B68D8
S31508029000DB68013B5B029BB21A437B681B69013B27
S315080290101B0403F4FE031A437B685B69013B1B06C8
S3150802902003F0FE43284913434B64274B1B6B23F07B
S315080290300C027B689B69244913430B63224B1B6B07
S3150802904023F020027B68DB691F4913430B631E4B1F
S315080290501A6B7B685B6A1C4913430B631A4B1B6BBF
S31508029060194A23F010031363174B9B6C23F47F43AF
S3150802907023F0F8037A68126AD200134913438B6401
S31508029080114B1B6B104A43F0100313630E4B1B68FC
S315080290900D4A43F080531360F8F726F9F86008E0A2
S315080290A0F8F722F90246FB68D31A022B01D90323E1
S315080290B006E0054B1B6803F00053002BF0D0002393
S315080290C018461037BD4680BD000C024480B582B0F2
S315080290D000AF78607B68002B01D1012349E07B68E9
S315080290E093F83D30DBB2002B06D17B68002283F869
S315080290F03C20786815F028FF7B68022283F83D2019
S315080291007B681A687B6804331946104600F0F0FE3D
S315080291107B68012283F848207B68012283F83E2077
S315080291207B68012283F83F207B68012283F840206E
S315080291307B68012283F841207B68012283F842205A
S315080291407B68012283F843207B68012283F8442046
S315080291507B68012283F845207B68012283F8462032
S315080291607B68012283F847207B68012283F83D2029
S31508029170002318460837BD4680BD000080B485B076
S3150802918000AF78607B6893F83D30DBB2012B01D0E3
S31508029190012374E07B68022283F83D207B681B6802
S315080291A03A4A93424AD07B681B68394A934245D069
S315080291B07B681B68B3F1804F40D07B681B68B3F1AC
S315080291C0A04F3BD07B681B68324A934236D07B68F5
S315080291D01B68314A934231D07B681B682F4A9342F7
S315080291E02CD07B681B682E4A934227D07B681B6863
S315080291F02C4A934222D07B681B682B4A93421DD085
S315080292007B681B68294A934218D07B681B68284AE0
S31508029210934213D07B681B68264A93420ED07B681A
S315080292201B68254A934209D07B681B68234A9342E6
S3150802923004D07B681B68224A934215D17B681B6857
S315080292409A68204B1340FB60FB68062B15D0FB6817
S31508029250B3F5803F11D07B681B681A687B681B6868
S3150802926042F001021A6008E07B681B681A687B688C
S315080292701B6842F001021A6000E000BF002318468C
S315080292801437BD465DF8047B704700BF002C0140C9
S31508029290002C015000040040000400500008004061
S315080292A000080050000C0040000C00500034014039
S315080292B000340150001800400018005000400140D8
S315080292C0004001500700010080B485B000AF786005
S315080292D07B6893F83D30DBB2012B01D001237CE099
S315080292E07B68022283F83D207B681B68DA687B6804
S315080292F01B6842F00102DA607B681B683A4A9342AD
S315080293004AD07B681B68394A934245D07B681B68FA
S31508029310B3F1804F40D07B681B68B3F1A04F3BD0B6
S315080293207B681B68324A934236D07B681B68314A8F
S31508029330934231D07B681B682F4A93422CD07B68B4
S315080293401B682E4A934227D07B681B682C4A934295
S3150802935022D07B681B682B4A93421DD07B681B6808
S31508029360294A934218D07B681B68284A934213D02D
S315080293707B681B68264A93420ED07B681B68254A7F
S31508029380934209D07B681B68234A934204D07B68C0
S315080293901B68224A934215D17B681B689A68204B40
S315080293A01340FB60FB68062B15D0FB68B3F5803FBC
S315080293B011D07B681B681A687B681B6842F0010239
S315080293C01A6008E07B681B681A687B681B6842F0AB
S315080293D001021A6000E000BF002318461437BD4692
S315080293E05DF8047B704700BF002C0140002C015039
S315080293F00004004000040050000800400008005025
S31508029400000C0040000C00500034014000340150AA
S31508029410001800400018005000400140004001506A
S315080294200700010080B582B000AF78607B68002B28
S3150802943001D1012349E07B6893F83D30DBB2002B6A
S3150802944006D17B68002283F83C20786800F041F850
S315080294507B68022283F83D207B681A687B6804339E
S315080294601946104600F044FD7B68012283F848201D
S315080294707B68012283F83E207B68012283F83F201D
S315080294807B68012283F840207B68012283F8412009
S315080294907B68012283F842207B68012283F84320F5
S315080294A07B68012283F844207B68012283F84520E1
S315080294B07B68012283F846207B68012283F84720CD
S315080294C07B68012283F83D20002318460837BD46EB
S315080294D080BD80B483B000AF786000BF0C37BD464C
S315080294E05DF8047B7047000080B584B000AF7860F1
S315080294F039603B68002B09D17B6893F83E30DBB2B2
S31508029500012B14BF01230023DBB23CE03B68042B8A
S3150802951009D17B6893F83F30DBB2012B14BF0123D4
S315080295200023DBB22FE03B68082B09D17B6893F84E
S315080295304030DBB2012B14BF01230023DBB222E049
S315080295403B680C2B09D17B6893F84130DBB2012BBF
S3150802955014BF01230023DBB215E03B68102B09D1A7
S315080295607B6893F84230DBB2012B14BF0123002338
S31508029570DBB208E07B6893F84330DBB2012B14BFF9
S3150802958001230023DBB2002B01D00123E2E03B6872
S31508029590002B04D17B68022283F83E2023E03B6835
S315080295A0042B04D17B68022283F83F201BE03B6828
S315080295B0082B04D17B68022283F8402013E03B681B
S315080295C00C2B04D17B68022283F841200BE03B680E
S315080295D0102B04D17B68022283F8422003E07B68C1
S315080295E0022283F843207B681B68012239681846E1
S315080295F001F00EFA7B681B68584A93422CD07B68A6
S315080296001B68574A934227D07B681B68554A934280
S3150802961022D07B681B68544A93421DD07B681B681C
S31508029620524A934218D07B681B68514A934213D018
S315080296307B681B684F4A93420ED07B681B684E4A6A
S31508029640934209D07B681B684C4A934204D07B68D4
S315080296501B684B4A934201D1012300E00023002BE9
S3150802966007D07B681B685A6C7B681B6842F4004209
S315080296705A647B681B68394A93424AD07B681B68DE
S31508029680374A934245D07B681B68B3F1804F40D076
S315080296907B681B68B3F1A04F3BD07B681B68394ACD
S315080296A0934236D07B681B68374A934231D07B682F
S315080296B01B68364A93422CD07B681B68344A93420D
S315080296C027D07B681B68334A934222D07B681B6883
S315080296D0314A93421DD07B681B68224A934218D0AE
S315080296E07B681B68204A934213D07B681B682B4A07
S315080296F093420ED07B681B68294A934209D07B683D
S315080297001B681A4A934204D07B681B68184A93421C
S3150802971015D17B681B689A68224B1340FB60FB686D
S31508029720062B15D0FB68B3F5803F11D07B681B6802
S315080297301A687B681B6842F001021A6008E07B68B7
S315080297401B681A687B681B6842F001021A6000E00F
S3150802975000BF002318461037BD4680BD002C0140C5
S31508029760002C0150003401400034015000400140F1
S3150802977000400150004401400044015000480140A5
S315080297800048015000040040000400500008004050
S3150802979000080050000C0040000C00500018004061
S315080297A0001800500700010080B584B000AF786049
S315080297B07B681B68DB68FB607B681B681B69BB6090
S315080297C0BB6803F00203002B20D0FB6803F00203F8
S315080297D0002B1BD07B681B686FF002021A617B683C
S315080297E001221A777B681B689B6903F00303002B27
S315080297F003D0786800F05EFB05E0786800F050FB5D
S31508029800786800F061FB7B6800221A77BB6803F070
S315080298100403002B20D0FB6803F00403002B1BD0A3
S315080298207B681B686FF004021A617B6802221A774A
S315080298307B681B689B6903F44073002B03D0786826
S3150802984000F038FB05E0786800F02AFB786800F03B
S315080298503BFB7B6800221A77BB6803F00803002BE0
S3150802986020D0FB6803F00803002B1BD07B681B681B
S315080298706FF008021A617B6804221A777B681B68F4
S31508029880DB6903F00303002B03D0786800F012FBB0
S3150802989005E0786800F004FB786800F015FB7B6841
S315080298A000221A77BB6803F01003002B20D0FB684E
S315080298B003F01003002B1BD07B681B686FF01002A5
S315080298C01A617B6808221A777B681B68DB6903F4CE
S315080298D04073002B03D0786800F0ECFA05E078684C
S315080298E000F0DEFA786800F0EFFA7B6800221A7751
S315080298F0BB6803F00103002B0CD0FB6803F00103DD
S31508029900002B07D07B681B686FF001021A61786822
S3150802991012F000F9BB6803F08003002B0CD0FB6839
S3150802992003F08003002B07D07B681B686FF0800268
S315080299301A61786801F06CF9BB6803F48073002B2E
S315080299400CD0FB6803F08003002B07D07B681B68EA
S315080299506FF480721A61786801F064F9BB6803F0E3
S315080299604003002B0CD0FB6803F04003002B07D002
S315080299707B681B686FF040021A61786800F0AEFADD
S31508029980BB6803F02003002B0CD0FB6803F020030E
S31508029990002B07D07B681B686FF020021A61786873
S315080299A001F02CF9BB6803F48013002B0CD0FB687A
S315080299B003F48013002B07D07B681B686FF48012B0
S315080299C01A61786801F038F9BB6803F40013002BB2
S315080299D00CD0FB6803F40013002B07D07B681B68C6
S315080299E06FF400121A61786801F030F9BB6803F463
S315080299F08003002B0CD0FB6803F48003002B07D0EE
S31508029A007B681B686FF480021A61786801F028F98E
S31508029A10BB6803F40003002B0CD0FB6803F40003B5
S31508029A20002B07D07B681B686FF400021A617868FE
S31508029A3001F020F900BF1037BD4680BD80B586B05B
S31508029A4000AFF860B9607A600023FB75FB6893F88B
S31508029A503C30012B01D10223FFE0FB68012283F887
S31508029A603C207B68142B00F2F08001A252F823F006
S31508029A70C59A02084B9C02084B9C02084B9C02089A
S31508029A80059B02084B9C02084B9C02084B9C020849
S31508029A90479B02084B9C02084B9C02084B9C0208F7
S31508029AA0879B02084B9C02084B9C02084B9C0208A7
S31508029AB0C99B02084B9C02084B9C02084B9C020855
S31508029AC0099C0208FB681B68B968184600F02EFB59
S31508029AD0FB681B689A69FB681B6842F008029A6170
S31508029AE0FB681B689A69FB681B6822F004029A6184
S31508029AF0FB681B689969BB681A69FB681B680A4395
S31508029B009A61A5E0FB681B68B968184600F0D0FBA5
S31508029B10FB681B689A69FB681B6842F400629A61D3
S31508029B20FB681B689A69FB681B6822F480629A6163
S31508029B30FB681B689969BB681B691A02FB681B6884
S31508029B400A439A6184E0FB681B68B968184600F004
S31508029B505FFCFB681B68DA69FB681B6842F008024F
S31508029B60DA61FB681B68DA69FB681B6822F0040283
S31508029B70DA61FB681B68D969BB681A69FB681B68E6
S31508029B800A43DA6164E0FB681B68B968184600F0A4
S31508029B90EDFCFB681B68DA69FB681B6842F4006225
S31508029BA0DA61FB681B68DA69FB681B6822F4806263
S31508029BB0DA61FB681B68D969BB681B691A02FB680C
S31508029BC01B680A43DA6143E0FB681B68B9681846F2
S31508029BD000F07CFDFB681B681A6DFB681B6842F087
S31508029BE008021A65FB681B681A6DFB681B6822F077
S31508029BF004021A65FB681B68196DBB681A69FB685B
S31508029C001B680A431A6523E0FB681B68B96818468D
S31508029C1000F0DEFDFB681B681A6DFB681B6842F4E0
S31508029C2000621A65FB681B681A6DFB681B6822F4DA
S31508029C3080621A65FB681B68196DBB681B691A0284
S31508029C40FB681B680A431A6502E00123FB7500BF1D
S31508029C50FB68002283F83C20FB7D18461837BD4670
S31508029C6080BD00BF80B584B000AF7860396000233C
S31508029C70FB737B6893F83C30012B01D10223FEE08B
S31508029C807B68012283F83C207B68022283F83D2008
S31508029C907B681B689B68BB60BB6823F4441323F08C
S31508029CA07703BB60BB6823F47F43BB607B681B6892
S31508029CB0BA689A603B681B68B3F5001F00F0C98052
S31508029CC0B3F5001F00F2CE806F4A934200F0C180BE
S31508029CD06D4A934200F2C6806C4A934200F0B980FC
S31508029CE06A4A934200F2BE80694A934200F0B18002
S31508029CF0674A934200F2B680664A934200F0A98008
S31508029D00644A934200F2AE80634A934200F0A1800D
S31508029D10614A934200F2A680604A934200F0998013
S31508029D205E4A934200F29E80B3F1101F00F09180C2
S31508029D30B3F1101F00F29680B3F5801F00F08980F8
S31508029D40B3F5801F00F28E80B3F5005F3ED0B3F5FF
S31508029D50005F00F28780B3F5805F00F08680B3F576
S31508029D60805F7FD8702B1AD0702B7BD8602B50D08F
S31508029D70602B77D8502B3CD0502B73D8402B58D019
S31508029D80402B6FD8302B64D0302B6BD8202B60D069
S31508029D90202B67D8002B5CD0102B5AD062E07B6848
S31508029DA018683B6899683B685A683B68DB6800F044
S31508029DB00FFE7B681B689B68BB60BB6843F0770332
S31508029DC0BB607B681B68BA689A604FE07B68186854
S31508029DD03B6899683B685A683B68DB6800F0F8FD9F
S31508029DE07B681B689A687B681B6842F480429A60A3
S31508029DF03CE07B6818683B6859683B68DB681A462A
S31508029E0000F06AFD7B681B685021184600F0C3FD06
S31508029E102CE07B6818683B6859683B68DB681A4619
S31508029E2000F089FD7B681B686021184600F0B3FDC7
S31508029E301CE07B6818683B6859683B68DB681A4609
S31508029E4000F04AFD7B681B684021184600F0A3FD16
S31508029E500CE07B681A683B681B681946104600F0D6
S31508029E609AFD03E00123FB7300E000BF7B68012231
S31508029E7083F83D207B68002283F83C20FB7B18464A
S31508029E801037BD4680BD00BF70001000600010008C
S31508029E905000100040001000300010002000100092
S31508029EA080B483B000AF786000BF0C37BD465DF85A
S31508029EB0047B704780B483B000AF786000BF0C376C
S31508029EC0BD465DF8047B704780B483B000AF786006
S31508029ED000BF0C37BD465DF8047B704780B483B07B
S31508029EE000AF786000BF0C37BD465DF8047B70474B
S31508029EF080B485B000AF786039607B681B68FB6008
S31508029F007B68744A93422BD07B68734A934227D064
S31508029F107B68B3F1804F23D07B68B3F1A04F1FD083
S31508029F207B686E4A93421BD07B686D4A934217D070
S31508029F307B686C4A934213D07B686B4A93420FD074
S31508029F407B686A4A93420BD07B68694A934207D078
S31508029F507B68684A934203D07B68674A934208D172
S31508029F60FB6823F07003FB603B685B68FA6813437F
S31508029F70FB607B68574A93425BD07B68564A93429A
S31508029F8057D07B68B3F1804F53D07B68B3F1A04FAB
S31508029F904FD07B68514A93424BD07B68504A9342D2
S31508029FA047D07B684F4A934243D07B684E4A9342D6
S31508029FB03FD07B684D4A93423BD07B684C4A9342DA
S31508029FC037D07B684B4A934233D07B684A4A9342DE
S31508029FD02FD07B68494A93422BD07B68484A9342E2
S31508029FE027D07B68474A934223D07B68464A9342E6
S31508029FF01FD07B68454A93421BD07B68444A9342EA
S3150802A00017D07B68434A934213D07B68424A9342ED
S3150802A0100FD07B68414A93420BD07B68404A9342F1
S3150802A02007D07B683F4A934203D07B683E4A9342F5
S3150802A03008D1FB6823F44073FB603B68DB68FA6867
S3150802A0401343FB60FB6823F080023B685B6913439A
S3150802A050FB607B68FA681A603B689A687B68DA6212
S3150802A0603B681A687B689A627B681A4A934223D0CD
S3150802A0707B68194A93421FD07B681E4A93421BD0BB
S3150802A0807B681D4A934217D07B68224A934213D0B3
S3150802A0907B68214A93420FD07B68204A93420BD0B1
S3150802A0A07B681F4A934207D07B681E4A934203D0B5
S3150802A0B07B681D4A934203D13B681A697B681A6317
S3150802A0C07B6801225A6100BF1437BD465DF8047BDE
S3150802A0D0704700BF002C0140002C015000040040CC
S3150802A0E0000400500008004000080050000C004020
S3150802A0F0000C0050003401400034015000180040A2
S3150802A10000180050001C0040001C005000200040AF
S3150802A1100020005000400140004001500044014028
S3150802A12000440150004801400048015080B487B0FD
S3150802A13000AF786039607B681B6A7B617B681B6A43
S3150802A14023F001027B681A627B685B683B617B6865
S3150802A1509B69FB60FB6823F4803323F07003FB6082
S3150802A160FB6823F00303FB603B681B68FA6813432A
S3150802A170FB607B6923F002037B613B689B687A6913
S3150802A18013437B617B68404A934223D07B683F4AEC
S3150802A19093421FD07B683E4A93421BD07B683D4A56
S3150802A1A0934217D07B683C4A934213D07B683B4A5A
S3150802A1B093420FD07B683A4A93420BD07B68394A5E
S3150802A1C0934207D07B68384A934203D07B68374A62
S3150802A1D093420CD17B6923F008037B613B68DB68F9
S3150802A1E07A6913437B617B6923F004037B617B688D
S3150802A1F0254A934223D07B68244A93421FD07B6820
S3150802A200234A93421BD07B68224A934217D07B6823
S3150802A210214A934213D07B68204A93420FD07B6827
S3150802A2201F4A93420BD07B681E4A934207D07B682B
S3150802A2301D4A934203D07B681C4A934211D13B695B
S3150802A24023F480733B613B6923F400733B613B68EB
S3150802A2505B693A6913433B613B689B693A691343F5
S3150802A2603B617B683A695A607B68FA689A613B681F
S3150802A2705A687B685A637B687A691A6200BF1C3718
S3150802A280BD465DF8047B7047002C0140002C015046
S3150802A29000340140003401500040014000400150A2
S3150802A2A00044014000440150004801400048015062
S3150802A2B080B487B000AF786039607B681B6A7B61BF
S3150802A2C07B681B6A23F010027B681A627B685B68EC
S3150802A2D03B617B689B69FB60FB6823F0807323F410
S3150802A2E0E043FB60FB6823F44073FB603B681B6832
S3150802A2F01B02FA681343FB607B6923F020037B6128
S3150802A3003B689B681B017A6913437B617B68364A03
S3150802A31093420BD07B68354A934207D07B68344A0E
S3150802A320934203D07B68334A93420DD17B6923F06B
S3150802A33080037B613B68DB681B017A6913437B6197
S3150802A3407B6923F040037B617B68274A934223D0CB
S3150802A3507B68264A93421FD07B68254A93421BD0C4
S3150802A3607B68244A934217D07B68234A934213D0C8
S3150802A3707B68224A93420FD07B68214A93420BD0CC
S3150802A3807B68204A934207D07B681F4A934203D0D0
S3150802A3907B681E4A934213D13B6923F480633B616F
S3150802A3A03B6923F400633B613B685B699B003A693E
S3150802A3B013433B613B689B699B003A6913433B61C4
S3150802A3C07B683A695A607B68FA689A613B685A6898
S3150802A3D07B689A637B687A691A6200BF1C37BD4636
S3150802A3E05DF8047B704700BF002C0140002C015029
S3150802A3F00034014000340150004001400040015041
S3150802A4000044014000440150004801400048015000
S3150802A41080B487B000AF786039607B681B6A7B615D
S3150802A4207B681B6A23F480727B681A627B685B68A6
S3150802A4303B617B68DB69FB60FB6823F4803323F0AE
S3150802A4407003FB60FB6823F00303FB603B681B6831
S3150802A450FA681343FB607B6923F400737B613B68EC
S3150802A4609B681B027A6913437B617B68354A934270
S3150802A4700BD07B68344A934207D07B68334A9342AF
S3150802A48003D07B68324A93420DD17B6923F4006379
S3150802A4907B613B68DB681B027A6913437B617B69D4
S3150802A4A023F480637B617B68264A934223D07B68C8
S3150802A4B0254A93421FD07B68244A93421BD07B6865
S3150802A4C0234A934217D07B68224A934213D07B6869
S3150802A4D0214A93420FD07B68204A93420BD07B686D
S3150802A4E01F4A934207D07B681E4A934203D07B6871
S3150802A4F01D4A934213D13B6923F480533B613B695E
S3150802A50023F400533B613B685B691B013A691343B9
S3150802A5103B613B689B691B013A6913433B617B6854
S3150802A5203A695A607B68FA68DA613B685A687B68F6
S3150802A530DA637B687A691A6200BF1C37BD465DF822
S3150802A540047B7047002C0140002C01500034014066
S3150802A55000340150004001400040015000440140CF
S3150802A56000440150004801400048015080B487B0B9
S3150802A57000AF786039607B681B6A7B617B681B6AFF
S3150802A58023F480527B681A627B685B683B617B684E
S3150802A590DB69FB60FB6823F0807323F4E043FB600E
S3150802A5A0FB6823F44073FB603B681B681B02FA686E
S3150802A5B01343FB607B6923F400537B613B689B680A
S3150802A5C01B037A6913437B617B68364A93420BD035
S3150802A5D07B68354A934207D07B68344A934203D054
S3150802A5E07B68334A93420DD17B6923F400437B612E
S3150802A5F03B68DB681B037A6913437B617B6923F437
S3150802A60080437B617B68274A934223D07B68264A2C
S3150802A61093421FD07B68254A93421BD07B68244A03
S3150802A620934217D07B68234A934213D07B68224A07
S3150802A63093420FD07B68214A93420BD07B68204A0B
S3150802A640934207D07B681F4A934203D07B681E4A0F
S3150802A650934213D13B6923F480433B613B6923F45C
S3150802A66000433B613B685B699B013A6913433B6163
S3150802A6703B689B699B013A6913433B617B683A696C
S3150802A6805A607B68FA68DA613B685A687B681A64BA
S3150802A6907B687A691A6200BF1C37BD465DF8047B7F
S3150802A6A0704700BF002C0140002C015000340140C5
S3150802A6B0003401500040014000400150004401406E
S3150802A6C000440150004801400048015080B487B058
S3150802A6D000AF786039607B681B6A3B617B681B6ADE
S3150802A6E023F480327B681A627B685B687B617B68CD
S3150802A6F01B6DFB60FB6823F4803323F07003FB6059
S3150802A7003B681B68FA681343FB603B6923F4003312
S3150802A7103B613B689B681B043A6913433B617B6850
S3150802A720214A934223D07B68204A93421FD07B68F2
S3150802A7301F4A93421BD07B681E4A934217D07B68F6
S3150802A7401D4A934213D07B681C4A93420FD07B68FA
S3150802A7501B4A93420BD07B681A4A934207D07B68FE
S3150802A760194A934203D07B68184A934209D17B69F6
S3150802A77023F480337B613B685B691B027A69134366
S3150802A7807B617B687A695A607B68FA681A653B68F6
S3150802A7905A687B689A647B683A691A6200BF1C37F2
S3150802A7A0BD465DF8047B7047002C0140002C015021
S3150802A7B0003401400034015000400140004001507D
S3150802A7C0004401400044015000480140004801503D
S3150802A7D080B487B000AF786039607B681B6A3B61DA
S3150802A7E07B681B6A23F480127B681A627B685B6843
S3150802A7F07B617B681B6DFB60FB6823F0807323F427
S3150802A800E043FB603B681B681B02FA681343FB6064
S3150802A8103B6923F400133B613B689B681B053A6955
S3150802A82013433B617B68224A934223D07B68214AC1
S3150802A83093421FD07B68204A93421BD07B681F4AEB
S3150802A840934217D07B681E4A934213D07B681D4AEF
S3150802A85093420FD07B681C4A93420BD07B681B4AF3
S3150802A860934207D07B681A4A934203D07B68194AF7
S3150802A870934209D17B6923F480237B613B685B6938
S3150802A8809B027A6913437B617B687A695A607B68A3
S3150802A890FA681A653B685A687B68DA647B683A69BB
S3150802A8A01A6200BF1C37BD465DF8047B704700BFBD
S3150802A8B0002C0140002C01500034014000340150A4
S3150802A8C0004001400040015000440140004401504C
S3150802A8D0004801400048015080B487B000AFF860D4
S3150802A8E0B9607A60FB681B6A7B61FB681B6A23F0A6
S3150802A8F00102FB681A62FB689B693B613B6923F0AC
S3150802A900F0033B617B681B013A6913433B617B6930
S3150802A91023F00A037B617A69BB6813437B61FB6890
S3150802A9203A699A61FB687A691A6200BF1C37BD46A2
S3150802A9305DF8047B704780B487B000AFF860B960F1
S3150802A9407A60FB681B6A7B61FB681B6A23F010024C
S3150802A950FB681A62FB689B693B613B6923F4704397
S3150802A9603B617B681B033A6913433B617B6923F0AE
S3150802A970A0037B61BB681B017A6913437B61FB6891
S3150802A9803A699A61FB687A691A6200BF1C37BD4642
S3150802A9905DF8047B704780B485B000AF7860396093
S3150802A9A07B689B68FB60FB6823F4401323F0700303
S3150802A9B0FB603A68FB68134343F00703FB607B6856
S3150802A9C0FA689A6000BF1437BD465DF8047B704783
S3150802A9D080B487B000AFF860B9607A603B60FB6804
S3150802A9E09B687B617B6923F47F437B613B681A0220
S3150802A9F07B681A43BB6813437A6913437B61FB6816
S3150802AA007A699A6000BF1C37BD465DF8047B7047B9
S3150802AA1080B487B000AFF860B9607A60BB6803F0AB
S3150802AA201F03012202FA03F37B61FB681A6A7B6938
S3150802AA30DB431A40FB681A62FB681A6ABB6803F0B2
S3150802AA401F03796801FA03F31A43FB681A6200BF07
S3150802AA501C37BD465DF8047B7047000080B485B09C
S3150802AA6000AF786039607B6893F83C30012B01D1DE
S3150802AA700223A1E07B68012283F83C207B6802223C
S3150802AA8083F83D207B681B685B68FB607B681B68F4
S3150802AA909B68BB607B681B684A4A93420ED07B68F8
S3150802AAA01B68494A934209D07B681B68474A934206
S3150802AAB004D07B681B68464A934208D1FB6823F494
S3150802AAC07003FB603B685B68FA681343FB60FB68CC
S3150802AAD023F0007323F07003FB603B681B68FA6877
S3150802AAE01343FB607B681B68FA685A607B681B68BD
S3150802AAF0344A93424AD07B681B68334A934245D00C
S3150802AB007B681B68B3F1804F40D07B681B68B3F142
S3150802AB10A04F3BD07B681B682E4A934236D07B688F
S3150802AB201B682D4A934231D07B681B682B4A934295
S3150802AB302CD07B681B682A4A934227D07B681B68FD
S3150802AB40284A934222D07B681B68274A93421DD023
S3150802AB507B681B681D4A934218D07B681B681C4A8F
S3150802AB60934213D07B681B68204A93420ED07B68B7
S3150802AB701B681F4A934209D07B681B681D4A934289
S3150802AB8004D07B681B681C4A93420CD1BB6823F02D
S3150802AB908003BB603B689B68BA681343BB607B68EB
S3150802ABA01B68BA689A607B68012283F83D207B6835
S3150802ABB0002283F83C20002318461437BD465DF868
S3150802ABC0047B7047002C0140002C015000340140E0
S3150802ABD00034015000040040000400500008004000
S3150802ABE000080050000C0040000C005000180040FD
S3150802ABF000180050004001400040015080B483B064
S3150802AC0000AF786000BF0C37BD465DF8047B70471D
S3150802AC1080B483B000AF786000BF0C37BD465DF8DC
S3150802AC20047B704780B483B000AF786000BF0C37EE
S3150802AC30BD465DF8047B704780B483B000AF786088
S3150802AC4000BF0C37BD465DF8047B704780B483B0FD
S3150802AC5000AF786000BF0C37BD465DF8047B7047CD
S3150802AC6080B483B000AF786000BF0C37BD465DF88C
S3150802AC70047B704780B483B000AF786000BF0C379E
S3150802AC80BD465DF8047B704780B582B000AF786038
S3150802AC907B68002B01D1012342E07B68D3F8883018
S3150802ACA0002B06D17B68002283F88420786814F08A
S3150802ACB089FA7B682422C3F888207B681B681A688D
S3150802ACC07B681B6822F001021A607B689B6A002B6C
S3150802ACD002D0786800F020FF786800F02FFD03465E
S3150802ACE0012B01D101231BE07B681B685A687B682C
S3150802ACF01B6822F490425A607B681B689A687B68D4
S3150802AD001B6822F02A029A607B681B681A687B68AD
S3150802AD101B6842F001021A60786800F09FFF03463A
S3150802AD2018460837BD4680BD80B582B000AF786048
S3150802AD307B68002B01D1012331E07B682422C3F80A
S3150802AD4088207B681B681A687B681B6822F00102E8
S3150802AD501A607B681B6800221A607B681B680022DF
S3150802AD605A607B681B6800229A60786814F0C0FAF9
S3150802AD707B680022C3F890207B680022C3F88820EB
S3150802AD807B680022C3F88C207B680022DA667B681F
S3150802AD9000221A677B68002283F88420002318465B
S3150802ADA00837BD4680BD80B58AB002AFF860B96083
S3150802ADB03B601346FB80FB68D3F88830202B40F0B3
S3150802ADC08B80BB68002B02D0FB88002B01D10123A4
S3150802ADD083E0FB681B689B6803F08003802B07D11E
S3150802ADE0FB681B689A68FB681B6822F080029A60F7
S3150802ADF0FB680022C3F89020FB682122C3F888204A
S3150802AE00F6F772FA7861FB68FA88A3F85420FB68A9
S3150802AE10FA88A3F85620FB689B68B3F5805F08D1C9
S3150802AE20FB681B69002B04D10023FB61BB68BB616D
S3150802AE3003E0BB68FB610023BB6130E03B6800931B
S3150802AE407B6900228021F86800F0B2FF0346002BD6
S3150802AE5005D0FB682022C3F8882003233DE0FB695E
S3150802AE60002B0BD1BB691B881A46FB681B68C2F309
S3150802AE7008029A62BB690233BB6107E0FB691A786A
S3150802AE80FB681B689A62FB690133FB61FB68B3F8CE
S3150802AE9056309BB2013B9AB2FB68A3F85620FB6870
S3150802AEA0B3F856309BB2002BC8D13B6800937B6936
S3150802AEB000224021F86800F07BFF0346002B05D0EC
S3150802AEC0FB682022C3F88820032306E0FB682022B9
S3150802AED0C3F88820002300E0022318462037BD461F
S3150802AEE080BD000080B58AB000AFF860B96013462D
S3150802AEF0FB80FB68D3F88C30202B4BD1BB68002B28
S3150802AF0002D0FB88002B01D1012344E0FB68002212
S3150802AF10DA66FB681B689B6803F04003402B07D17F
S3150802AF20FB681B689A68FB681B6822F040029A60F5
S3150802AF30FB681B681A4A934224D0FB681B68194AA5
S3150802AF4093421FD0FB681B685B6803F40003002B5F
S3150802AF5018D0FB681B687B617B6953E8003F3B613D
S3150802AF603B6943F080637B62FB681B681A467B6A0F
S3150802AF703B62FA61F9693A6A41E80023BB61BB6937
S3150802AF80002BE6D1FB881A46B968F86800F078FF04
S3150802AF90034600E0022318462837BD4680BD00BF97
S3150802AFA0002400440024005480B594B000AF7860B1
S3150802AFB07B681B687B637B6B53E8003F3B633B6B99
S3150802AFC023F49073FB647B681B681A46FB6C3B642C
S3150802AFD0FA63F96B3A6C41E80023BB63BB6B002B3F
S3150802AFE0E6D17B681B6808333B623B6A53E8003F3D
S3150802AFF0FB61FB6923F0805323F00103BB647B6882
S3150802B0001B680833BA6CFA62BB62B96AFA6A41E823
S3150802B01000237B627B6A002BE3D17B68DB6E012B04
S3150802B02018D17B681B68FB60FB6853E8003FBB606E
S3150802B030BB6823F010037B647B681B681A467B6C2B
S3150802B040BB617A617969BA6941E800233B613B6968
S3150802B050002BE6D17B681B689B6803F04003402BF4
S3150802B0603AD17B68D3F88030002B17D07B68D3F8A7
S3150802B0708030264ADA667B68D3F880301846F6F7B7
S3150802B080CDFA0346002B3CD07B68D3F88030DB6EC2
S3150802B0907A68D2F880201046984732E07B68002208
S3150802B0A0A3F85E207B6800229A657B681B680F22DC
S3150802B0B01A627B681B689A697B681B6842F00802F9
S3150802B0C09A617B682022C3F88C207B680022DA66A4
S3150802B0D0786800F0FBFA14E07B680022A3F85E2089
S3150802B0E07B6800229A657B681B680F221A627B6856
S3150802B0F02022C3F88C207B680022DA66786800F082
S3150802B100E5FA002318465037BD4680BDBDC1020880
S3150802B11080B5AEB000AF78607B681B68DB69C7F89C
S3150802B120B4307B681B681B68C7F8B0307B681B683D
S3150802B1309B68C7F8AC30D7F8B42040F60F03134023
S3150802B140C7F8A830D7F8A830002B1BD1D7F8B430E7
S3150802B15003F02003002B15D0D7F8B03003F02003F4
S3150802B160002B05D1D7F8AC3003F08053002B09D059
S3150802B1707B685B6F002B00F093827B685B6F786855
S3150802B18098478DE2D7F8A830002B00F0FD80D7F853
S3150802B190AC207A4B1340002B06D1D7F8B020784B57
S3150802B1A01340002B00F0F080D7F8B43003F0010307
S3150802B1B0002B11D0D7F8B03003F48073002B0BD0D4
S3150802B1C07B681B6801221A627B68D3F8903043F0C9
S3150802B1D001027B68C3F89020D7F8B43003F0020363
S3150802B1E0002B11D0D7F8AC3003F00103002B0BD09B
S3150802B1F07B681B6802221A627B68D3F8903043F098
S3150802B20004027B68C3F89020D7F8B43003F004032D
S3150802B210002B11D0D7F8AC3003F00103002B0BD06A
S3150802B2207B681B6804221A627B68D3F8903043F065
S3150802B23002027B68C3F89020D7F8B43003F00803FB
S3150802B240002B17D0D7F8B03003F02003002B05D116
S3150802B250D7F8AC20494B1340002B0BD07B681B68F0
S3150802B26008221A627B68D3F8903043F008027B689A
S3150802B270C3F89020D7F8B43003F40063002B12D039
S3150802B280D7F8B03003F08063002B0CD07B681B68BC
S3150802B2904FF400621A627B68D3F8903043F02002BA
S3150802B2A07B68C3F890207B68D3F89030002B00F0B7
S3150802B2B0F981D7F8B43003F02003002B13D0D7F85E
S3150802B2C0B03003F02003002B05D1D7F8AC3003F0D9
S3150802B2D08053002B07D07B685B6F002B03D07B68FB
S3150802B2E05B6F786898477B68D3F89030C7F8A430C4
S3150802B2F07B681B689B6803F04003402B05D0D7F890
S3150802B300A43003F02803002B2ED0786800F0DAFE6A
S3150802B3107B681B689B6803F04003402B20D17B683F
S3150802B320D3F88030002B17D07B68D3F88030154AC3
S3150802B330DA667B68D3F880301846F6F76FF9034663
S3150802B340002B19D07B68D3F88030DB6E7A68D2F886
S3150802B3508020104698470FE078682AF00FFA0BE02B
S3150802B36078682AF00BFA07E078682AF007FA7B6809
S3150802B3700022C3F8902095E100BF93E10100001076
S3150802B3802001000491C102087B68DB6E012B40F0A4
S3150802B3902981D7F8B43003F01003002B00F022817C
S3150802B3A0D7F8B03003F01003002B00F01B817B683E
S3150802B3B01B6810221A627B681B689B6803F04003AD
S3150802B3C0402B40F091807B68D3F880301B689B6CD9
S3150802B3D0A7F89230B7F89230002B00F065817B68A7
S3150802B3E0B3F85C30B7F892209A4280F05D817B68A8
S3150802B3F0B7F89220A3F85E207B68D3F880301B6DDD
S3150802B400812B60D07B681B687B677B6F53E8003FA4
S3150802B4103B673B6F23F48073C7F88C307B681B68E5
S3150802B4201A46D7F88C30C7F88030FA67F96FD7F81A
S3150802B430802041E80023BB67BB6F002BE2D17B6803
S3150802B4401B6808333B663B6E53E8003FFB65FB6DA2
S3150802B45023F00103C7F888307B681B680833D7F8DE
S3150802B4608820FA66BB66B96EFA6E41E800237B66E7
S3150802B4707B6E002BE3D17B682022C3F88C207B6885
S3150802B4800022DA667B681B68FB64FB6C53E8003FA4
S3150802B490BB64BB6C23F01003C7F884307B681B6857
S3150802B4A01A46D7F88430BB657A65796DBA6D41E874
S3150802B4B000233B653B6D002BE4D17B68D3F88030D3
S3150802B4C01846F6F72FF87B6802221A677B68B3F8E4
S3150802B4D05C207B68B3F85E309BB2D31A9BB21946DE
S3150802B4E0786800F0FDF8DFE07B68B3F85C207B68DB
S3150802B4F0B3F85E309BB2D31AA7F8A2307B68B3F8CA
S3150802B5005E309BB2002B00F0D180B7F8A230002B38
S3150802B51000F0CC807B681B68BB63BB6B53E8003FBB
S3150802B5207B637B6B23F49073C7F89C307B681B683C
S3150802B5301A46D7F89C307B643A64396C7A6C41E8CF
S3150802B5400023FB63FB6B002BE4D17B681B68083383
S3150802B5507B627B6A53E8003F3B623B6A23F0805377
S3150802B56023F00103C7F898307B681B680833D7F8BD
S3150802B57098203A63FB62F96A3A6B41E80023BB6298
S3150802B580BB6A002BE1D17B682022C3F88C207B683A
S3150802B5900022DA667B6800225A677B681B683B6171
S3150802B5A03B6953E8003FFB60FB6823F01003C7F8CA
S3150802B5B094307B681B681A46D7F89430FB61BA61E7
S3150802B5C0B969FA6941E800237B617B69002BE4D1FA
S3150802B5D07B6802221A67B7F8A2301946786800F023
S3150802B5E07FF863E0D7F8B43003F48013002B0ED04B
S3150802B5F0D7F8AC3003F48003002B08D07B681B68AD
S3150802B6004FF480121A62786801F060FB51E0D7F8AD
S3150802B610B43003F08003002B14D0D7F8B03003F00F
S3150802B6208003002B05D1D7F8AC3003F40003002BB6
S3150802B63008D07B689B6F002B3AD07B689B6F786833
S3150802B640984735E0D7F8B43003F04003002B09D009
S3150802B650D7F8B03003F04003002B03D0786800F027
S3150802B660D2FD26E0D7F8B43003F40003002B09D044
S3150802B670D7F8B03003F08043002B03D0786801F086
S3150802B68039FB16E0D7F8B43003F08073002B10D0DC
S3150802B690D7F8B030002B0CDA786801F021FB08E005
S3150802B6A000BF06E000BF04E000BF02E000BF00E002
S3150802B6B000BFB837BD4680BD80B483B000AF78609E
S3150802B6C000BF0C37BD465DF8047B704780B483B073
S3150802B6D000AF786000BF0C37BD465DF8047B704743
S3150802B6E080B483B000AF78600B467B8000BF0C370E
S3150802B6F0BD465DF8047B704780B485B000AF7860BC
S3150802B7007B68D3F88830FB607B68D3F88C30BB60E3
S3150802B710FA68BB68134318461437BD465DF8047BBE
S3150802B720704780B483B000AF78607B68D3F89030F6
S3150802B73018460C37BD465DF8047B70472DE9B04FB5
S3150802B74094B000AFF862002387F84730FB6A1A689C
S3150802B750784B9A42FB6A9A68FB6A1B691A43FB6A28
S3150802B7605B691A43FB6ADB691343FB64FB6A1B6862
S3150802B7701B6871491940FB6A1A68FB6C0B43136014
S3150802B780FB6A1B685B6823F44050FB6AD968FB6A4C
S3150802B7901A6840EA01035360FB6A9B69FB64FB6A09
S3150802B7A01A68644B9A4209D0FB6A1A68634B9A4232
S3150802B7B004D0FB6A1A6AFB6C1343FB64FB6A1B68B8
S3150802B7C09B6823F06E4121F43061FB6A1A68FB6CB0
S3150802B7D00B439360FB6A1B68DB6A23F00F00FB6A64
S3150802B7E0596AFB6A1A6840EA0103D362FB6A1A6855
S3150802B7F0534B9A4202D10123BB6466E0FB6A1A687C
S3150802B800504B9A4202D10223BB645EE0FB6A1A6875
S3150802B8104D4B9A4202D10423BB6456E0FB6A1A686E
S3150802B8204A4B9A4202D10823BB644EE0FB6A1A6865
S3150802B830474B9A4202D11023BB6446E0FB6A1A6858
S3150802B840444B9A4202D12023BB643EE0FB6A1A6843
S3150802B850414B9A4202D14023BB6436E0FB6A1A681E
S3150802B8603E4B9A4202D18023BB642EE0FB6A1A68D9
S3150802B8703B4B9A4203D14FF48073BB6425E0FB6AC3
S3150802B8801A68384B9A4203D14FF40073BB641CE022
S3150802B890FB6A1A68344B9A4203D14FF48063BB643D
S3150802B8A013E0FB6A1A68314B9A4203D14FF40063DC
S3150802B8B0BB640AE0FB6A1A681E4B9A4203D14FF42C
S3150802B8C08053BB6401E00023BB64FB6A1A68194B08
S3150802B8D09A4205D0FB6A1A68184B9A4240F094803D
S3150802B8E0BB6C00223B627A62D7E90801FAF764FF69
S3150802B8F038643B6C002B00F0F780FB6A5B6A1C4AD3
S3150802B90032F813301A463B6CB3FBF2F37B63FB6ADD
S3150802B9105A6813465B0013447A6B9A4205D3FB6A4C
S3150802B9205B681B037A6B9A4224D9012387F847304E
S3150802B93069E000BF00240044F369FFCF00240054E5
S3150802B940003801400044004000480040004C0040D6
S3150802B950005000400064004000780040007C00402F
S3150802B9600080004000680040006C004000840040EF
S3150802B970B48D08083B6C0022BB61FA61FB6A5B6AFC
S3150802B980644A32F813309BB200223B617A61D7E9E6
S3150802B9900423D7E90601F5F7ABFA02460B46104629
S3150802B9A019464FF000024FF000030B0243EA1063F8
S3150802B9B00202F96A4968490800200C46054612EB54
S3150802B9C0040843EB0509FB6A5B680022BB60FA6060
S3150802B9D0D7E9022340464946F5F78AFA02460B4654
S3150802B9E01346FB63FB6BB3F5407F08D3FB6BB3F5DA
S3150802B9F0801F04D2FB6A1B68FA6BDA6003E0012334
S3150802BA0087F8473070E06FE0FB6ADB69B3F5004FF1
S3150802BA103CD1BB6C00223B607A60D7E90001FAF799
S3150802BA20CBFE38643B6C002B5ED0FB6A5B6A394AF4
S3150802BA3032F813301A463B6CB3FBF2F35A00FB6A30
S3150802BA405B685B081A44FB6A5B68B2FBF3F3FB6349
S3150802BA50FB6B0F2B16D9FB6BB3F5803F12D2FB6B30
S3150802BA609BB223F00F037B87FB6B5B089BB203F049
S3150802BA7007039AB27B8F13437B87FB6A1B687A8F0D
S3150802BA80DA6031E0012387F847302DE0BB6C0022EB
S3150802BA909A46934650465946FAF78EFE38643B6CE8
S3150802BAA0002B21D0FB6A5B6A1A4A32F813301A460F
S3150802BAB03B6CB3FBF2F2FB6A5B685B081A44FB6AEF
S3150802BAC05B68B2FBF3F3FB63FB6B0F2B09D9FB6BCA
S3150802BAD0B3F5803F05D2FB6B9AB2FB6A1B68DA6044
S3150802BAE002E0012387F84730FB6A0122A3F86A209D
S3150802BAF0FB6A0122A3F86820FB6A00225A67FB6ADE
S3150802BB0000229A6797F8473018465037BD46BDE86F
S3150802BB10B08F00BFB48D080880B483B000AF7860D8
S3150802BB207B689B6A03F00803002B0AD07B681B68B4
S3150802BB305B6823F400417B689A6B7B681B680A433F
S3150802BB405A607B689B6A03F00103002B0AD07B6864
S3150802BB501B685B6823F400317B68DA6A7B681B68BA
S3150802BB600A435A607B689B6A03F00203002B0AD0D9
S3150802BB707B681B685B6823F480317B681A6B7B6879
S3150802BB801B680A435A607B689B6A03F00403002B0E
S3150802BB900AD07B681B685B6823F480217B685A6B32
S3150802BBA07B681B680A435A607B689B6A03F010032A
S3150802BBB0002B0AD07B681B689B6823F480517B683C
S3150802BBC0DA6B7B681B680A439A607B689B6A03F098
S3150802BBD02003002B0AD07B681B689B6823F400515C
S3150802BBE07B681A6C7B681B680A439A607B689B6A47
S3150802BBF003F04003002B1AD07B681B685B6823F4AA
S3150802BC0080117B685A6C7B681B680A435A607B689A
S3150802BC105B6CB3F5801F0AD17B681B685B6823F4EB
S3150802BC20C0017B689A6C7B681B680A435A607B680A
S3150802BC309B6A03F08003002B0AD07B681B685B684B
S3150802BC4023F400217B68DA6C7B681B680A435A6016
S3150802BC5000BF0C37BD465DF8047B704780B598B0C7
S3150802BC6002AF78607B680022C3F89020F5F73CFBA8
S3150802BC7078657B681B681B6803F00803082B2FD1BD
S3150802BC806FF07E4300937B6D00224FF400117868B3
S3150802BC9000F08EF80346002B22D07B681B68BB6334
S3150802BCA0BB6B53E8003F7B637B6B23F080033B65EA
S3150802BCB07B681B681A463B6D7B643A64396C7A6CFE
S3150802BCC041E80023FB63FB6B002BE6D17B6820224D
S3150802BCD0C3F888207B68002283F88420032363E064
S3150802BCE07B681B681B6803F00403042B49D16FF0B9
S3150802BCF07E4300937B6D00224FF48001786800F042
S3150802BD0057F80346002B3CD07B681B687B627B6A2C
S3150802BD1053E8003F3B623B6A23F49073FB647B68FB
S3150802BD201B681A46FB6C3B63FA62F96A3A6B41E88E
S3150802BD300023BB62BB6A002BE6D17B681B6808330B
S3150802BD403B613B6953E8003FFB60FB6823F0010354
S3150802BD50BB647B681B680833BA6CFA61BB61B96954
S3150802BD60FA6941E800237B617B69002BE5D17B6890
S3150802BD702022C3F88C207B68002283F884200323C0
S3150802BD8012E07B682022C3F888207B682022C3F849
S3150802BD908C207B680022DA667B6800221A677B6839
S3150802BDA0002283F88420002318465837BD4680BDF2
S3150802BDB080B584B000AFF860B9603B601346FB718A
S3150802BDC049E0BB69B3F1FF3F45D0F5F78DFA024664
S3150802BDD03B68D31ABA699A4202D3BB69002B01D1CE
S3150802BDE0032348E0FB681B681B6803F00403002B67
S3150802BDF031D0FB681B68DB6903F00803082B10D1F6
S3150802BE00FB681B6808221A62F86800F05BF9FB688F
S3150802BE100822C3F89020FB68002283F884200123B5
S3150802BE2029E0FB681B68DB6903F40063B3F5006F5E
S3150802BE3011D1FB681B684FF400621A62F86800F0B9
S3150802BE4041F9FB682022C3F89020FB68002283F898
S3150802BE50842003230FE0FB681B68DA69BB6813407A
S3150802BE60BA689A420CBF01230023DBB21A46FB7951
S3150802BE709A42A6D0002318461037BD4680BD000058
S3150802BE8080B4A3B000AFF860B9601346FB80FB68C4
S3150802BE90BA689A65FB68FA88A3F85C20FB68FA8890
S3150802BEA0A3F85E20FB6800225A67FB689B68B3F515
S3150802BEB0805F0ED1FB681B69002B05D1FB6840F237
S3150802BEC0FF12A3F860202DE0FB68FF22A3F860208A
S3150802BED028E0FB689B68002B0DD1FB681B69002BC9
S3150802BEE004D1FB68FF22A3F860201BE0FB687F22CF
S3150802BEF0A3F8602016E0FB689B68B3F1805F0DD15A
S3150802BF00FB681B69002B04D1FB687F22A3F860201B
S3150802BF1008E0FB683F22A3F8602003E0FB680022E2
S3150802BF20A3F86020FB680022C3F89020FB6822224F
S3150802BF30C3F88C20FB681B6808337B667B6E53E864
S3150802BF40003F3B663B6E43F00103C7F88430FB684B
S3150802BF501B680833D7F884203A67FB66F96E3A6F8E
S3150802BF6041E80023BB66BB6E002BE3D1FB685B6E20
S3150802BF70B3F1005F4FD1FB68B3F86830FA889A428A
S3150802BF8049D3FB689B68B3F5805F07D1FB681B69D9
S3150802BF90002B03D1FB68474A5A6702E0FB68464A08
S3150802BFA05A67FB681B69002B1AD0FB681B683B653E
S3150802BFB03B6D53E8003FFB64FB6C43F48073C7F8A0
S3150802BFC08030FB681B681A46D7F88030FB65BA656D
S3150802BFD0B96DFA6D41E800237B657B6D002BE4D1D0
S3150802BFE0FB681B680833FB63FB6B53E8003FBB63C4
S3150802BFF0BB6B43F08053FB67FB681B680833FA6F19
S3150802C000BA647B64796CBA6C41E800233B643B6C86
S3150802C010002BE5D146E0FB689B68B3F5805F07D144
S3150802C020FB681B69002B03D1FB68244A5A6702E0A6
S3150802C030FB68234A5A67FB681B69002B19D0FB6801
S3150802C0401B68BB62BB6A53E8003F7B627B6A43F4A8
S3150802C05090737B67FB681B681A467B6F7B633A6340
S3150802C060396B7A6B41E80023FB62FB6A002BE6D147
S3150802C07018E0FB681B687B617B6953E8003F3B61FC
S3150802C0803B6943F02003BB67FB681B681A46BB6F14
S3150802C0903B62FA61F9693A6A41E80023BB61BB6906
S3150802C0A0002BE6D1002318468C37BD465DF8047B83
S3150802C0B0704700BF55C90208E5C5020821C402082F
S3150802C0C05DC2020880B495B000AF78607B681B68D1
S3150802C0D07B637B6B53E8003F3B633B6B23F49073B4
S3150802C0E0FB647B681B681A46FB6C3B64FA63F96B54
S3150802C0F03A6C41E80023BB63BB6B002BE6D17B6835
S3150802C1001B6808333B623B6A53E8003FFB61FB69E5
S3150802C11023F0805323F00103BB647B681B68083352
S3150802C120BA6CFA62BB62B96AFA6A41E800237B62B0
S3150802C1307B6A002BE3D17B68DB6E012B18D17B6807
S3150802C1401B68FB60FB6853E8003FBB60BB6823F0D3
S3150802C15010037B647B681B681A467B6CBB617A6139
S3150802C1607969BA6941E800233B613B69002BE6D14C
S3150802C1707B682022C3F88C207B680022DA667B68FB
S3150802C18000225A6700BF5437BD465DF8047B7047E4
S3150802C19080B584B000AF78607B68DB6DFB60FB68B6
S3150802C1A00022A3F85E20FB680022A3F85620F8684E
S3150802C1B029F0E4FA00BF1037BD4680BD80B584B0C9
S3150802C1C000AF78607B68DB6DFB60FB680022A3F832
S3150802C1D05E20FB681B680F221A62FB681B689A6955
S3150802C1E0FB681B6842F008029A61FB682022C3F8C2
S3150802C1F08C20FB680022DA66F868FFF767FA00BF48
S3150802C2001037BD4680BD80B588B000AF78607B68C0
S3150802C2101B68FB60FB6853E8003FBB60BB6823F002
S3150802C2204003FB617B681B681A46FB69BB617A613E
S3150802C2307969BA6941E800233B613B69002BE6D17B
S3150802C2407B682022C3F888207B6800229A67786870
S3150802C250FFF732FA00BF2037BD4680BD80B59CB0D5
S3150802C26000AF78607B68B3F86030A7F86E307B68F9
S3150802C270D3F88C30222B40F0C3807B681B685B6A3C
S3150802C280A7F86C30B7F86C30D9B2B7F86E30DAB2B4
S3150802C2907B689B6D0A40D2B21A707B689B6D5A1CEA
S3150802C2A07B689A657B68B3F85E309BB2013B9AB2AB
S3150802C2B07B68A3F85E207B68B3F85E309BB2002BDE
S3150802C2C040F0A6807B681B68FB64FB6C53E8003F62
S3150802C2D0BB64BB6C23F49073BB667B681B681A4607
S3150802C2E0BB6EBB657A65796DBA6D41E800233B651D
S3150802C2F03B6D002BE6D17B681B680833BB63BB6BBF
S3150802C30053E8003F7B637B6B23F001037B667B6804
S3150802C3101B6808337A6E7A643B64396C7A6C41E836
S3150802C3200023FB63FB6B002BE5D17B682022C3F855
S3150802C3308C207B6800225A677B6800221A677B6812
S3150802C3401B68354A934224D07B681B68334A93425A
S3150802C3501FD07B681B685B6803F40003002B18D0A8
S3150802C3607B681B687B627B6A53E8003F3B623B6AD9
S3150802C37023F080633B667B681B681A463B6E3B6309
S3150802C380FA62F96A3A6B41E80023BB62BB6A002B80
S3150802C390E6D17B68DB6E012B2ED17B680022DA663A
S3150802C3A07B681B683B613B6953E8003FFB60FB689F
S3150802C3B023F01003FB657B681B681A46FB6DFB615D
S3150802C3C0BA61B969FA6941E800237B617B69002B86
S3150802C3D0E6D17B681B68DB6903F01003102B03D1D7
S3150802C3E07B681B6810221A627B68B3F85C301946B0
S3150802C3F07868FFF775F90BE0786829F09FF907E086
S3150802C4007B681B689A697B681B6842F008029A6116
S3150802C41000BF7037BD4680BD002400440024005486
S3150802C42080B59CB000AF78607B68B3F86030A7F837
S3150802C4306E307B68D3F88C30222B40F0C3807B6841
S3150802C4401B685B6AA7F86C307B689B6DBB66B7F89E
S3150802C4506C20B7F86E3013409AB2BB6E1A807B68AE
S3150802C4609B6D9A1C7B689A657B68B3F85E309BB2B3
S3150802C470013B9AB27B68A3F85E207B68B3F85E300C
S3150802C4809BB2002B40F0A6807B681B68BB64BB6C22
S3150802C49053E8003F7B647B6C23F490737B667B686E
S3150802C4A01B681A467B6E7B653A65396D7A6D41E87B
S3150802C4B00023FB64FB6C002BE6D17B681B68083300
S3150802C4C07B637B6B53E8003F3B633B6B23F00103C3
S3150802C4D03B667B681B6808333A6E3A64FB63F96B02
S3150802C4E03A6C41E80023BB63BB6B002BE5D17B6842
S3150802C4F02022C3F88C207B6800225A677B680022B8
S3150802C5001A677B681B68354A934224D07B681B6886
S3150802C510334A93421FD07B681B685B6803F40003A7
S3150802C520002B18D07B681B683B623B6A53E8003FC6
S3150802C530FB61FB6923F08063FB657B681B681A460F
S3150802C540FB6DFB62BA62B96AFA6A41E800237B624A
S3150802C5507B6A002BE6D17B68DB6E012B2ED17B68CA
S3150802C5600022DA667B681B68FB60FB6853E8003FBB
S3150802C570BB60BB6823F01003BB657B681B681A4661
S3150802C580BB6DBB617A617969BA6941E800233B618F
S3150802C5903B69002BE6D17B681B68DB6903F0100355
S3150802C5A0102B03D17B681B6810221A627B68B3F8CA
S3150802C5B05C3019467868FFF793F80BE0786829F03B
S3150802C5C0BDF807E07B681B689A697B681B6842F0BE
S3150802C5D008029A6100BF7037BD4680BD0024004438
S3150802C5E00024005480B5ACB000AF78607B68B3F81D
S3150802C5F06030A7F8AA307B681B68DB69C7F8AC30DD
S3150802C6007B681B681B68C7F8A4307B681B689B6835
S3150802C610C7F8A0307B68D3F88C30222B40F087818C
S3150802C6207B68B3F86830A7F89E302AE17B681B68F6
S3150802C6305B6AA7F89C30B7F89C30D9B2B7F8AA302B
S3150802C640DAB27B689B6D0A40D2B21A707B689B6D20
S3150802C6505A1C7B689A657B68B3F85E309BB2013BCD
S3150802C6609AB27B68A3F85E207B681B68DB69C7F809
S3150802C670AC30D7F8AC3003F00703002B53D0D7F809
S3150802C680AC3003F00103002B11D0D7F8A43003F421
S3150802C6908073002B0BD07B681B6801221A627B68A9
S3150802C6A0D3F8903043F001027B68C3F89020D7F89C
S3150802C6B0AC3003F00203002B11D0D7F8A03003F0F8
S3150802C6C00103002B0BD07B681B6802221A627B6867
S3150802C6D0D3F8903043F004027B68C3F89020D7F869
S3150802C6E0AC3003F00403002B11D0D7F8A03003F0C6
S3150802C6F00103002B0BD07B681B6804221A627B6835
S3150802C700D3F8903043F002027B68C3F890207B6826
S3150802C710D3F89030002B06D0786829F02FF87B687A
S3150802C7200022C3F890207B68B3F85E309BB2002BD8
S3150802C73040F0A7807B681B683B673B6F53E8003F66
S3150802C740FB66FB6E23F48073C7F898307B681B6818
S3150802C7501A46D7F89830FB67BA67B96FFA6F41E895
S3150802C76000237B677B6F002BE4D17B681B68083349
S3150802C770FB65FB6D53E8003FBB65BB6D23F0805339
S3150802C78023F00103C7F894307B681B680833D7F88F
S3150802C7909420BA667B66796EBA6E41E800233B66D8
S3150802C7A03B6E002BE1D17B682022C3F88C207B6884
S3150802C7B000225A677B6800221A677B681B68624AEE
S3150802C7C0934226D07B681B68604A934221D07B68D5
S3150802C7D01B685B6803F40003002B1AD07B681B688E
S3150802C7E0BB64BB6C53E8003F7B647B6C23F08063BD
S3150802C7F0C7F890307B681B681A46D7F890307B6575
S3150802C8003A65396D7A6D41E80023FB64FB6C002BAF
S3150802C810E4D17B68DB6E012B30D17B680022DA66B5
S3150802C8207B681B687B637B6B53E8003F3B633B6B10
S3150802C83023F01003C7F88C307B681B681A46D7F8B2
S3150802C8408C303B64FA63F96B3A6C41E80023BB63AC
S3150802C850BB6B002BE4D17B681B68DB6903F0100312
S3150802C860102B03D17B681B6810221A627B68B3F807
S3150802C8705C3019467868FEF733FF02E0786828F0DC
S3150802C8805DFFB7F89E30002B06D0D7F8AC3003F020
S3150802C8902003002B7FF4CAAE7B68B3F85E30A7F894
S3150802C8A08A30B7F88A30002B49D07B68B3F86830EB
S3150802C8B0B7F88A209A4242D27B681B6808333B62E1
S3150802C8C03B6A53E8003FFB61FB6923F08053C7F8D4
S3150802C8D084307B681B680833D7F88420FA62BB6207
S3150802C8E0B96AFA6A41E800237B627B6A002BE3D1C4
S3150802C8F07B68174A5A677B681B68FB60FB6853E8C4
S3150802C900003FBB60BB6843F02003C7F880307B68F2
S3150802C9101B681A46D7F88030BB617A617969BA69A9
S3150802C92041E800233B613B69002BE4D107E07B68C1
S3150802C9301B689A697B681B6842F008029A6100BF05
S3150802C940B037BD4680BD00BF002400440024005411
S3150802C9505DC2020880B5AEB000AF78607B68B3F8F6
S3150802C9606030A7F8B2307B681B68DB69C7F8B43059
S3150802C9707B681B681B68C7F8AC307B681B689B68BA
S3150802C980C7F8A8307B68D3F88C30222B40F08B810D
S3150802C9907B68B3F86830A7F8A6302EE17B681B6877
S3150802C9A05B6AA7F8A4307B689B6DC7F8A030B7F816
S3150802C9B0A420B7F8B23013409AB2D7F8A0301A803A
S3150802C9C07B689B6D9A1C7B689A657B68B3F85E30B8
S3150802C9D09BB2013B9AB27B68A3F85E207B681B6810
S3150802C9E0DB69C7F8B430D7F8B43003F00703002B75
S3150802C9F053D0D7F8B43003F00103002B11D0D7F87F
S3150802CA00AC3003F48073002B0BD07B681B680122C1
S3150802CA101A627B68D3F8903043F001027B68C3F848
S3150802CA209020D7F8B43003F00203002B11D0D7F8C0
S3150802CA30A83003F00103002B0BD07B681B68022287
S3150802CA401A627B68D3F8903043F004027B68C3F815
S3150802CA509020D7F8B43003F00403002B11D0D7F88E
S3150802CA60A83003F00103002B0BD07B681B68042255
S3150802CA701A627B68D3F8903043F002027B68C3F8E7
S3150802CA8090207B68D3F89030002B06D0786828F07F
S3150802CA9075FE7B680022C3F890207B68B3F85E3087
S3150802CAA09BB2002B40F0A9807B681B687B677B6F73
S3150802CAB053E8003F3B673B6F23F48073C7F89C300B
S3150802CAC07B681B681A46D7F89C30C7F88030FA6725
S3150802CAD0F96FD7F8802041E80023BB67BB6F002BAC
S3150802CAE0E2D17B681B6808333B663B6E53E8003F1E
S3150802CAF0FB65FB6D23F0805323F00103C7F89830DA
S3150802CB007B681B680833D7F89820FA66BB66B96E45
S3150802CB10FA6E41E800237B667B6E002BE1D17B68C7
S3150802CB202022C3F88C207B6800225A677B68002281
S3150802CB301A677B681B68624A934226D07B681B6821
S3150802CB40604A934221D07B681B685B6803F4000342
S3150802CB50002B1AD07B681B68FB64FB6C53E8003F0A
S3150802CB60BB64BB6C23F08063C7F894307B681B6890
S3150802CB701A46D7F89430BB657A65796DBA6D41E87D
S3150802CB8000233B653B6D002BE4D17B68DB6E012BF2
S3150802CB9030D17B680022DA667B681B68BB63BB6B95
S3150802CBA053E8003F7B637B6B23F01003C7F8903092
S3150802CBB07B681B681A46D7F890307B643A64396CEE
S3150802CBC07A6C41E80023FB63FB6B002BE4D17B689C
S3150802CBD01B68DB6903F01003102B03D17B681B6803
S3150802CBE010221A627B68B3F85C3019467868FEF739
S3150802CBF077FD02E0786828F0A1FDB7F8A630002B89
S3150802CC0006D0D7F8B43003F02003002B7FF4C6AE63
S3150802CC107B68B3F85E30A7F88E30B7F88E30002BF3
S3150802CC2049D07B68B3F86830B7F88E209A4242D268
S3150802CC307B681B6808337B627B6A53E8003F3B626A
S3150802CC403B6A23F08053C7F888307B681B68083331
S3150802CC50D7F888203A63FB62F96A3A6B41E80023FF
S3150802CC60BB62BB6A002BE3D17B68174A5A677B68AB
S3150802CC701B683B613B6953E8003FFB60FB6843F076
S3150802CC802003C7F884307B681B681A46D7F88430B5
S3150802CC90FB61BA61B969FA6941E800237B617B697C
S3150802CCA0002BE4D107E07B681B689A697B681B68DE
S3150802CCB042F008029A6100BFB837BD4680BD00BF80
S3150802CCC0002400440024005421C4020880B483B01E
S3150802CCD000AF786000BF0C37BD465DF8047B70472D
S3150802CCE080B483B000AF786000BF0C37BD465DF8EC
S3150802CCF0047B704780B483B000AF786000BF0C37FE
S3150802CD00BD465DF8047B704780B485B000AF786095
S3150802CD107B6893F88430012B01D1022327E07B68D4
S3150802CD20012283F884207B682422C3F888207B6842
S3150802CD301B681B68FB607B681B681A687B681B6834
S3150802CD4022F001021A60FB6823F00053FB607B683D
S3150802CD5000225A667B681B68FA681A607B6820227A
S3150802CD60C3F888207B68002283F8842000231846AB
S3150802CD701437BD465DF8047B704780B584B000AFB2
S3150802CD80786039607B6893F88430012B01D10223DD
S3150802CD902DE07B68012283F884207B682422C3F86D
S3150802CDA088207B681B681B68FB607B681B681A689F
S3150802CDB07B681B6822F001021A607B681B689B6805
S3150802CDC023F060417B681B683A680A439A60786870
S3150802CDD000F050F87B681B68FA681A607B682022A4
S3150802CDE0C3F888207B68002283F88420002318462B
S3150802CDF01037BD4680BD80B584B000AF7860396013
S3150802CE007B6893F88430012B01D102232DE07B68DD
S3150802CE10012283F884207B682422C3F888207B6851
S3150802CE201B681B68FB607B681B681A687B681B6843
S3150802CE3022F001021A607B681B689B6823F0606116
S3150802CE407B681B683A680A439A60786800F012F8A9
S3150802CE507B681B68FA681A607B682022C3F88820F8
S3150802CE607B68002283F88420002318461037BD46C3
S3150802CE7080BD000080B485B000AF78607B685B6EC9
S3150802CE80002B08D17B680122A3F86A207B6801225D
S3150802CE90A3F8682031E00823FB730823BB737B6879
S3150802CEA01B689B685B0EDBB203F007037B737B6828
S3150802CEB01B689B685B0FDBB203F007033B73BB7B04
S3150802CEC03A7B11498A5C02FB03F33A7B0F498A5C77
S3150802CED093FBF2F39AB27B68A3F86A20FB7B7A7B10
S3150802CEE009498A5C02FB03F37A7B08498A5C93FB4D
S3150802CEF0F2F39AB27B68A3F8682000BF1437BD46DE
S3150802CF005DF8047B704700BFCC8D0808D48D0808ED
S3150802CF1080B596B000AFF860B9607A603B607B680E
S3150802CF20033323F003037B60EFF310837B637B6B8E
S3150802CF303B6372B63B6B7B65554B1B68BB64002330
S3150802CF40FB64FB68BA6C1A627B6D7B627B6A83F34D
S3150802CF50108800BF7968F86800F0B2F97864EFF3D0
S3150802CF601083FB62FB6ABB6272B6BB6A7B657B6C2B
S3150802CF70002B02D00123FB6406E0FB681B6ABA6C2D
S3150802CF809A4201D10123FB64FB6C002BD9D0BB6802
S3150802CF907A6C1A607B6C002B08D07B6D3B623B6A0D
S3150802CFA083F3108800BF00233B656CE03B68002BC7
S3150802CFB061D0384B1B68002B07D010233B657B6D6D
S3150802CFC0FB61FB6983F310885DE0BB6C324A9A66A3
S3150802CFD0BB6CFA68DA66BB6CBA68DA67BB6C7A68E5
S3150802CFE09A67BB6CD3F8AC305A1CBB6CC3F8AC203E
S3150802CFF0FB689B6A3B64FB689B6A5A1CFB689A62DD
S3150802D0003B6C002B09D1FB68BA6C5A62BB6CBA6CD2
S3150802D0101A67BB6CBA6C5A6711E0FB685B6AFB63FA
S3150802D020BB6CFA6B1A67FB6B5B6FBB63BB6CBA6B49
S3150802D0305A67BB6BBA6C1A67FB6BBA6C5A67BB6CDE
S3150802D04009221A63BB6C01229A63BB6C3A68DA64DA
S3150802D050104B1B6801330F4A13607B6DBB61BB69BA
S3150802D06083F3108800BFB86C01F096FBBB6CD3F84B
S3150802D07084303B6507E07B6D7B617B6983F31088AF
S3150802D08000BF10233B653B6D18465837BD4680BD29
S3150802D090F0140020881500209DD0020880B58EB0B5
S3150802D0A000AF78603960EFF310833B623B6AFB613D
S3150802D0B072B6FB697B637B689B6E334A934258D18F
S3150802D0C07B68D3F8AC303A689A4252D17B68DB6EF9
S3150802D0D03B633B6B002B4CD03B6B1B682B4A934242
S3150802D0E047D13B6B9B6A002B43D07B6800229A662A
S3150802D0F03B6B9B6A5A1E3B6B9A623B6B9B6AFB6253
S3150802D100FB6A002B03D13B6B00225A6213E07B6851
S3150802D1101B6FBB627B685B6F7B62BB6A7A6A5A6704
S3150802D1207B6ABA6A1A673B6B5B6A7A689A4202D169
S3150802D1303B6BBA6A5A627B681B6B092B19D17B68EF
S3150802D1401022C3F88420124B1B680133104A13605D
S3150802D1507B6B3B613B6983F3108800BF786801F0FB
S3150802D1601BFAEFF31083BB61BB697B6172B67B69FD
S3150802D1707B637B6BFB60FB6883F3108800BF00BF91
S3150802D1803837BD4680BD00BF9DD002084554594276
S3150802D1908815002080B58EB000AFF860B9607A6055
S3150802D1A03B6034220021F86848F05CFF3B6823F0B4
S3150802D1B003033B60FB68BA685A60FB687A689A613F
S3150802D1C0FB683A68DA61FB687A681A61FB687A680A
S3150802D1D05A613B68A3F10802FB689A60FB6802225F
S3150802D1E0DA607B687B637A6B3B6813447B637B6B91
S3150802D1F0043B7B63FB683B637B6BFB62FB6A3A6BB4
S3150802D2001A607B6B043B7B637B6BFB62FB6A7A6807
S3150802D2101A607B683B633B6BFB62FB6A7A6B1A603C
S3150802D2207B687B637B6B04337B637B6BBB62BB6A0A
S3150802D2301F4A1A60FB6800221A62EFF31083BB6169
S3150802D240BB697B6172B67B697B62FB68194A1A60A5
S3150802D250194B1B68002B09D1184AFB681360FB6837
S3150802D260FA68DA62FB68FA681A6311E0134B1B68FC
S3150802D2703B623B6A1B6BFB613B6AFA681A63FB6992
S3150802D280FA68DA62FB68FA691A63FB683A6ADA626A
S3150802D290094B1B680133084A13607B6A3B613B6989
S3150802D2A083F3108800BF002318463837BD4680BD71
S3150802D2B0EEEEFFFF45545942E4140020E014002024
S3150802D2C080B497B000AF7860396000237B64EFF3CF
S3150802D2D010837B627B6A3B6272B63B6A7B657B68BC
S3150802D2E09A687B68DB68023BDB0013443B643A6856
S3150802D2F03B6C9A4208D37B6DFB61FB6983F310880A
S3150802D30000BF00233B65DDE0724B1B68FB637B684D
S3150802D310FA6B1A627B685B693B657B68DB6801337B
S3150802D320BB640023FB643B6D0433BB63BB6B7B634B
S3150802D3307B6B1B68684A934243D17B6C002B04D1F2
S3150802D3407B683A6D5A6101237B643B6D3B633B6B99
S3150802D3501B68FB62FA6A3B6DD31AFB64FB6C083BDB
S3150802D360FB64FA6C3B689A4257D20023FB64FB6A59
S3150802D3700433BB63BB6B7B637B6B1B68564A934266
S3150802D38013D1FB6ABB62BB6A1A683B6B1A607B687D
S3150802D390DB685A1E7B68DA607B685B69FA6A9A42BE
S3150802D3A014D17B683A6D5A6110E0FB6ABB62BB6AAC
S3150802D3B01B683B65BB6C002B08D0BB6C013BBB648E
S3150802D3C004E03B6D3B633B6B1B683B65BB6C002B08
S3150802D3D002D0BB6C013BBB647B6D3B613B6983F34B
S3150802D3E0108800BFEFF31083BB61BB697B6172B61D
S3150802D3F07B697B657B681B6AFA6B9A4209D07B68F4
S3150802D4005B693B657B68DB680133BB647B68FA6BE7
S3150802D4101A62BB6C002B86D100E000BFFB6C002BA6
S3150802D42048D0FA6C3B68D31A132B1ED93B680833CB
S3150802D4303A6D1344FB62FB6ABB623B6D3B633B6B13
S3150802D4401A68BB6A1A60FB6A0433BB63BB6B7B63ED
S3150802D4507B6B214A1A607B68DB685A1C7B68DA6038
S3150802D4603B6BFA6A1A603B68FB643B6D0433BB6329
S3150802D470BB6B3B633B6B7A681A607B689A68FB6C8A
S3150802D480D31AA3F108027B689A607B685B693A6DD6
S3150802D4909A4205D13B6D3B633B6B1A687B685A61BE
S3150802D4A07B6DFB60FB6883F3108800BF3B6D083316
S3150802D4B03B6507E07B6DBB60BB6883F3108800BFE2
S3150802D4C000233B653B6D18465C37BD465DF8047B19
S3150802D4D0704700BFF0140020EEEEFFFF80B500AFE4
S3150802D4E000F018FF01F020FB124B00221A60124BC3
S3150802D4F000221A60114B00221A60114B00221A6090
S3150802D500104B00221A60104B00221A600F4B0022A1
S3150802D5101A600F4B00221A600E4B00221A600E4B3D
S3150802D52000221A600D4B00221A600D4B00221A6067
S3150802D53000BF80BDB8140020BC140020C01400200F
S3150802D540C4140020C8140020CC140020D8140020CB
S3150802D550DC140020E0140020E4140020D01400207B
S3150802D560D414002080B500AF104B1B6813F10F3F8F
S3150802D5700CD00E4B4FF0F0321A60F2F771FFFFF73C
S3150802D580ADFF0B4B1B680133094A1360074B4FF07B
S3150802D590F0321A60074B1B68184602F099FD034BD6
S3150802D5A000221A60F2F77AFE00BF80BD240000202E
S3150802D5B088150020E814002080B58EB000AF786088
S3150802D5C03960EFF310833B623B6AFB6172B6FB6913
S3150802D5D07B637B689B6E334A934258D17B68D3F848
S3150802D5E0AC303A689A4252D17B68DB6E3B633B6B3E
S3150802D5F0002B4CD03B6B1B682B4A934247D13B6BA3
S3150802D600DB69002B43D07B6800229A663B6BDB6999
S3150802D6105A1E3B6BDA613B6BDB69FB62FB6A002BCA
S3150802D62003D13B6B00229A6113E07B681B6FBB62D6
S3150802D6307B685B6F7B62BB6A7A6A5A677B6ABA6A7D
S3150802D6401A673B6B9B697A689A4202D13B6BBA6A44
S3150802D6509A617B681B6B0D2B19D17B681D22C3F857
S3150802D6608420124B1B680133104A13607B6B3B61A3
S3150802D6703B6983F3108800BF786800F08DFFEFF3EB
S3150802D6801083BB61BB697B6172B67B697B637B6B0B
S3150802D690FB60FB6883F3108800BF00BF3837BD46BE
S3150802D6A080BD00BFB9D502084554554D88150020DE
S3150802D6B080B58AB000AF7860EFF31083FB61FB692F
S3150802D6C0BB6172B6BB697B621A4B1B680133194A86
S3150802D6D013607B68D3F8A4303B623B6A002B17D0F1
S3150802D6E03B6A01229A607B6AFB60FB6883F31088B7
S3150802D6F000BF386A00F0F2FAEFF310837B617B69A8
S3150802D7003B6172B63B697B627B68D3F8A4303B62A5
S3150802D7103B6A002BDDD1074B1B68013B054A1360A8
S3150802D7207B6ABB60BB6883F3108800BF00BF2837DB
S3150802D730BD4680BD8815002080B58AB000AFF86066
S3150802D740B9607A6034220021F86848F08BFCFB68DD
S3150802D750BA685A60FB687A681A61EFF31083BB618C
S3150802D760BB697B6172B67B697B62FB681A4A1A607F
S3150802D7701A4B1B4A1A601B4B1B68002B09D11A4A03
S3150802D780FB681360FB68FA681A62FB68FA685A62F1
S3150802D79011E0154B1B683B623B6A5B6AFB613B6A9D
S3150802D7A0FA685A62FB69FA681A62FB68FA695A6287
S3150802D7B0FB683A6A1A620B4B1B680133094A136003
S3150802D7C07B6A3B613B6983F3108800BF00231846D6
S3150802D7D02837BD4680BD00BF4554554D8C150020DF
S3150802D7E0B1D60208D4140020D014002080B592B015
S3150802D7F000AF78603960EFF310837B627B6A3B6225
S3150802D80072B63B6A3B647A4B1B68FB637B689B6810
S3150802D810002B44D17B6801229A607B68FA6BDA6036
S3150802D820FB6B002B32D07B681B69012B06D1FB6B85
S3150802D830DA6A7B685A617B6820229A62FB6BD3F8A4
S3150802D840A430FB62FB6A002B0FD0FB6A1B6BBB6220
S3150802D850FB6A7A681A63BB6A7A68DA627B68BA6AAA
S3150802D8601A637B68FA6ADA6209E0FB6B7A68C3F8BC
S3150802D870A4207B687A68DA627B687A681A63FB6B2B
S3150802D880D3F8A0305A1CFB6BC3F8A0203B6CFB6193
S3150802D890FB6983F3108800BF00237B64A2E07B68E0
S3150802D8A0DB68FA6B9A420DD17B689B685A1C7B68C7
S3150802D8B09A603B6CBB61BB6983F3108800BF002387
S3150802D8C07B648FE03B68002B00F08480494B1B6821
S3150802D8D0002B08D03B6C7B617B6983F3108800BF01
S3150802D8E01D237B647EE07B68DB68BB63FB6B424A75
S3150802D8F09A66FB6B7A68DA66FB6BD3F8AC305A1C0D
S3150802D900FB6BC3F8AC207B68DB69002B09D17B680B
S3150802D910FA6B9A61FB6BFA6B1A67FB6BFA6B5A67BF
S3150802D92011E07B689B697B63FB6B7A6B1A677B6B7F
S3150802D9305B6F3B63FB6B3A6B5A673B6BFA6B1A6717
S3150802D9407B6BFA6B5A677B68DB695A1C7B68DA6100
S3150802D950FB6B0D221A63FB6B01229A63FB6B3A6817
S3150802D960DA64244B1B680133224A13603B6C3B6121
S3150802D9703B6983F3108800BF7B681B69012B21D1A1
S3150802D9807B689A6AFB6BDB6A9A4203D9FB6BDA6A93
S3150802D9907B689A62FB6BDA6ABB6BD3F89C309A4255
S3150802D9A004D2FB6BDA6ABB6BC3F89C20BB6BDA6AE0
S3150802D9B0FB6BDB6A9A4205D9FB6BDB6A1946B86BC5
S3150802D9C000F0CEF8F86B00F0E7FEFB6BD3F8843074
S3150802D9D07B6407E03B6CFB60FB6883F3108800BF3F
S3150802D9E01D237B647B6C18464837BD4680BD00BF45
S3150802D9F0F014002088150020B9D5020880B592B027
S3150802DA0000AF7860EFF310837B627B6A3B6272B683
S3150802DA103B6A7B647B68DB697B637B6B012B05D87E
S3150802DA207B6CFB61FB6983F3108892E07B6B022BAC
S3150802DA3014D17B689B69BB63BB6B1B6FFB62FB6A7A
S3150802DA40DA6ABB6BDB6A9A4202D27B68FA6A9A6125
S3150802DA507B6CBB61BB6983F310887AE07B689B6940
S3150802DA60BB63BB6BFB63FB6B1B6F3B643B4B1B686C
S3150802DA7001333A4A136000233B633B6CDA6AFB6B59
S3150802DA80DB6A9A4201D23B6CFB637B6CFB60FB68E8
S3150802DA9083F3108800BFEFF310837B617B693B61D8
S3150802DAA072B63B697B647B689B69BA6B9A4202D001
S3150802DAB001233B6306E07B68DB697A6B9A4201D0F5
S3150802DAC001233B633B6B002B03D13B6C1B6F3B640F
S3150802DAD00CE07B689B69BB637B68DB697B63BB6B1A
S3150802DAE0FB63FB6B1B6F3B6400233B633A6CBB6BAC
S3150802DAF09A42C2D1194B1B68013B184A1360FA6B4A
S3150802DB00BB6B9A421DD0FB6B1B6FFB62FB6B5B6F99
S3150802DB10BB62FB6ABA6A5A67BB6AFA6A1A67BB6B5E
S3150802DB205B6FBB62FB6BBA6B1A67FB6BBA6A5A67A7
S3150802DB30BB6AFA6B1A67BB6BFA6B5A677B68FA6B36
S3150802DB409A617B6CBB60BB6883F3108800BF00F0E8
S3150802DB50E9FC002318464837BD4680BD88150020D3
S3150802DB6080B590B000AF78603960EFF31083FB623E
S3150802DB70FB6ABB6272B6BB6AFB637B681B6B002BD4
S3150802DB8017D07B683A68DA627B68D3F898303A68C5
S3150802DB909A4205D97B68D3F898207B68DA6302E053
S3150802DBA07B683A68DA63FB6B7B627B6A83F310886D
S3150802DBB089E0474B1B68BB637B68DB6A7B63454B23
S3150802DBC01B680233434A13607B680E221A637B681A
S3150802DBD001229A637B680022DA64FB6BBB61BB692C
S3150802DBE083F3108800BF786800F0D6FDEFF3108340
S3150802DBF03B623B6AFB6172B6FB69FB637B683A6808
S3150802DC00DA627B68D3F898303A689A4205D97B6813
S3150802DC10D3F898207B68DA6302E07B683A68DA63AD
S3150802DC20FB6BFB60FB6883F3108800BF786800F023
S3150802DC30B3FCEFF310837B617B693B6172B63B6988
S3150802DC40FB63234B1B683B637A683B6B9A4234D06F
S3150802DC507B681B6B002B30D17B68DA6A3B6BDB6A0D
S3150802DC609A4211D87A68BB6B9A4226D1184A7B68BF
S3150802DC7013607A6B3B689A421FD27B68DB6A164945
S3150802DC807A6841F8232018E07B68DA6B7B68DB6ADE
S3150802DC909A4212D27B68DA6B3B6BDB6A9A420CD8E1
S3150802DCA00B4A7B6813607A6B3B689A4205D27B689B
S3150802DCB0DB6A09497A6841F82320FB6BBB60BB68BB
S3150802DCC083F3108800BF00BF4037BD4680BD00BF42
S3150802DCD0F4140020881500200815002080B5A6B087
S3150802DCE000AF78602023C7F88830EFF31083FB650E
S3150802DCF0FB6DBB6572B6BB6DC7F894307B689B68D3
S3150802DD00002B00F0FF817B68DB68FB67A34B1B686F
S3150802DD10BB677B68DB68BA6F9A420DD0A04B1B685B
S3150802DD20002B09D1D7F894307B657B6D83F3108875
S3150802DD3000BF1E23C7F88830D7F88830202B40F05A
S3150802DD40EB817B689B685A1E7B689A607B689B6836
S3150802DD50002B0AD0D7F894303B653B6D83F31088C5
S3150802DD6000BF0023C7F88830D6E1FB6F002B0AD123
S3150802DD70D7F89430FB64FB6C83F3108800BF00234A
S3150802DD80C7F88830C8E1FB6FD3F8A0305A1EFB6F7C
S3150802DD90C3F8A020FB6FD3F8A030002B04D1FB6F89
S3150802DDA00022C3F8A42019E07B68DB6AC7F884302E
S3150802DDB07B681B6B7B67D7F884307A6F1A637B6F35
S3150802DDC0D7F88420DA62FB6FD3F8A4307A689A42CD
S3150802DDD004D1FB6FD7F88420C3F8A4207B689B691B
S3150802DDE0002B10D17B681B69002B0CD17B680022A3
S3150802DDF0DA60D7F89430BB64BB6C83F3108800BF33
S3150802DE000023C7F88830D7F88830202B40F0848161
S3150802DE100023C7F89030FB6FD3F89430C7F88C30DC
S3150802DE207B681B69012B55D15D4B1B6801335C4A24
S3150802DE301360D7F894307B647B6C83F3108800BF39
S3150802DE402023C7F88030FB6FD3F8A430C7F8843094
S3150802DE501FE0D7F884301B69012B0BD1D7F8843021
S3150802DE609B6AD7F880209A4204D9D7F884309B6AED
S3150802DE70C7F88030D7F88430DB6AC7F88430FB6F7E
S3150802DE80D3F8A430D7F884209A4202D10023C7F8DF
S3150802DE908430D7F88430002BDBD1EFF310833B6450
S3150802DEA03B6CFB6372B6FB6BC7F894303C4B1B6842
S3150802DEB0013B3B4A1360FB6FD7F88020C3F89C20CE
S3150802DEC0D7F88020D7F88C309A4203D2D7F8803018
S3150802DED0C7F88C307B68DB69012B20D97B681B6904
S3150802DEE0012B1CD12E4B1B6801332D4A1360D7F820
S3150802DEF094303B633B6B83F3108800BF7868FFF767
S3150802DF007DFDEFF31083BB63BB6B7B6372B67B6BE2
S3150802DF10C7F89430224B1B68013B214A13607B6881
S3150802DF209B69002B3ED11E4B1B6801331C4A1360AA
S3150802DF30D7F89430FB62FB6A83F3108800BF7B68CC
S3150802DF4020229A627B68DB68DB6AD7F88C209A42C1
S3150802DF5006D07B68DB68D7F88C101846FFF700FEF8
S3150802DF60EFF310837B627B6A3B6272B63B6AC7F841
S3150802DF7094300B4B1B68013B094A13607B680022ED
S3150802DF80DA60D7F89430BB62BB6A83F3108800BFA5
S3150802DF9000F0C8FA0023C7F88830BDE0F014002064
S3150802DFA0881500207B689B69FB677B681B69012BC8
S3150802DFB00AD17B68DB68C7F89030FB6FDA6A7B6840
S3150802DFC05A617B6820229A62FB6FD3F8A0303B67BE
S3150802DFD03B6F002B0AD1FB6F7A68C3F8A4207B68D3
S3150802DFE07A68DA627B687A681A6316E0FB6FD3F896
S3150802DFF0A430C7F88430D7F884301B6B7B67D7F810
S3150802E00084307A681A637B6F7A68DA627B687A6F19
S3150802E0101A637B68D7F88420DA623B6F5A1CFB6F57
S3150802E020C3F8A0207B6801229A607B68FA6FDA60DF
S3150802E0307B68DB695A1E7B68DA617B68DB69FB668B
S3150802E040FB6E002B03D17B6800229A610EE0FB6F00
S3150802E0501B6FBB667B68BA6E9A61FB6F5B6F7B66EA
S3150802E060BB6E7A6E5A677B6EBA6E1A67FB6F0022B0
S3150802E0709A66FB6F0022C3F884202A4B1B68013379
S3150802E080284A1360D7F89430FB61FB6983F310883A
S3150802E09000BF7B681B69012B2DD17B68DB69002BCE
S3150802E0A01CD07868FFF7AAFCEFF31083BB61BB6943
S3150802E0B07B6172B67B69C7F894307B689B693B665D
S3150802E0C03B6E002B03D03B6EDA6A7B689A62D7F8FE
S3150802E0D094303B613B6983F3108800BFD7F89030D0
S3150802E0E0DB6AD7F88C209A4205D0D7F88C10D7F875
S3150802E0F09000FFF735FDF86F00F04EFA0023C7F8D7
S3150802E100883009E0D7F89430FB60FB6883F31088FF
S3150802E11000BF1E23C7F88830D7F8883018469837C4
S3150802E120BD4680BD8815002080B592B000AFF86064
S3150802E130B9607A603B6000233B647A6DEF21386DE3
S3150802E14047F090FFB0220021F86847F08BFFFB6882
S3150802E150BA689A62FB687A685A64FB683A689A648B
S3150802E160FB683A6DDA60FB687A6D5A61FB68BA6DCC
S3150802E170DA62FB68BA6DC3F89420FB683A6E9A6154
S3150802E180FB683A6EDA61FB682022C3F89C203B6D75
S3150802E190FB637B6D013BFA6B1344FB63FB68FA6B0B
S3150802E1A01A61BA6DFB6D9A4207D0FB680022DA63E0
S3150802E1B0FB680022C3F8982006E0FB68BA6DDA63AA
S3150802E1C0FB68BA6DC3F89820FB6803221A63FB68DA
S3150802E1D0484A5A65FA68FB689A654749F868F2F741
S3150802E1E0C3F8EFF31083FB62FB6ABB6272B6BB6AC3
S3150802E1F0BB63FB68414A1A60414B1B68002B0BD173
S3150802E200404AFB681360FB68FA68C3F88820FB6813
S3150802E210FA68C3F88C2016E03A4B1B687B637B6B63
S3150802E220D3F88C303B637B6BFA68C3F88C203B6B64
S3150802E230FA68C3F88820FB683A6BC3F88C20FB6837
S3150802E2407A6BC3F888202E4B1B6801332C4A13605D
S3150802E2502D4B1B6801332C4A13607B6E012B29D187
S3150802E260EFF305837B627A6A284B1B681343B3F183
S3150802E270F03F0DD3264B1B687B647B6C002B09D0C1
S3150802E2807B6CDB6B3B647B6CDA6A7B6CDA6301E082
S3150802E29000237B64BB6B3B623B6A83F3108800BF37
S3150802E2A0F86800F079F97B6C002B1ED07B6C3A6C0F
S3150802E2B0DA631AE0BB6B3B613B6983F3108800BFE4
S3150802E2C0EFF31083BB61BB697B6172B67B69BB6383
S3150802E2D00D4B1B68013B0C4A1360BB6BFB61FB6968
S3150802E2E083F3108800BF00F01DF90023184648374B
S3150802E2F0BD4680BD6DEA02088DE3020844524854C1
S3150802E300FC140020F81400208815002024000020A0
S3150802E310F414002080B500AF124B00221A60124B8B
S3150802E32000221A60114B00221A60114B20221A6031
S3150802E330802200210F4847F095FE0F4B00221A60F3
S3150802E3400E4B00221A600E4B00221A600D4B002259
S3150802E3501A600D4B1B6843F085730B4A136000BFA6
S3150802E36080BD00BFF0140020F41400200015002020
S3150802E3700415002008150020F8140020FC140020BB
S3150802E380881500208C1500209015002080B588B0CD
S3150802E39000AF214B1B68FB61FB695B6CFA69926CE7
S3150802E3A0104698471D4B1B68002B03D01B4B1B6856
S3150802E3B0F8699847EFF310837B607B683B6072B617
S3150802E3C03B68BB61FB6901221A63FB6901229A63F6
S3150802E3D0FB690022DA64124B1B680133104A136088
S3150802E3E0BB69BB60BB6883F3108800BFEFF3148375
S3150802E3F0FB60FB687B617B6923F004037B617B69B5
S3150802E4003B613B6983F3148800BFF86900F0C4F9DD
S3150802E41000BF2037BD4680BDF01400208C150020B1
S3150802E4208815002080B58EB000AF7860EFF31083B0
S3150802E430BB62BB6A7B6272B67B6A3B63354B1B68FF
S3150802E440FB62FB6A002B08D13B6B3B623B6A83F398
S3150802E450108800BF13237B6356E0EFF30583FB6145
S3150802E460FA692D4B1B681343002B08D03B6BBB6123
S3150802E470BB6983F3108800BF13237B6344E0FB6AFE
S3150802E480264A934208D13B6B7B617B6983F31088EA
S3150802E49000BF13237B6337E07B68002B08D13B6BF5
S3150802E4A03B613B6983F3108800BF00237B632BE043
S3150802E4B01B4B1B68002B08D03B6BFB60FB6883F386
S3150802E4C0108800BF13237B631EE0FB6A04221A63CB
S3150802E4D0FB6A01229A63FB6A0022C3F88420FB6A5C
S3150802E4E07A68DA640E4B1B6801330D4A13603B6B7C
S3150802E4F0BB60BB6883F3108800BFF86A00F04CF96A
S3150802E500FB6AD3F884307B637B6B18463837BD4683
S3150802E51080BD00BFF0140020240000203816002019
S3150802E5208815002080B489B000AF174B1B68FB61C1
S3150802E530FB69002B21D1154B1B68BB61144B1B6869
S3150802E5407B61BA697B699A4217D0124B4FF08052A7
S3150802E5501A60EFF305833B613B69002B0CD1EFF39D
S3150802E5601083FB60FB68BB6062B600BFBB687B605A
S3150802E5707B6883F3108800BF00BF00BF2437BD46FF
S3150802E5805DF8047B704700BF88150020F014002050
S3150802E590F414002004ED00E080B596B000AF786070
S3150802E5A0EFF310837B637B6B3B6372B63B6B7B65D6
S3150802E5B07B685B6E002B05D07B684C33184600F0EF
S3150802E5C091FB02E07B680022DA646C4B1B68013B14
S3150802E5D06A4A13607B689B6B002B40F083807B68DA
S3150802E5E01B6B002B00F097807B685B6B002B72D14C
S3150802E5F07B6800221A637B68DB6A3B65604A3B6D6F
S3150802E60052F82330FB64FB6C002B54D15C493B6DFA
S3150802E6107A6841F823207B687A681A627B687A6886
S3150802E6205A6201223B6D02FA03F37B64554B1A6860
S3150802E6307B6C1343534A1360534B1B683A6D9A42D9
S3150802E64069D2514A3B6D1360504B1B683B643B6C65
S3150802E650002B03D14D4A7B6813605CE03B6CDB6B95
S3150802E6603A6D9A4257D2494A7B6813607B6DFB62C0
S3150802E670FB6A83F3108800BF404B1B68FB63FB6B86
S3150802E680002B74D1424B4FF080521A60EFF3058388
S3150802E690BB62BB6A002B0CD1EFF310837B627B6AE9
S3150802E6A03B6262B600BF3B6AFB61FB6983F3108873
S3150802E6B000BF00BF5BE0FB6C5B6ABB64BB6C7A683D
S3150802E6C01A62FB6C7A685A627B68BA6C5A627B6811
S3150802E6D0FA6C1A621FE07B6800225A637B6803227F
S3150802E6E01A6318E07B681B6B012B14D07B681B6BC3
S3150802E6F0022B10D07B685B6B002B06D17B6800224D
S3150802E7009A637B6800221A6305E07B6800225A63D3
S3150802E7107B6803221A631F4B1B68BB637B6DBB6155
S3150802E720BB6983F3108800BF184B1B68BA6B9A4201
S3150802E73020D0124B1B68FB63FB6B002B1AD1144BC0
S3150802E7404FF080521A60EFF305837B617B69002BD9
S3150802E7500FD1EFF310833B613B69FB6062B600BFE2
S3150802E760FB68BB60BB6883F3108800BF01E000BF8B
S3150802E77000E000BF5837BD4680BD00BF881500209F
S3150802E780081500200015002004150020F4140020A6
S3150802E79004ED00E0F014002080B59EB000AF78606A
S3150802E7A0814B1B687B67EFF31083FB64FB6CBB64CE
S3150802E7B072B6BB6C3B677A687B6F9A4212D17B68EA
S3150802E7C0DB6CFB66FB6E002B08D0FB6EB3F1FF3FDA
S3150802E7D004D07B684C33184600F022FA7B68DB6962
S3150802E7E0724A1360724B1B68013B714A13607B685D
S3150802E7F09B6B012B40F0A6807B6800229A637B689C
S3150802E800DB6ABB667B681B6A7B667A6E7B689A42A2
S3150802E81015D07B685B6A3B657B6E3A6D5A623B6DC7
S3150802E8207A6E1A62634ABB6E52F823307A689A4243
S3150802E83057D16049BB6E7A6E41F8232051E05D4A92
S3150802E840BB6E002142F823100122BB6E02FA03F3C3
S3150802E8503B66594B1A683B6EDB431340564A1360B4
S3150802E8600023FB65544B1B68BB65BB6D002B2BD184
S3150802E870524B20221A60524B00221A603B6F7B646D
S3150802E8807B6C83F3108800BF494B1B687B657B6DE5
S3150802E890002B40F081804B4B4FF080521A60EFF309
S3150802E8A005833B643B6C002B0CD1EFF31083FB63AF
S3150802E8B0FB6BBB6362B600BFBB6B7B637B6B83F38D
S3150802E8C0108800BF00BF67E0BB6D93FAA3F3BB6570
S3150802E8D0BB6DB3FA83F33B66FA6D3B6E1344374A54
S3150802E8E01360374B1B687A689A422BD1334B1B68E5
S3150802E8F0304A52F82330324A13603B6F3B633B6B14
S3150802E90083F3108800BF2A4B1B687B657B6D002B3F
S3150802E91044D12C4B4FF080521A60EFF30583FB6209
S3150802E920FB6A002B0CD1EFF31083BB62BB6A7B62D6
S3150802E93062B600BF7B6A3B623B6A83F3108800BFFC
S3150802E94000BF2BE03B6FFB61FB6983F3108800BFB6
S3150802E9501B4B1B687A6F9A4222D0154B1B687B6544
S3150802E9607B6D002B1CD1174B4FF080521A60EFF3C8
S3150802E9700583BB61BB69002B0CD1EFF310837B6166
S3150802E9807B693B6162B600BF3B69FB60FB6883F348
S3150802E990108800BF00BF03E000BF02E000BF00E02E
S3150802E9A000BF7837BD4680BDF0140020F41A002057
S3150802E9B088150020081500200015002004150020DF
S3150802E9C0F414002004ED00E080B487B000AF214BB8
S3150802E9D01B687B61EFF31083FB60FB68BB6072B652
S3150802E9E0BB683B611C4B00221A607B69002B24D052
S3150802E9F07B691B6B002B20D17B69DA697B699A617B
S3150802EA007B699B69154A13607B691B6A7A699A4214
S3150802EA1013D07B69DA6A7B69DB6B9A420DD17B6913
S3150802EA20DB6A7A69126A0E4941F823200D4B1B6884
S3150802EA300B4A52F823300C4A13603B697B607B68A9
S3150802EA4083F3108800BF00BF1C37BD465DF8047B00
S3150802EA50704700BFF014002098150020F41A002011
S3150802EA600815002004150020F414002080B58AB089
S3150802EA7000AF78607B687B62EFF310837B617B690A
S3150802EA803B6172B63B693B627B6A1B6B042B0ED1F8
S3150802EA90134B1B680133124A13603B6AFB60FB681F
S3150802EAA083F3108800BF786AFFF776FD13E07B6A66
S3150802EAB09B6EFB617B6AD3F8AC30BB613B6ABB6079
S3150802EAC0BB6883F3108800BFFB69002B03D0FB6980
S3150802EAD0B969786A984700BF2837BD4680BD00BF26
S3150802EAE08815002080B584B000AFEFF310837B60F1
S3150802EAF07B683B6072B63B68FB60094B1B68013357
S3150802EB00074A1360FB68BB60BB6883F3108800BFC3
S3150802EB100448FFF741FD00BF1037BD4680BD00BF60
S3150802EB20881500203816002090B589B006AF284B04
S3150802EB3000221A60274B00221A60274B00221A600D
S3150802EB40264B00221A60264B00221A6080220021D8
S3150802EB50244847F087FA244B224A1A60234B214A53
S3150802EB601A60234B234A1A60214B1B680433204A36
S3150802EB701360214B214A1A60214B4FF480621A60B6
S3150802EB80204B00221A601C4B1B681D4A12681D493D
S3150802EB9009681C480068002405940024049403901C
S3150802EBA0029101920093184B184A19491948FFF71E
S3150802EBB0BBFA78607B68002BE5D1174B00221A60F6
S3150802EBC0164B00221A6000BF0C37BD4690BD00BF27
S3150802EBD094150020F41A0020981500202816002003
S3150802EBE0341600209C1500201C160020241600202E
S3150802EBF02016002018160020E8160020F416002019
S3150802EC00EC160020F01600204D49544155ED020835
S3150802EC1010960708381600202C16002030160020F9
S3150802EC2080B489B000AF78607B681B687B617B69BA
S3150802EC30002B4AD07B69B3F1FF3F46D07B689B69BC
S3150802EC40002B42D17B69202B02D91F23BB6102E02C
S3150802EC507B69013BBB61204B1A68BB699B00134465
S3150802EC60FB611E4B1B68FA699A420BD31B4B1B6846
S3150802EC70FA69D31A9B103B61194B1A683B699B00C8
S3150802EC801344FB61FB691B68002B09D17B687A6810
S3150802EC901A617B687A685A61FB697A681A6011E0B8
S3150802ECA0FB691B68FB60FB685B69BB60BB687A68CB
S3150802ECB01A61FB687A685A617B68FA681A617B6826
S3150802ECC0BA685A617B68FA699A6100BF2437BD46F9
S3150802ECD05DF8047B704700BF24160020201600202A
S3150802ECE01C16002080B487B000AF78607B689B69E9
S3150802ECF07B617B69002B26D07B681B693B617A683E
S3150802ED003B699A4208D17B691B687A689A4217D18D
S3150802ED107B6900221A6013E07B685B69FB603B69CA
S3150802ED20FA685A61FB683A691A617B691B687A68EC
S3150802ED309A4205D13B697A699A617B693A691A608E
S3150802ED407B6800229A6100BF1C37BD465DF8047BCA
S3150802ED507047000080B598B000AF786000237B65E5
S3150802ED607B68734A934240F0DE80EFF310833B647C
S3150802ED703B6CFB6372B6FB6BFB656E4B1B681B68D1
S3150802ED80FB60FB68002B03D0FB6807F10C029A6153
S3150802ED90684B1B6800221A60664B1B680433654A77
S3150802EDA01360644B1A68644B1B689A4203D1634B1F
S3150802EDB01B68604A1360624B00221A60FB6D3B6354
S3150802EDC03B6B83F3108800BFEFF31083BB63BB6B07
S3150802EDD07B6372B67B6BFB657FE0FB68FB64FB6853
S3150802EDE01B69BB640023BB60FA6CBB6C9A4202D1F6
S3150802EDF00023FB600EE0FB6C5B697B64BB6C7A6C80
S3150802EE005A617B6CBA6C1A61BB6C07F10C029A6187
S3150802EE10BB6CFB60FB6C1B68202B11D9FB6C1B6857
S3150802EE20A3F12002FB6C1A600023BB65FB6C07F199
S3150802EE3008029A61FB6CFA6C1A61FB6CBB601AE0F9
S3150802EE40FB6C9B68BB65FB6CDB687B65FB6C5A6875
S3150802EE50FB6C1A60FB6C1B68002B09D0FB6C07F174
S3150802EE6008029A61FB6CFA6C1A61FB6CBB6002E0E1
S3150802EE70FB6C00229A61334AFB6C1360FB6DFB62E2
S3150802EE80FB6A83F3108800BFBB6D002B02D0BB6DF3
S3150802EE90786D9847EFF31083BB62BB6A7B6272B6E2
S3150802EEA07B6AFB65274B00221A60BB68FA6C9A429A
S3150802EEB005D1FB6C00229A61F86CFFF7B1FEFB6D77
S3150802EEC0BB61BB6983F3108800BFEFF310833B6213
S3150802EED03B6AFB6172B6FB69FB65FB68002B7FF434
S3150802EEE07CAF174B1B68002B16D1174B3B653B6D46
S3150802EEF003221A633B6D01229A63144B1B68013382
S3150802EF00124A1360FB6D7B617B6983F3108800BF2D
S3150802EF10386DFFF741FC28E7FB6D3B613B6983F3DC
S3150802EF20108800BF21E700BF6037BD4680BD00BF1D
S3150802EF304D49544124160020201600201C16002094
S3150802EF4028160020341600203816002088150020BE
S3150802EF5080B58AB000AFF860B9607A603B6000237A
S3150802EF607B62FB68002B02D102237B6229E0FB68E5
S3150802EF701B682D4A934202D002237B6221E0BB68BA
S3150802EF80002B02D103237B621BE07B68002B02D194
S3150802EF9005237B6215E0FB68DB697A689A4202D927
S3150802EFA005237B620DE03B68002B0AD0EFF305834D
S3150802EFB0FB61FA691D4B1B681343002B01D004231E
S3150802EFC07B627B6A002B08D1194B1B683B623B6A42
S3150802EFD0184A934201D113237B627B6A002B14D110
S3150802EFE0EFF30583BB61BA69104B1B681343002B09
S3150802EFF00BD0EFF305837B617A690C4B1B681343CD
S3150802F000B3F1F03F01D213237B627B6A002B06D150
S3150802F0103B687A68B968F868FDF77AFF78627B6AAE
S3150802F02018462837BD4680BD45545942240000205B
S3150802F030F01400203816002080B592B000AFF860B0
S3150802F040B9607A603B6000237B64FB68002B02D1BF
S3150802F05002237B6475E03B6D342B02D002237B646A
S3150802F0606FE0EFF31083FB62FB6ABB6272B6BB6AA0
S3150802F070BB633B4B1B680133394A1360BB6B3B636B
S3150802F0803B6B83F3108800BF364B1B68FB63002378
S3150802F0903B6409E0FA68FB6B9A420BD0FB6BDB6AAE
S3150802F0A0FB633B6C01333B642F4B1B683A6C9A42F9
S3150802F0B0F0D300E000BFEFF310833B623B6AFB61CB
S3150802F0C072B6FB69BB63264B1B68013B244A136075
S3150802F0D0BB6B7B627B6A83F3108800BFFFF722FA59
S3150802F0E0FA68FB6B9A4202D102237B6429E07B68A9
S3150802F0F0002B02D103237B6423E03B68632B02D8EF
S3150802F10005237B641DE0194B1B687B637B6B184ADE
S3150802F110934201D113237B64EFF30583BB61BA697A
S3150802F120144B1B681343002B0BD0EFF305837B614B
S3150802F1307A69104B1B681343B3F1F03F01D21323CC
S3150802F1407B647B6C002B06D13B687A68B968F868E1
S3150802F150FEF720F878647B6C18464837BD4680BDB2
S3150802F16088150020E0140020E4140020F014002082
S3150802F170381600202400002080B592B000AFF8604F
S3150802F180B9607A603B6000237B64FB68002B02D17E
S3150802F1901C237B6453E03B68342B02D01C237B641C
S3150802F1A04DE0EFF31083FB62FB6ABB6272B6BB6A81
S3150802F1B0BB633A4B1B680133384A1360BB6B3B632C
S3150802F1C03B6B83F3108800BF354B1B68FB63002338
S3150802F1D03B6409E0FA68FB6B9A420BD0FB6B1B6A2D
S3150802F1E0FB633B6C01333B642E4B1B683A6C9A42B9
S3150802F1F0F0D300E000BFEFF310833B623B6AFB618A
S3150802F20072B6FB69BB63254B1B68013B234A136035
S3150802F210BB6B7B627B6A83F3108800BFFFF782F9B8
S3150802F220FA68FB6B9A4202D11C237B6407E07B686F
S3150802F230012B04D07B68002B01D01F237B647B6CD7
S3150802F240002B1DD1184B1B687B637B6B174A9342B5
S3150802F25001D113237B64EFF30583BB61BA69144BAF
S3150802F2601B681343002B0BD0EFF305837B617A6986
S3150802F2700F4B1B681343B3F1F03F01D213237B6490
S3150802F2807B6C002B05D17A68B968F868FEF754FAE0
S3150802F29078647B6C18464837BD4680BD88150020C1
S3150802F2A0D0140020D4140020F014002038160020B0
S3150802F2B02400002080B588B000AF7860396000234A
S3150802F2C0FB617B68002B02D11C23FB611FE07B6874
S3150802F2D01B68214A934202D01C23FB6117E03B6854
S3150802F2E0002B14D0EFF305837B617A691B4B1B68ED
S3150802F2F01343002B02D00423FB6108E0184B1B685A
S3150802F300BB61BB69174A934201D10423FB61FB69BE
S3150802F310002B14D1EFF305833B613A690F4B1B6847
S3150802F3201343002B0BD0EFF30583FB60FA680B4BF4
S3150802F3301B681343B3F1F03F01D21323FB61FB6948
S3150802F340002B04D139687868FEF750FAF861FB6930
S3150802F35018462037BD4680BD4554554D2400002029
S3150802F360F01400203816002080B586B000AF786009
S3150802F37000237B617B68002B02D11C237B611CE086
S3150802F3807B681B68134A934202D01C237B6114E0F4
S3150802F390EFF305833B613A690F4B1B681343002B56
S3150802F3A00BD0EFF30583FB60FA680B4B1B6813431C
S3150802F3B0B3F1F03F01D213237B617B69002B03D1A2
S3150802F3C07868FEF78BFC78617B6918461837BD4664
S3150802F3D080BD00BF4554554D2400002080B59AB023
S3150802F3E006AFF860B9607A603B600023FB64FB688D
S3150802F3F0002B02D10E23FB64BBE03B6FB02B02D07D
S3150802F4000E23FB64B5E0EFF31083BB62BB6A7B6233
S3150802F41072B67B6AFB63644B1B680133624A1360EC
S3150802F420FB6BFB62FB6A83F3108800BF0023BB6495
S3150802F4305E4B1B683B64BB6DBB63FB6D013BBA6BE2
S3150802F4401344BB63BB6B7B6300237B642BE0FA68C4
S3150802F4503B6C9A4201D10123BB64BB6C012B28D0B9
S3150802F4603B6CDB68BA6D9A4208D33B6C1B69BA6D72
S3150802F4709A4203D20023BB650123BB643B6CDB685B
S3150802F4807A6B9A4208D33B6C1B697A6B9A4203D20F
S3150802F4900023BB650123BB643B6CD3F888303B640D
S3150802F4A07B6C01337B64424B1B687A6C9A42CED3DF
S3150802F4B000E000BFEFF31083FB61FB69BB6172B624
S3150802F4C0BB69FB63384B1B68013B374A1360FB6B0E
S3150802F4D03B623B6A83F3108800BFFFF723F8FA689A
S3150802F4E03B6C9A4202D10E23FB6442E0BB6D002BB1
S3150802F4F002D10323FB643CE07B68002B02D1032381
S3150802F500FB6436E0FB6DC72B02D80523FB6430E0AB
S3150802F5103B6E1F2B02D90F23FB642AE07A6E3B6EE1
S3150802F5209A4202D91823FB6423E0FB6E012B02D907
S3150802F5301023FB641DE01F4B1B683B633B6B1E4A93
S3150802F540934201D11323FB64EFF305837B617A6946
S3150802F5501A4B1B681343002B0BD0EFF305833B6151
S3150802F5603A69164B1B681343B3F1F03F01D21323D2
S3150802F570FB64FB6C002B12D1FB6E0593BB6E0493E6
S3150802F5807B6E03933B6E0293FB6D0193BB6D0093F7
S3150802F5903B687A68B968F868FEF7C6FDF864FB6CDA
S3150802F5A018465037BD4680BD88150020F81400203D
S3150802F5B0FC140020F0140020381600202400002035
S3150802F5C080B483B000AF03460A46FB711346BB807C
S3150802F5D0FB79002B0AD1164B1B6800225A62144B80
S3150802F5E01B685A6ABB889A42F9D31AE0FB79012B3F
S3150802F5F00AD1104B1B6800225A620E4B1B685A6AC4
S3150802F600BB889A42F9D30CE0FB79022B09D10A4B43
S3150802F6101B6800225A62084B1B685A6ABB889A42C0
S3150802F620F9D300BF0C37BD465DF8047B704700BFAF
S3150802F630C4800220108102205C81022080B582B03B
S3150802F64000AF0346FB71FB79002B06D101224FF46A
S3150802F65000610D48F3F73AFC11E0FB79012B05D15D
S3150802F660012210210948F3F731FC08E0FB79022B45
S3150802F67005D101224FF480710548F3F727FC00BF34
S3150802F6800837BD4680BD00BF000C02420008024290
S3150802F6900014024280B582B000AF0346FB71FB79C3
S3150802F6A0002B06D100224FF400610D48F3F70EFC39
S3150802F6B011E0FB79012B05D1002210210948F3F745
S3150802F6C005FC08E0FB79022B05D100224FF4807174
S3150802F6D00548F3F7FBFB00BF0837BD4680BD00BFF0
S3150802F6E0000C0242000802420014024280B582B0AF
S3150802F6F000AF0346FB71FB79002B06D101224FF4BA
S3150802F70080610C48F3F7E2FB10E0FB79012B05D187
S3150802F710012220210848F3F7D9FB07E0FB79022BDF
S3150802F72004D1012280210548F3F7D0FB00BF083730
S3150802F730BD4680BD000C024200000242001402428D
S3150802F74080B582B000AF0346FB71FB79002B06D168
S3150802F75000224FF480610C48F3F7B8FB10E0FB79FE
S3150802F760012B05D1002220210848F3F7AFFB07E059
S3150802F770FB79022B04D1002280210548F3F7A6FB68
S3150802F78000BF0837BD4680BD000C02420000024297
S3150802F7900014024280B582B000AF0346FB71FB79C2
S3150802F7A0002B04D100210B48F9F79EFE0EE0FB79E7
S3150802F7B0012B04D104210748F9F796FE06E0FB79E6
S3150802F7C0022B03D108210348F9F78EFE00BF08373A
S3150802F7D0BD4680BD2C80022080B483B000AF0346AC
S3150802F7E00A46FB711346BB71FB79002B04D10D4BFC
S3150802F7F01B68BA795A630EE0FB79012B04D1094BCF
S3150802F8001B68BA799A6306E0FB79022B03D1054B8A
S3150802F8101B68BA79DA6300BF0C37BD465DF8047B0C
S3150802F820704700BF2C80022080B582B000AF034625
S3150802F830FB71FB79002B06D101224FF400710C48AB
S3150802F840F3F744FB10E0FB79012B05D101221021C5
S3150802F8500848F3F73BFB07E0FB79022B04D10122A8
S3150802F86004210548F3F732FB00BF0837BD4680BDC1
S3150802F870000C0242000002420014024280B582B025
S3150802F88000AF0346FB71FB79002B06D100224FF429
S3150802F89000710C48F3F71AFB10E0FB79012B05D12E
S3150802F8A0002210210848F3F711FB07E0FB79022B27
S3150802F8B004D1002204210548F3F708FB00BF0837E4
S3150802F8C0BD4680BD000C02420000024200140242FC
S3150802F8D080B582B000AF0346FB71FB79002B06D1D7
S3150802F8E001224FF480710C48F3F7F0FA10E0FB7925
S3150802F8F0012B05D1012204210848F3F7E7FA07E0AC
S3150802F900FB79022B04D1012202210548F3F7DEFA1C
S3150802F91000BF0837BD4680BD000C024200080242FD
S3150802F9200014024280B582B000AF0346FB71FB7930
S3150802F930002B06D100224FF480710C48F3F7C6FA61
S3150802F94010E0FB79012B05D1002204210848F3F7C0
S3150802F950BDFA07E0FB79022B04D1002202210548F1
S3150802F960F3F7B4FA00BF0837BD4680BD000C024261
S3150802F970000802420014024280B582B000AF034674
S3150802F980FB71FB79002B04D100210B48F9F7ACFD7A
S3150802F9900EE0FB79012B04D104210748F9F7A4FDEF
S3150802F9A006E0FB79022B03D108210348F9F79CFDEF
S3150802F9B000BF0837BD4680BD7880022080B483B078
S3150802F9C000AF03460A46FB711346BB71FB79002B4F
S3150802F9D004D10D4B1B68BA795A630EE0FB79012BE9
S3150802F9E004D1094B1B68BA799A6306E0FB79022BA4
S3150802F9F003D1054B1B68BA79DA6300BF0C37BD46DB
S3150802FA005DF8047B704700BF7880022080B582B01B
S3150802FA1000AF0346FB71FB79002B06D100224FF497
S3150802FA2080510C48F3F752FA10E0FB79012B05D105
S3150802FA30002202210848F3F749FA07E0FB79022B6C
S3150802FA4004D1002201210348F3F740FA00BF083720
S3150802FA50BD4680BD001402420008024280B582B04B
S3150802FA6000AF0346FB71FB79002B06D101224FF446
S3150802FA7080510C48F3F72AFA10E0FB79012B05D1DD
S3150802FA80012202210848F3F721FA07E0FB79022B43
S3150802FA9004D1012201210348F3F718FA00BF0837F7
S3150802FAA0BD4680BD001402420008024280B582B0FB
S3150802FAB000AF0346FB71FB79002B05D10022042116
S3150802FAC00C48F3F703FA11E0FB79012B05D1002262
S3150802FAD020210948F3F7FAF908E0FB79022B05D148
S3150802FAE000224FF400710548F3F7F0F900BF083712
S3150802FAF0BD4680BD001802420008024200140242B6
S3150802FB0080B582B000AF0346FB71FB79002B05D1A5
S3150802FB10012204210C48F3F7D9F911E0FB79012BEC
S3150802FB2005D1012220210948F3F7D0F908E0FB792B
S3150802FB30022B05D101224FF400710548F3F7C6F9E5
S3150802FB4000BF0837BD4680BD0018024200080242BF
S3150802FB500014024280B582B000AF0346FB71FB79FE
S3150802FB60002B05D1002208210C48F3F7AFF911E062
S3150802FB70FB79012B06D100224FF400610848F3F7FE
S3150802FB80A5F907E0FB79022B04D1002201210548D9
S3150802FB90F3F79CF900BF0837BD4680BD001802423C
S3150802FBA0001402420008024280B582B000AF034642
S3150802FBB0FB71FB79002B05D1012208210C48F3F7CA
S3150802FBC085F911E0FB79012B06D101224FF4006178
S3150802FBD00848F3F77BF907E0FB79022B04D10122E7
S3150802FBE001210548F3F772F900BF0837BD4680BD03
S3150802FBF000180242001402420008024280B582B08E
S3150802FC0000AF0346FB71FB79002B04D100210B4898
S3150802FC10F9F76AFC0EE0FB79012B04D104210748A7
S3150802FC20F9F762FC06E0FB79022B03D108210348A7
S3150802FC30F9F75AFC00BF0837BD4680BDE07F0220AF
S3150802FC4080B483B000AF03460A46FB711346BB7104
S3150802FC50FB79002B04D10D4B1B68BA795A630EE067
S3150802FC60FB79012B04D1094B1B68BA799A6306E022
S3150802FC70FB79022B03D1054B1B68BA79DA6300BFFD
S3150802FC800C37BD465DF8047B704700BFE07F022053
S3150802FC9080B582B000AF0346FB71FB79002B0BD10E
S3150802FCA04FF400511648F3F7F9F80346012B14BF2F
S3150802FCB001230023DBB21EE0FB79012B0BD14FF4A3
S3150802FCC080610F48F3F7EAF80346012B14BF0123B4
S3150802FCD00023DBB20FE0FB79022B0BD14FF4004174
S3150802FCE00848F3F7DBF80346012B14BF0123002368
S3150802FCF0DBB200E0002318460837BD4680BD00BFC8
S3150802FD00001002420014024280B582B000AF0346D8
S3150802FD10FB71FB79002B0AD140211648F3F7BEF88E
S3150802FD200346012B14BF01230023DBB21DE0FB7936
S3150802FD30012B0BD14FF480510F48F3F7AFF8034666
S3150802FD40012B14BF01230023DBB20EE0FB79022B41
S3150802FD500AD140210948F3F7A1F80346012B14BF3B
S3150802FD6001230023DBB200E0002318460837BD460C
S3150802FD7080BD00BF000C0242001802420004024283
S3150802FD8080B582B000AF0346FB71FB79002B0AD11E
S3150802FD9080211648F3F782F80346012B14BF012384
S3150802FDA00023DBB21DE0FB79012B0BD14FF4005186
S3150802FDB00F48F3F773F80346012B14BF01230023F8
S3150802FDC0DBB20EE0FB79022B0AD180210948F3F750
S3150802FDD065F80346012B14BF01230023DBB200E0BA
S3150802FDE0002318460837BD4680BD00BF000C0242F4
S3150802FDF0001802420004024280B582B000AF0346F0
S3150802FE00FB71FB79002B0AD180211648F3F746F8D5
S3150802FE100346012B14BF01230023DBB21DE0FB7945
S3150802FE20012B0BD14FF480710E48F3F737F80346CE
S3150802FE30012B14BF01230023DBB20EE0FB79022B50
S3150802FE400AD180210848F3F729F80346012B14BF83
S3150802FE5001230023DBB200E0002318460837BD461B
S3150802FE6080BD00BF001802420008024280B582B077
S3150802FE7000AF0346FB71FB79002B0BD14FF480715F
S3150802FE801648F3F70BF80346012B0CBF0123002390
S3150802FE90DBB21EE0FB79012B0BD14FF400710F4840
S3150802FEA0F2F7FCFF0346012B0CBF01230023DBB24A
S3150802FEB00FE0FB79022B0BD14FF480710848F2F759
S3150802FEC0EDFF0346012B0CBF01230023DBB200E042
S3150802FED0002318460837BD4680BD00BF0008024207
S3150802FEE00000024280B582B000AF78607B681A686B
S3150802FEF07B689B8819461046F2F7D0FF0346002B0B
S3150802FF0001D0012300E0002318460837BD4680BD0C
S3150802FF1080B582B000AF78600B46FB70FB78002B89
S3150802FF2008D07B6898687B689B8901221946F2F794
S3150802FF30CDFF07E07B6898687B689B890022194693
S3150802FF40F2F7C4FF00BF0837BD4680BD80B584B04E
S3150802FF5000AFF860B9603B601346FB80FB68BA687D
S3150802FF601A60FB68FA889A80FB683A689A60FB68A6
S3150802FF703A8B9A81FB68FA691A613B6A07EE903AEC
S3150802FF80B8EEE77ADFED0C6AC7EE267AFB68C3EDB0
S3150802FF90057AFB6802221A760121F868FFF7B8FF8C
S3150802FFA06420FEF73FFA0021F868FFF7B1FF00BFA9
S3150802FFB01037BD4680BD00BF0000484380B588B0F3
S3150802FFC000AF78600023FB610023FB760023FB74F5
S3150802FFD000237B6107E0FB695A1CFA61224A9342B5
S3150802FFE001D900233CE07868FFF77CFF0346002B23
S3150802FFF0F1D10120F0F74CF9F8600023FB761BE0FB
S3150803000001217868FFF784FF7B695B007B61002128
S315080300107868FFF77DFF7868FFF764FF0346FB748C
S31508030020FB7C002B02D07B6901337B6197F91B307C
S31508030030DBB20133DBB2FB7697F91B30172BDFDD17
S3150803004001217868FFF764FF7B6983F400037B610A
S3150803005000217868FFF75CFFF868F0F719F97B6900
S3150803006018462037BD4680BD40420F0080B584B090
S3150803007000AF78600B46FB700023FB600023FB721E
S315080300800023FB7209E07868FFF798FF0246FB68CE
S315080300901344FB60FB7A0133FB72FA7AFB789A42C4
S315080300A0F1D3FB78FA6892FBF3F318461037BD468B
S315080300B080BD80B483B000AF786039607B683A68E6
S315080300C01A6100BF0C37BD465DF8047B7047000014
S315080300D080B586B002AF78600023FB6034230093B3
S315080300E04FF400330B4A0C490C48FEF7A5FF0346A9
S315080300F0002B0AD1094BBB60B86803F043FEF860CE
S31508030100FB68002B01D000BFFDE700BF1037BD46D3
S3150803011080BD00BFF81A002024960708F81A0220A3
S3150803012080B582B000AF786020220021786845F058
S3150803013099FF7B68114A1A607B6800225A607B68BC
S3150803014000221A727B6803225A727B6800229A720B
S315080301507B680022DA727B6801221A737B680122A4
S315080301605A737B6801229A737B6803221A74786828
S3150803017000F06EF800BF0837BD4680BD3430424DE7
S3150803018080B588B000AFF860B9601346FB710023E9
S31508030190FB6100233B61BB687B617B69BB61002311
S315080301A0FB6110E0FA69FB68134418463EF0FAFA55
S315080301B003463B613A69BB691A60BB690433BB6191
S315080301C0FB690433FB61FB79FA699A42EADB01238B
S315080301D018462037BD4680BD80B58AB000AF786023
S315080301E020220021786845F03DFF07F10803202205
S315080301F00021184645F036FF07F108032022194661
S315080302000F48FFF7BDFFBB680E4A934207D07868CD
S31508030210FFF786FF10210C4825F0DAF90AE007F103
S31508030220080320221946786845F0D3FF0F210748AB
S3150803023025F0CEF9002318462837BD4680BD00BFF2
S3150803024000C01F083430424D389607084C960708F5
S3150803025090B589B000AF78600023FB617B68BB610A
S31508030260FE203EF0CEFA0023FB611FE007F10803E8
S3150803027010220021184645F0F5FEBB6907F108046C
S31508030280186859689A68DB680FC4FB6903F1016348
S3150803029003F57C2307F10802114618463EF096FA41
S315080302A0BB691033BB61FB691033FB61FB691F2B09
S315080302B0DCD9012318462437BD4690BD80B483B0E4
S315080302C000AF78607B685B6818460C37BD465DF8F7
S315080302D0047B704780B483B000AF786039607B686D
S315080302E03A685A6000BF0C37BD465DF8047B704711
S315080302F080B483B000AF78607B681B7A18460C37E6
S31508030300BD465DF8047B704780B483B000AF786060
S315080303100B46FB707B68FA781A7200BF0C37BD462A
S315080303205DF8047B704780B483B000AF78600B46F2
S31508030330FB70FB78042B04D8FB787A6813449B7A02
S3150803034000E0002318460C37BD465DF8047B70476A
S3150803035080B483B000AF78600B46FB701346BB705E
S31508030360FB78042B0DD8BB78002B05D0FB787A686D
S31508030370134401229A7204E0FB787A681344002234
S315080303809A7200BF0C37BD465DF8047B704780B48C
S3150803039083B000AF78607B68DB7B18460C37BD46B5
S315080303A05DF8047B704780B483B000AF78600B4672
S315080303B0FB707B68FA78DA7300BF0C37BD465DF8C5
S315080303C0047B704780B483B000AF78607B681B7C7E
S315080303D0FF2B02D07B681B7C00E0002318460C37F2
S315080303E0BD465DF8047B704780B483B000AF786080
S315080303F07B681B7C18460C37BD465DF8047B704743
S3150803040080B483B000AF78600B46FB707B68FA78DC
S315080304101A7400BF0C37BD465DF8047B704780B578
S3150803042082B000AF78607868FFF7CCFF034603F025
S315080304300103DBB2002B01D1002300E00123184698
S315080304400837BD4680BD80B582B000AF786078684E
S31508030450FFF7B8FF0346012B07D97868FFF7B2FF02
S315080304600346032B01D8012300E000231846083767
S31508030470BD4680BD80B483B000AF0346FB71FB79EC
S31508030480002B02D10A4B1B680CE0FB79012B02D126
S31508030490084B1B6806E0FB79022B02D1064B1B6847
S315080304A000E0002318460C37BD465DF8047B704709
S315080304B02C1B0220301B0220341B022080B483B07D
S315080304C000AF03463960FB71FB79002B03D10B4A56
S315080304D03B6813600CE0FB79012B03D1084A3B68A0
S315080304E0136005E0FB79022B02D1064A3B681360C9
S315080304F000BF0C37BD465DF8047B70472C1B0220F2
S31508030500301B0220341B022080B483B000AF03469D
S31508030510FB71044AFB79137000BF0C37BD465DF8BF
S31508030520047B70471931022080B400AF034B1B7854
S315080305301846BD465DF8047B704700BF1931022093
S3150803054080B586B000AFF8600B467A60FB7200236D
S31508030550FB752D4825F082F80023FB754CE0FB7DDF
S315080305602A4A4FF48E7101FB03F313441B78012BBC
S315080305703FD1FB7D4FF48E7202FB03F3234A1344E8
S3150803058002331946224825F069F8224825F066F809
S31508030590FB7D4FF48E7202FB03F318331B4A134495
S315080305A0043319461A4825F059F81B4825F056F816
S315080305B0FB7D164A4FF48E7101FB03F313449C33F8
S315080305C01B782D2B12D0154825F048F8FB7D4FF4E0
S315080305D08E7202FB03F398330C4A13440433194609
S315080305E00B4825F03BF80C4825F038F80A4825F05F
S315080305F035F8FB7D0133FB75FB7D0A2BAFD900BFAD
S3150803060000BF1837BD4680BD5C9607082800002042
S3150803061084960708889607088C960708909607080D
S3150803062080B584B000AFF8600B467A60FB7213F0AE
S3150803063031FA0346184613F065FA00BF1037BD466C
S3150803064080BD000080B586B000AFF8600B467A60BF
S31508030650FB7200237B617B6803F5007303224C4915
S31508030660184645F007FD0346002B22D17B6803F5A0
S3150803067000731846EFF730FF0346032B19D17B683F
S3150803068003F58063184644F0EAFB78617B69002B1F
S3150803069007D013F0FFF903460121184613F093FB1D
S315080306A071E013F0F7F903460121184613F0A8FB86
S315080306B069E07B6803F5007305223649184645F059
S315080306C0D9FC0346002B22D17B6803F50073184631
S315080306D0EFF702FF0346052B19D17B6803F5806301
S315080306E0184644F0BCFB78617B69002B07D013F0EE
S315080306F0D1F903460421184613F065FB43E013F0CA
S31508030700C9F903460421184613F07AFB3BE07B68D4
S3150803071003F5007303222049184645F0ABFC03464C
S31508030720002B30D17B6803F500731846EFF7D4FE28
S315080307300346032B27D17B6803F58063184644F0E9
S315080307408EFB78617B69002B0ED013F0A3F9034661
S315080307500121184613F037FB13F09CF903460421CD
S31508030760184613F030FB0EE013F094F90346012103
S31508030770184613F045FB13F08DF903460421184672
S3150803078013F03EFBFFE700BF1837BD4680BD00BF29
S315080307909C960708A0960708A896070880B584B00C
S315080307A000AFF8600B467A60FB727B6803F500734B
S315080307B01A78B54B1B78D31A002B12D17B6803F52D
S315080307C000731846EFF788FE0346012B09D1AF4895
S315080307D024F044FFAE4824F041FFAE4824F03EFF20
S315080307E04FE27B6803F500730B22AB49184645F0C5
S315080307F041FC0346002B40F0C5817B6803F5007373
S315080308001846EFF769FE03460B2B40F0BB817B685E
S3150803081003F580630922A149184645F02BFC0346D4
S31508030820002B6FD17B6803F580631846EFF754FEF8
S315080308300346092B66D17B6803F5C0631A78984B80
S315080308401B78D31A002B08D17B6803F5C0631846B7
S31508030850EFF742FE0346012B13D07B6803F5C0630B
S3150803086002229049184645F005FC0346002B13D18E
S315080308707B6803F5C0631846EFF72EFE0346022B83
S315080308800AD113F007F903460121184613F0F7FABC
S31508030890854824F0E3FE34E07B6803F5C0631A78E1
S315080308A0824B1B78D31A002B08D17B6803F5C063E8
S315080308B01846EFF711FE0346012B13D07B6803F5A1
S315080308C0C06303227A49184645F0D4FB0346002B36
S315080308D013D17B6803F5C0631846EFF7FDFD03469E
S315080308E0032B0AD113F0D6F803460121184613F051
S315080308F0E3FA704824F0B2FE03E06F4824F0AEFE34
S31508030900BFE13EE17B6803F5806309226B4918461C
S3150803091045F0B0FB0346002B6FD17B6803F5806374
S315080309201846EFF7D9FD0346092B66D17B6803F50D
S31508030930C0631A785A4B1B78D31A002B08D17B68E5
S3150803094003F5C0631846EFF7C7FD0346012B13D01B
S315080309507B6803F5C06302225249184645F08AFBB1
S315080309600346002B13D17B6803F5C0631846EFF7DC
S31508030970B3FD0346022B0AD113F08CF80346022172
S31508030980184613F07CFA4E4824F068FE34E07B6878
S3150803099003F5C0631A78454B1B78D31A002B08D185
S315080309A07B6803F5C0631846EFF796FD0346012BEC
S315080309B013D07B6803F5C06303223D49184645F007
S315080309C059FB0346002B13D17B6803F5C06318460E
S315080309D0EFF782FD0346032B0AD113F05BF80346B0
